:1000000000800020BD01000069A8000021A80000B8
:1000100021A8000021A8000021A8000021A80000BC
:1000200021A8000021A8000021A8000069A8000064
:1000300069A8000021A80000E99E0000ED9F0000D3
:1000400069A8000069A8000069A8000069A800006C
:1000500069A8000069A8000069A8000069A800005C
:1000600069A8000069A8000069A8000069A800004C
:1000700069A8000069A8000069A8000069A800003C
:1000800069A8000069A8000069A8000069A800002C
:1000900069A8000069A8000069A8000069A800001C
:1000A000258400003184000069A8000069A80000D0
:1000B00069A8000069A8000069A8000069A80000FC
:1000C00069A8000069A8000069A8000069A80000EC
:1000D00069A8000069A8000069A8000069A80000DC
:1000E00069A8000069A8000069A8000069A80000CC
:1000F00069A80000D5C8000069A8000001CA000076
:1001000069A8000041B2000069A8000069A80000C9
:1001100069A8000069A8000069A8000069A800009B
:1001200069A8000069A8000069A8000069A800008B
:1001300069A8000069A8000069A8000069A800007B
:1001400069A8000069A8000069A8000069A800006B
:10015000D9A00000EDA0000001A1000015A1000041
:1001600069A800005DB5000069A8000069A800004A
:1001700069A8000069A8000069A8000069A800003B
:1001800069A8000069A8000069A8000069A800002B
:1001900069A8000069A8000069A8000069A800001B
:1001A00069A8000069A8000069A8000069A800000B
:1001B00069A8000069A8000069A80000564B4CF22D
:1001C000205210B51A804DF628121A8000BF00BFC9
:1001D0000AF04EFB514B4FF010621A60504A9A6081
:1001E000504ADA60504A136813F4807304D14F49BF
:1001F0000B604FF4A85313604D4B1A78110703D5C9
:100200001A7842F008021A704A4B4B492A221A7097
:100210004A4A4B4B8B4204D252F8040F43F8040B6A
:10022000F8E7484B484900228B4202D243F8042B9E
:10023000FAE74649464A002352F8230041F82300D2
:1002400001336F2BF8D1434B434A802103F8011B44
:100250009342FBD1414B3D4A1A60414B8A221A70AE
:10026000A3F5805324225A70A0221A709A7992071B
:10027000FCD59A79D406FCD43A4A937903F00C035E
:10028000082B384BF9D103221A7140225A719A79FE
:100290009006FCD5334A9179324B4906FBD5324A58
:1002A000324911600221516020221A709A7902F0BD
:1002B0000C020C2AFAD12E4B2E4A1A602E4B2F4AD2
:1002C0001A6000225A60072243F8042C2C4AC3F813
:1002D0000C2D62B60AF07CFE144B1B68DA0705D5BC
:1002E00028480AF049FC284B284A1A60284B1B78FA
:1002F0005B0609D5244C254B22689A4204D121483B
:100300000AF03AFC002323600DF032FE0AF0B6FA40
:100310000AF0E4F9FEE700BF0E20054030800440FB
:10032000823F04000100002B10D0034014D0034092
:1003300002D0074000E007401C9BFF1FB40E0100E5
:100340004088FF1F1C9BFF1F04A3FF1F0082FF1F8D
:100350000000000000E400E05FE400E008ED00E0E1
:100360000050064000400640448004400000030165
:1003700004800440C010050014E000E0FF76010096
:10038000000020202D6EC15E1CE00340A5C3945ADE
:1003900000F00740FFFFFFFFFFFFFFFFFFFFFFFF32
:1003A000FFFFFFFFFFFFFFFFFFFFFFFFFFFFFFFF5D
:1003B000FFFFFFFFFFFFFFFFFFFFFFFFFFFFFFFF4D
:1003C000FFFFFFFFFFFFFFFFFFFFFFFFFFFFFFFF3D
:1003D000FFFFFFFFFFFFFFFFFFFFFFFFFFFFFFFF2D
:1003E000FFFFFFFFFFFFFFFFFFFFFFFFFFFFFFFF1D
:1003F000FFFFFFFFFFFFFFFFFFFFFFFFFFFFFFFF0D
:10040000FFFFFFFFFFFFFFFFFFFFFFFFDEF9FFFF23
:1004100010B5054C237833B9044B13B10448AFF33E
:1004200000800123237010BD1C9BFF1F00000000F3
:10043000B80E0100084B10B51BB108490848AFF3CE
:1004400000800848036803B910BD074B002BFBD0A0
:10045000BDE81040184700BF00000000209BFF1FB0
:10046000B80E01001C9BFF1F0000000038B50446B9
:10047000104621700A491D460DF05CFB01464FF005
:100480007E500DF00BFC07490DF054FBE5606060F9
:10049000256165610AF02CFDE061204638BD00BF92
:1004A000DB0FC9400024744938B50446104621705A
:1004B00009491D460DF03EFB01464FF07E500DF000
:1004C000EDFB06490DF036FBE56060602561656176
:1004D0000AF00EFDE06138BDDB0FC940002474490D
:1004E00038B503780446032B20D8DFE803F01A1848
:1004F0001002C16840690DF013FA0D4905466068A5
:100500000DF0CCFB014628460DF0C8FB38BD08496C
:1005100040680DF0C3FBE1680DF00CFB38BDC0680E
:1005200038BDC16840690DF0FBF938BD002038BD09
:100530000024744970B504460E460AF0D9FC0546FD
:10054000E069281A0DF0A2FAE3682361E5616661AB
:10055000A061014660680DF0A1FB0146A060104853
:100560000DF09CFB0CF072FE0CF012FB0DF084F908
:10057000054601464FF07E500DF0D2F961690DF04D
:10058000D9FA2169064628460DF0D4FA01463046CC
:100590000DF0C8F9E0602046BDE87040FFF7A0BF4D
:1005A000000080BF38B50E201C4C09F071FF218877
:1005B0001B4B884205461A881DDA0023511AB1F5F3
:1005C000805FAABF1B03C3EB03330131142093FBED
:1005D000F1F10AF0E3FA134B1988F1B923889D422F
:1005E00010DAC3F57F630F33282091FBF3F1BDE8E8
:1005F00038400AF0D3BA9042D4BFC1EB0003C1EB3C
:100600000203DBE740F6FF718D42D4BFC3EB050167
:10061000C3EB0101C1EB0131E3E738BDFA9BFF1FDA
:10062000A09DFF1F4C9DFF1F10B5044609F032FD31
:10063000204610BD70B44C88A04220D9012301335C
:10064000DBB21CB2660031F8144084421D46F6D37A
:10065000A04211D005F10045013D965B31F815101F
:1006600032F81530401AF21A00FB02F0641A90FBBF
:10067000F4F4E01870BC7047905B70BC70470226C1
:100680000125E5E700280CDA064A434282FB0320F5
:10069000DA17C2EB600000EB4000A3EB8000C0F172
:1006A0000C007047ABAAAA2A2DE9F0470C2009F0EC
:1006B000BBFE0C200AF070FBA04914200AF07CFB62
:1006C0009F49A04807F0B4FB022103200AF00AFC6E
:1006D000022104200AF006FC022105200AF002FC97
:1006E000022106200AF0FEFB01210A200AF0FAFB93
:1006F000012109200AF0F6FB01210D200AF0F2FB8E
:10070000012128200AF0EEFB012114200AF0EAFB67
:10071000012116200AF0E6FB172001210AF0E2FB76
:1007200004200AF0D1FB002833D005200AF0CCFBCE
:100730000446002834D000242046834D287004F05D
:1007400041FF2D780DBB204606F052FB7F4B8049C0
:100750001B88804C098821707F4A804EA3F5AF71B9
:1007600040F23A7303FB01F382FB0312DB17A3EBA6
:100770006213323301210D2033600AF09FFB5D21AB
:10078000774807F0FFFE90B9FEE7BDE8F04707F0B5
:100790005FBA06200AF098FB0028C6D10124CCE7F6
:1007A00003200AF091FBB0FA80F04009C5E75C2114
:1007B0006C4807F0E7FE00B9FEE75B216A4807F0E6
:1007C000E1FE00B9FEE729460D200AF077FB674AF3
:1007D00067481268DFF8E8A1DFF8A091654EDFF8FE
:1007E000E481654F00230121FFF75EFE0123C9F874
:1007F00000503560C8F800508AF8003004250F20FA
:100800000AF08AFDD8F8003003440E20C8F8003002
:1008100009F03EFED9F800309AF800200344C9F8E8
:1008200000301520002A78D009F032FE33681844D1
:10083000306005F0010080F0010003F0D9FD3B8835
:10084000002B14BF4B20FA200AF074FB013DD6D1D7
:10085000D8F80030D9F80020484930683D88DFF8E2
:1008600068E1474F002BB8BF0333002AB8BF0332FB
:1008700092100A604349444A098812880028B8BF88
:1008800003309B10801030605E1A19443E60CEF831
:1008900000103E4F3E4E3F49C8F80030C2EB000EFC
:1008A0000244C7F800E032600B605DB94FF4FA70A3
:1008B00003F0AEFD03F098FD05F078F94FF4AF605A
:1008C0000AF038FB344B012504201D600AF0FCFAC5
:1008D00010B9324B20701D70314B1B881C2B23D05C
:1008E000304C04F1C805232009F0D2FD44F8040F70
:1008F00001200AF01FFBA542F5D12B4A2B4B1078A3
:10090000187006F07FF903F06BFD45F6BF522849D9
:100910002848BDE8F04709F073BB11200AF0FCFC41
:1009200033681844306084E7234B18880028D7D0F8
:10093000224BC0B2197806F0ADF8D1E7001B37465C
:10094000801A06002490FF1F719BFF1F9C9DFF1FB4
:10095000109DFF1FC49BFF1FB5814E1BC489FF1F45
:10096000709BFF1FF89BFF1F9C9BFF1F2489FF1F8D
:10097000149DFF1F389BFF1F429DFF1F509BFF1FB1
:10098000689DFF1FD689FF1F2C89FF1F909BFF1FAB
:10099000C89BFF1FB09DFF1F709DFF1F5F9BFF1F28
:1009A000769DFF1F049CFF1FFC9CFF1FE19CFF1F07
:1009B000A5050000949DFF1FCC9BFF1F889BFF1F78
:1009C0005C9DFF1F649DFF1FE49CFF1FF0B40E8819
:1009D00086420DD203F10043013B31F813508542AA
:1009E00002D9F0BCFFF726BE32F81300F0BC704706
:1009F0001088F0BC704700BF094B1B880C2B09D82E
:100A0000084A80B252F8232028B143F6FE73984278
:100A100003D9108C7047108870470349FFF70ABE4E
:100A20006C9BFF1FA4F000008CF10000374A38498E
:100A30001088384AF8B5384B12881B68834248DB67
:100A40009342A8BF134698420B60C8BF002342DD03
:100A5000101AB0F5804FAABF9B03C3EB833301305C
:100A600093FBF0F0FFF7C8FF2C4B2D4F1C883B6821
:100A7000C0F3C61505FB04F47F2CA8BF7F249D425C
:100A8000064608D0274B1B88002B38D1264B1B88E5
:100A9000002B30D13D60254D2B689E4205D0214B67
:100AA0001B885A1F032A1DD92E60214D2B689C429A
:100AB0000ED0204B188848B11A4B1F4A1B88D35CB4
:100AC000834203D0C0B2E1B205F0E4FF2C60F8BD70
:100AD000F8BD034608609A42D4BFC0EB0203C0EBE6
:100AE0000303B5E7144AD05C2030C0B206F07F01A2
:100AF00005F0D0FFD8E7284606F040F8CAE70E4ACE
:100B00002946D05C05F0C6FFC0E700BFFA9BFF1F77
:100B1000409BFF1FA09DFF1F489DFF1F549BFF1F71
:100B2000A49BFF1F389DFF1FF29BFF1FA89DFF1F67
:100B3000F49BFF1F7A9DFF1FC889FF1F2DE9F04F0F
:100B4000012089B00AF0E8FBAF4B186000200AF0E2
:100B5000E3FBAE4BAE4A1B8810600C2B00F03B81D0
:100B6000AC4BAD4A19880093AC4B52F8214000229F
:100B70001A70AB4BAB4D1B88AB4A2E88013B32F948
:100B80001370002E5CD0A94BA94A1B88A949127882
:100B9000013B31F91380002A40F0DF8011200AF078
:100BA000BBFBA54B0193D3F800A00646B24540F32A
:100BB000DF80A24BDFF8A4921B88A14A012BD9F851
:100BC0000030B2F800B09F4A02922046C8EB0308FA
:100BD00000F09A820CF05AFF029A52F82B100CF097
:100BE000A9FF014600200CF09BFE0DF069F9CAEB4D
:100BF0000802B045B8BFB0469042CAEB080880F280
:100C0000968200FB0888013298FBF2F08E4BDFF8E9
:100C100050820293D8F80030034403EBD3735B1087
:100C2000C8F800302B88012B12D1884BDFF834B282
:100C30000393874BDBF8005004934FF0000A47E022
:100C40007D4B0193DFF814927F4BDFF814820293FF
:100C50007E4B03931D460F200AF05EFB2B689842E3
:100C6000824641DA754A1288012A00F01D82744AD0
:100C700005931288734D049220460CF007FF049AE6
:100C8000DFF8E0B155F82210DBF800500CF052FF0D
:100C9000014600200CF044FE0DF012F9EF1B059BFD
:100CA0005745A7EB0302B8BF5746FF1A9042BABF99
:100CB000013200FB0777474397FBF2F7D8F8002093
:100CC000634B0493BB1803EBD3735B10C8F800307D
:100CD000604B1B88013B032B00F2B082DFE813F06E
:100CE0006301A901C4008601594B04931B68984213
:100CF00040F3C281514A1288012A00F0A682504A6C
:100D0000079311884F4A0691204605920CF0BEFECB
:100D1000059A0699DFF84CB152F82110DBF8005023
:100D20000CF008FF0DF0CCF8079B2F445745A7EBBC
:100D30000302A8BF5746FF1AD8F800309042BABF46
:100D400000FB07770132474397FBF2F73B4403EB85
:100D5000D3735B10C8F80030BAE7152009F098FB90
:100D6000354B0193D3F800A00646B2453FF721AFBB
:100D7000354B0293D3F800A0B24580F289812F4B06
:100D8000DFF8D8901B882E4A012BD9F80030B2F832
:100D900000B02C4A03922046984400F070820CF078
:100DA00075FE039A52F82B100CF0C4FE0DF088F873
:100DB000B045CAEB0802A8BFB046CAEB080890428B
:100DC000B6BF00FB088800FB08F8013298FBF2F080
:100DD000DFF88C801EE7204B1B78002B3FF4C0AE61
:100DE0000C4B0D4A198800930C4B52F8210001223C
:100DF0001A700CF04BFE4FF07C510CF09BFE0DF086
:100E00005FF80446B5E600BF989BFF1F769DFF1F65
:100E1000BC9DFF1F9E9BFF1F8C89FF1F469BFF1FD2
:100E2000D489FF1FEA9CFF1FD8F20000248AFF1F0D
:100E30005C9DFF1F68F10000909BFF1FE09BFF1F60
:100E4000689BFF1FF0F20000C89BFF1F689DFF1FFB
:100E5000E49CFF1F6089FF1F5E9BFF1F389BFF1FE5
:100E6000809DFF1F649DFF1F28460CF00FFEB249B6
:100E70000CF060FE054650460CF008FEAF490CF041
:100E800059FE014628460CF04DFD0DF019F80546B7
:100E9000CBF80050D9F800000CF0F8FDA6490CF092
:100EA00049FE074630460CF0F1FDA4490CF042FE25
:100EB000014638460CF036FD0DF002F8C9F8000086
:100EC0009F4AA04B168819889F4AA04B12681B881E
:100ED0009F4FC6EB050E3544039EC6F800E0461A48
:100EE000084404990D6001990E6002993E880860DB
:100EF0009A4280F289810025C3EB060E954974451C
:100F00000F6880F27681611C9F4205FB01F50EF1AE
:100F1000010E95FBFEF5C0F2BE81BE42A8BF3E4663
:100F2000F61A01FB06F494FBFEF49A4200F33681B4
:100F3000BB42C0F23381884C20680CF0A7FD874982
:100F40000CF0F8FD86490CF0EDFC0CF0B9FFA0F5B3
:100F5000FF531C3B082B98BF4FF40050D8F80030CB
:100F6000184400282060C0F24281B0F5804F80F222
:100F700052817C4B1B781BB1B0F5005F40F0538170
:100F8000794D2B78002B40F05481784D20682B68E8
:100F9000714C984204D080B205F05AFE23682B6051
:100FA00009B0BDE8F08F28460CF070FD70490CF0D8
:100FB000C1FD054650460CF069FD6E490CF0BAFDC6
:100FC000014628460CF0AEFC0CF07AFF0546CBF843
:100FD0000050D9F800000CF059FD65490CF0AAFD4D
:100FE000074630460CF052FD62495FE728460CF098
:100FF0004DFD5A490CF09EFD054650460CF046FD4D
:101000005D490CF097FD014628460CF08BFC0CF076
:1010100057FF0546CBF80050D9F800000CF036FD1C
:101020004E490CF087FD074630460CF02FFD524923
:101030003CE728460CF02AFD50490CF07BFD0546A4
:1010400050460CF023FD4E490CF074FD0146284635
:101050000CF068FC0CF034FF0546CBF80050D9F8D2
:1010600000000CF013FD45490CF064FD07463046C6
:101070000CF00CFD424919E7D8F80030DFF810B148
:1010800003EBD3735B10DBF80050C8F800301FE6A9
:10109000DFF80081DFF80091D8F8003003EBD3735C
:1010A0005B10C8F80030BDE5364A06931188364A11
:1010B000059120460492DFF8D8B00CF0E7FC049AC2
:1010C0000599DBF8005052F821100CF033FD0CF0BC
:1010D000F7FEEF1B069B5745A7EB0302B8BF574629
:1010E000FF1AD8F800309042BABF013200FB0777F0
:1010F000474397FBF2F73B4403EBD373234A049235
:101100005B10C8F80030E3E50CF0C0FC029A52F81E
:101110002B100CF00FFD0CF0D3FECAEB0802B0450B
:10112000B8BFB0468242CAEB08083FF76AAD00FB81
:1011300008F898FBF2F069E5CDCC4C3FCDCC4C3EA5
:10114000D689FF1F2C89FF1F989BFF1F469DFF1FFD
:10115000809BFF1FBC9DFF1FC089FF1F9A99193FED
:10116000CDCC4C45739EFF1FF09BFF1F2089FF1FB6
:101170003333733FCDCC4C3DCDCCCC3E6666663F21
:10118000CDCCCC3D689BFF1FF0F20000E49CFF1F1C
:10119000649DFF1F809DFF1F389BFF1F009B1B88C6
:1011A000002B3FF4C8AE2B1B002BB8BF5B42092BB2
:1011B00047DD05F500500130001B0CF067FC3B4992
:1011C0003B4C0CF0B7FC054620680CF05FFC39493D
:1011D0000CF0B0FC014628460CF0A4FB0CF070FEAD
:1011E000D8F80030184400282060BFF6BEAE0022B8
:1011F00013E09F4205FB04F5B8BF002195FBFEF507
:101200004BDA91FBFEF490E6B242D4BFC3EB020589
:10121000C3EB060570E643F6FF72274B22601B788E
:10122000002B3FF4ADAE03F0DFF8244B01221A701F
:10123000ABE603F0D5F800232B70A6E6D9F8000042
:101240003EE64FF400501A4C88E61D491D4A0693AD
:1012500020460D8805920CF019FC059ADFF868B05D
:1012600052F82510DBF800500CF064FC0146002019
:101270000CF056FB0CF024FE2F44069B56E50CF0B8
:1012800005FC039A52F82B100CF054FC0146002088
:101290000CF046FB8AE51E4642E6B742D4BFC3EBDC
:1012A0000701C3EB060104FB01F1AAE7CDCCCC3E5C
:1012B000C089FF1F9A99193F739EFF1FF09BFF1F64
:1012C000689BFF1FF0F20000649DFF1F38B5114CB2
:1012D0002320257809F0DCF80F4A42F82500131F77
:1012E00002F1C400002253F8041F83420A44FAD1D9
:1012F00023780A4907480A4C0133DBB2322B81FBC1
:10130000025108BF0023D217C2EB211203702260E2
:1013100038BD00BF569BFF1F089CFF1F1F85EB5168
:10132000609DFF1F2DE9F0479F4CA04D206882B0C3
:101330000CF0ACFB9E490CF0FDFB0646102009F0BA
:10134000EBFF0CF0A3FB9B490CF0F4FB31460CF0D7
:10135000E9FA0CF0B5FD2B882060192B00F0CA804B
:101360001A2B00F0F5801E2B00F0FB8001252E4685
:10137000914A1188002900F09180904B904A1B8877
:101380001288834240F3DD800020D31A8B42C6BF0F
:1013900001FB00000133484390FBF3F3894A1360DB
:1013A000894F388848B9894B1B8833B9884A1178E6
:1013B00001B1137002B0BDE8F087DFF80082216848
:1013C000B8F80030784A8B426EDCDFF804E29EF811
:1013D0000090B9F1000F2FD14FF0010C04288EF8C6
:1013E00000C029D1002D40F07181784B1888002869
:1013F000E0D0002EDED02368B8F80040704AA34247
:10140000128880F23E810023141B7E2C714DD5BFC3
:10141000C3EB8313C3EBC3135B00013493FBF4F4FE
:101420002B680134A34203D0C0B2E1B205F032FB15
:101430002C6002B0BDE8F087012800F0D5800228BA
:1014400000F0A9800328D0D1634B1B88092BCCD096
:10145000002DCAD02368B8F80050594AAB42128810
:1014600080F25C810023551B7E2DDFF874A1D5BF6F
:10147000C3EB8313C3EBC3135B00013593FBF5F59B
:10148000DAF800300135AB4203D0E9B24A2005F06A
:1014900001FBCAF80050A8E70D460E461E2B7FF44C
:1014A0007FAF00214D4F64E0494B1A78002A81D06C
:1014B000002401281C7062D0022840F0E980002D31
:1014C00063D0474D2B68002B5FD00420214605F0E8
:1014D000E1FA3E4B2C60188800283FF46BAF002ED9
:1014E0003FF468AFC0B2002105F0D4FA394B0022B6
:1014F0001A605FE7394F3B4E3A7872B13349098839
:1015000059B196F800E0964542D0C8B27F2105F067
:10151000C1FA3A782B8832700AE03178914237D09C
:101520002A4B0021187805F0B5FA3A782B883270EA
:10153000214A11880029AFD000251E2B2E4618D035
:101540001BE08242D4BFC3EB0200C3EB00001CE7E8
:10155000224F3A78002A0BBF0125002500260126DC
:1015600006E71E4F144B3D781988B5FA85F56D09CD
:1015700000263B78002B3FF411AF2068FDE625B133
:10158000174D2B68002B40F09A80104B1888A3E76A
:1015900000252E46ECE6002D3FF427AFDFF840A0F3
:1015A000074ADAF800304AE08C9BFF1F769DFF1F48
:1015B0009A99193FCDCCCC3EA49DFF1FF49CFF1FF0
:1015C000EE9CFF1F009CFF1F969BFF1F889DFF1F27
:1015D0007D9DFF1F749BFF1F389DFF1F5E9BFF1F9C
:1015E000049CFF1F5B9BFF1F002D3FF4FEAE534A80
:1015F00010888842D4BFC3EB0009C3EB0109C31AAA
:101600007E2B40F38280C9EBC91103F1010991FBE4
:10161000F9F909F10109DFF82CA1DAF800304B459E
:1016200006D05FFA89F10120019205F033FA019AA0
:101630003888CAF8009002287FF404AF4B4621682E
:10164000B8F800901088494558DA0022C9EB000923
:10165000B9F17E0FD3BFC2EB8212C2EBC21209F105
:101660000109520092FBF9F909F10109994504D0E9
:101670005FFA89F1042005F00DFA3888CAF8009065
:10168000E0E69342D4BFC4EB0303C4EB0203BBE622
:10169000032828D12A4B1B88092B3FF476AF002D55
:1016A0003FF473AF274D2B68002B3FF46EAF4A20F9
:1016B000214605F0EFF9244B2C6018880CE72146F1
:1016C00005F0E8F9204B2C60188805E740207F21C1
:1016D000019205F0DFF93888019A012825D0022807
:1016E0007FF4B0AE5AE704287FF44FAF002D3FF4EB
:1016F0004CAF2146402005F0CDF946E78142D4BFEA
:10170000C9EB0102C9EB0002A0E7C9EB89194FEA56
:10171000490999FBF3F909F101097CE79342D4BF28
:10172000C5EB0303C5EB02039DE61168B8F8003072
:10173000024A99421088FFF662AF5AE7EE9CFF1FFB
:10174000389DFF1F049CFF1F889DFF1F08B50F4B8E
:101750001B88022B0FD0032B12D0042B03D00C4B71
:1017600001221A7008BD7F21092005F093F9084B6A
:1017700001221A7008BD7F21412005F08BF9EEE7A8
:101780004021092005F086F9E9E700BFFE9BFF1F15
:10179000B79BFF1F38B51C4B1B881D2B26D01B4B3E
:1017A0001B88012B25D01A4A1A4B14881B681A4A29
:1017B000A342128818DB9342D4BFC4EB0303C4EBEB
:1017C0000203141B7F2CC6BFDB010134C3EBC31320
:1017D00093FBF4F4114D2B689C4203D0E1B2052039
:1017E00005F058F92C6038BD0023EAE70C4B1C8843
:1017F000F0E70C4B0C4A0D491B6812680C689B1AE9
:101800001C1B84F30704E5E7769DFF1FEA9CFF1F7E
:10181000B29BFF1F4C9BFF1F749DFF1F909DFF1FDE
:10182000889BFF1FB09DFF1F2889FF1FF89CFF1F8B
:1018300010B50F4C23685BB90E4B1B88022B11D0DF
:10184000033B012B09D90C4A00231370236010BD00
:101850000021052005F01EF9EEE70021092005F022
:1018600019F9F0E70021412005F014F9EBE700BF7A
:10187000909DFF1FFE9BFF1FB79BFF1F08B5274BC7
:101880001B78ABB1152008F003FE254A254B1288C2
:1018900018601D2A15D0244A1288EAB1012A25D0E1
:1018A000224B1B78002B34D0BDE80840FFF7C0BFA7
:1018B000112009F031FD1A4A1A4B128818601D2AAE
:1018C000E9D11B4B1B78002BEAD0184B1B780BB3CC
:1018D000BDE80840FFF75EBF164A1288002ADFD035
:1018E000154A1B6812889A42DADCEEE70F2009F0ED
:1018F00013FD104B114A1B88106033B1104B114A75
:101900001B6812689B1A9842DFDD084B1B78002B7E
:10191000CAD108BDFFF71AFFDAE700BF5C9DFF1FC1
:10192000769DFF1F4C9BFF1FEA9CFF1FB79BFF1F6D
:101930005E9BFF1FFE9BFF1FB29BFF1FF89CFF1FBC
:10194000B09DFF1F2889FF1F2DE9F04FDFF82CB352
:101950009BF80060012E93B000F02B82C0F0FD8157
:10196000022E00F0C7809D489D4B9E4DDFF800E39E
:101970009D4A9E499E4F9F4C009400789E4C1B7838
:101980002D789EF800E01278097897F800A0DFF82B
:10199000F0C2DFF8F082DFF8F0920194012E974C4C
:1019A00094BF0136002622708BF80060944C954E4F
:1019B00023703070944C954E21703570944C954E38
:1019C00084F800A03270BEF1000F40F0F980924C14
:1019D00024880D2C00F09B81DFF89CE20024264631
:1019E0008EF80040A3462BB18B4B1C88002C40F096
:1019F0009B812346894C248803EB0B0E002C40F07E
:101A00004581874B874C1B7899F8009024780133E7
:101A1000A3EB4903002C40F08A81019C2478C4EB9D
:101A2000030B002C40F043820023DFF840927E4CF1
:101A300099F800902478C3EB0B03A3EB49032B44E4
:101A4000181A002C00F08781B5FA85F56D099CF80D
:101A500000300544ED1A002B00F07B8119F10000E5
:101A600018BF0120009C98F8003027786F4C281A86
:101A7000C31AA3EB47030B449B1A21786C4A6D4CA5
:101A8000A3EB4A034FF00C0A1AFB013313602268E0
:101A900069496A4D09886A486A4F2D8800883F68FD
:101AA000033901EB4101C5EBC50503EB810101449D
:101AB0003D4465480C3950F825008E440EEB00017A
:101AC0000EB162480360914200F01D81604B614895
:101AD0001A680592059A02601B6806935E48069B89
:101AE000008821609B1A834284BF5C4B196013B04D
:101AF000BDE8F08F5A4F06AE0025E9B2594806F00E
:101B000005FD57F8043B0135C01A0C2D46F8040BAF
:101B1000F3D1554B079FB3F800C00E9B0D9E0F9D50
:101B20001098354C01946345ACBF4FF0000E4FF058
:101B3000010EBC45D4BF00270127B445D4BF002601
:101B40000126AC45D4BF4FF000084FF00108119BAF
:101B500084F800808445454C4549324ADFF8289195
:101B60001770D4BF4FF0000A4FF0010A9C45099B43
:101B700084F800A01B4C81F800E0D4BF00250125AB
:101B80009C450A9B2570154C154F174A89F8006033
:101B9000D4BF00200120164E144920709C45D4BFAC
:101BA00000230123134C96F800A03B7012780978AB
:101BB0009BF80060DFF8C8C0DFF8C8800094EDE64D
:101BC0002C4E2D4CB6F800B00126BBF1180F267034
:101BD00040F2BB804FF0000B05E700BFB59BFF1F35
:101BE000B69BFF1FB49BFF1F359DFF1F349DFF1F3A
:101BF000369DFF1F799DFF1F849DFF1FC19DFF1F05
:101C0000C39DFF1FC29DFF1FC59DFF1FC49DFF1FDA
:101C10007C9DFF1FC69DFF1FC89DFF1F449BFF1F8C
:101C2000D889FF1FB49DFF1F9E9DFF1FE99CFF1FCA
:101C30003C9DFF1FAC9BFF1F509DFF1F6C9DFF1F16
:101C4000589BFF1F009CFF1F18F30000849BFF1F81
:101C5000B09EFF1FD09BFF1F869DFF1FB89DFF1FDB
:101C60003089FF1FF89BFF1F9C9DFF1F8C9DFF1F4E
:101C7000C79DFF1F769DFF1F5E9BFF1FE09CFF1F00
:101C8000C09DFF1F789DFF1F8B9DFF1F012C00F043
:101C90007981022C00F0DA81032C9E4B00F00D813B
:101CA0001D78009B9CF800B0197899F800209A4B99
:101CB000019C98F8008093F800C02778A5EB4B05AD
:101CC000A1EB8104C2EB8273C8EB05012144C2EB96
:101CD00083028B1803EB4C0303EB8A0A27B18F4B6B
:101CE0001B78002B40F04E8201238D4A8D4C1178D9
:101CF0008D482268C1F10601534401EB410103EB19
:101D000081030360C4E6894A894B1268E4E6002B2C
:101D10003FF462AE874E884FB6F800B00126BBF1A3
:101D2000180F3E7011D9F346A4F10D0362E6019C31
:101D30002478B9F1000F40F09E80013BC4EB030B07
:101D4000002C3FF471AE4B466FE6ABF10C0B012655
:101D500049E6184686E6254679E6784F06AE002520
:101D6000E9B2774806F0D2FB57F8043B0135C01AB8
:101D7000062D46F8040BF3D1724A0B991288684B72
:101D8000002091421870C0F283800A998A4240F381
:101D9000DA816D486D4A6E4990F800A01278097892
:101DA000DFF8D4C1DFF8D48105201870694B0093A7
:101DB00051E0694F06AE0025E9B2684806F0A6FB7F
:101DC00057F8043B0135C01A0C2D46F8040BF3D12B
:101DD0005C4B099C18880A9F4F4B0E9ADFF89C8138
:101DE000DFF894C106A962C98442ACBF4FF0000974
:101DF0004FF00109B842D4BF00270127B042D4BF39
:101E00000026012683F80090A842524B0093D4BFCD
:101E10000025012588421D70D4BF002101214B4BB4
:101E20000D9C88F800609042D4BF002201221A70F5
:101E3000109B474E444D8CF80070A042D4BF4FF029
:101E4000000A4FF0010A9842317085F800A019DCB1
:101E5000002343480370434E4348444B444D454C94
:101E600096F800E000781B782D789BF80060DFF88A
:101E70001091019492E5002C40F07B8103F1FF3B2F
:101E80002346D2E50F9B9842D4BF00230123E0E70D
:101E90002E4A2F492C481D702E4B1278097890F845
:101EA00000A0DFF8D4C0DFF8D4800093D3E7B9F105
:101EB000000F3FF4B9AD0123B7E51978009B9CF8FA
:101EC00000C01A7898F8008099F80030124D019CF3
:101ED0002D782478A1EB4C01C8EB0108A2EB82021B
:101EE000C3EB83714244C3EB8103134403EB45030B
:101EF00003EB8A0A002C40F049810120084B0A4A72
:101F00001B78084C82440C2111FB03A31360226848
:101F1000BEE500BFD889FF1F9E9DFF1F8C9DFF1F40
:101F2000E99CFF1FAC9BFF1F3C9DFF1FD09BFF1F29
:101F3000B09EFF1F769DFF1F5E9BFF1F0C8AFF1F39
:101F4000709BFF1F9C9DFF1F369DFF1F359DFF1F30
:101F5000349DFF1F799DFF1FDC89FF1F9C9BFF1F86
:101F6000829BFF1FC79DFF1FB59BFF1FB69BFF1FD7
:101F7000B49BFF1F849DFF1FC09DFF1F789DFF1F07
:101F80008B9DFF1FAD4BDFF8E4B21F7899F800304E
:101F90009BF80090029307F1010BABEB43031F4644
:101FA000B9F1000F40F0B380019C94F800B0C9EB88
:101FB0000703CBEB03030193BBF1000F40F0BB80A1
:101FC0005B469F4CDFF88C92247803942746019C53
:101FD00099F80090E31AA3EB49032B44181A002F39
:101FE00000F0A480B5FA85F464099CF8003004443C
:101FF000E41A1BB119F1000318BF0123009898F8E7
:1020000000500078E31A5B1BA3EB40030B449B1AC0
:10201000029AA3EB4A03002A40F09280BBF1000F22
:1020200040F0C2805B4400287ED1BAF1000F0CBFA3
:1020300000226FF00902834883490078834C1A44D8
:102040000C2313FB00230B60226821E5019C804BCD
:1020500024780194009CDFF814B227787D4C98F81E
:102060000080247800949CF800C099F800909BF8B8
:1020700000B09DF8044083F806805A72DFF8F081C2
:102080009DF8002083F805C0DA709C7083F80090FA
:102090001D71DF71197283F80AA083F801B04FF047
:1020A000000C012200236A4F194645464C4607E0C2
:1020B000022A09D00B2B0BD017F8014F15F8012F6E
:1020C000944203F10103F3D101310B2BC9B2F3D1D7
:1020D0000A2907D80CF1010CBCF1110F4CD018F8EB
:1020E0000B2FDFE7554A5C4B1478554953F82C20E9
:1020F000544B09781B78544D01342244101A08447B
:102100000C22524C12FB03032B602268C0E4029B9A
:10211000002B44D0019B93F800B0BBF1000F07D116
:102120007B1E01935B464CE7002284E7039C5CE73F
:10213000CBEB07030193029B003318BF012340E759
:102140004FF0000B6EE709998A4235DC08998A4204
:1021500042DD4248424A434990F800A0127809788B
:10216000DFF810C1DFF81081032018703E4B009398
:1021700071E6C4EB030B9EE6344C334B22681A60C5
:10218000134685E4031C18BF0123AEE5314B1B78D1
:10219000002B3FF4B2AE003018BF0120AEE6019B29
:1021A000A14693F800B002E7B9F1000F0CBF4FF061
:1021B000000B4FF0090B35E72848294A294990F8C8
:1021C00000A012780978DFF8ACC0DFF8AC800420FA
:1021D0001870254B00933EE607998A420FDD1F4891
:1021E0001F4A204990F800A012780978DFF884C0CF
:1021F000DFF88480022018701B4B00932BE60699B1
:102200008A42174A17490DDD1448127890F800A049
:102210000978DFF860C0DFF8608001201870124B89
:10222000009318E60D4B127893F800A00E4B097836
:10223000DFF840C0DFF8408000930CE6D889FF1F2C
:102240009E9DFF1FE99CFF1F3C9DFF1FAC9BFF1F36
:10225000D49BFF1F8C9DFF1F3CF00000369DFF1F8D
:10226000359DFF1F349DFF1F799DFF1FB49DFF1FEC
:10227000B0F10000C09DFF1F789DFF1F2DE9F04FBA
:102280002E4B1B788BB0002B53D10E2008F000F999
:102290000BF0FCFB01462A482A4C2B4DFEF74AF96D
:1022A0002748FEF71DF90BF00BFE80F30C002060B1
:1022B000FFF74AFB2E68012E5AD0022E00F08782CB
:1022C000032E00F09783214C2368214A214E099365
:1022D000099B17783068204C07210122181A11FB3E
:1022E00007229042236000F26D821C4E32689A1AD7
:1022F0000D2A00F260821A4E32689A1A132A00F2EE
:102300005582184E32689A1A252A00F23C82164DE0
:102310002A689B1A502B00F2F581144B1B88012B65
:1023200000F00D8204F04AFC04F078FA0BB0BDE82E
:10233000F08F05F015FB0BB0BDE8F08F719BFF1F10
:10234000149DFF1F489DFF1F709DFF1FB09EFF1F24
:10235000E29CFF1FF09CFF1F0C9DFF1FE89BFF1FCF
:10236000BC9BFF1FC09BFF1F009DFF1F4C9DFF1FBD
:10237000DFF800839A4AB8F800001378834204D04B
:10238000C3B21846137004F055FBDFF8E492954A87
:10239000B9F800301178994204D0934F3978002968
:1023A00040F09887914A23681288914C9A42C0F273
:1023B000EE80904A1278002A40F0E980DFF8B8A257
:1023C000BAF8003023B98C4B1B88002B00F04285F3
:1023D0008A4A8B4B11881B888A4A0B4412685B100F
:1023E0009342894A126880F2B78400219342B4BFB5
:1023F00001230B4604910093ACBF4FF0010B8B46B9
:1024000005910E2008F044F8804B814A1B6817683C
:1024100003930133A7F25232002B8446029240F319
:102420006A87802BA8BF80237A4A7B491278019162
:10243000002A00F0B6800978914200F0B280B9F825
:102440000010DFF82CE2994201F061816649AEF894
:102450000030724B4FF0010E81F800E01978DFF880
:102460001CE2019B8EF800101A70009B002B00F0FC
:102470000781BAF80030002B00F00281684B1B681E
:102480005A1C002A40F33B87802A00F33787654EA9
:10249000654966483688098800683144B0EB610FA9
:1024A000C1F20982A3F148020F2A02D8473BA8F8DB
:1024B00000300E2007F0ECFF6FF454731F44874286
:1024C00002DC5B4B00221A705A4B1B88002B00F079
:1024D0003B84594B594A1B781178994240D0002BC4
:1024E0003ED057490E78002E00F0EE87554991F8FE
:1024F00000C0BCF1000F40F0E587534F0097534FE9
:1025000053480297504F007887F800C04F4F4FF064
:10251000010E87F800C081F800E0002841F08981B1
:102520004C490978002901F04A804B4903910E4635
:102530000978002941F040804848444F00783970BC
:1025400001210297317058B13F483E490090002068
:1025500008700099029F0870039901263E70087068
:1025600013703F4B1B88A3F11B02012A40F28D869A
:102570001D2B7FF4A9AE394F3B78002B41F00C8125
:10258000384E3378002B40F0958433709CE62168F8
:10259000354A069106983549106002220B602A6080
:1025A0000CE71E49DFF8D4E0097800293FF459AF61
:1025B0009EF8000081423FF454AF03984B2841F34A
:1025C00052801833802BB9F80000A8BF80239842AE
:1025D0003FF447AF2648038003480123037040E7D8
:1025E000E19CFF1FC49BFF1F5F9BFF1FFA9BFF1F08
:1025F000B09EFF1F6A9BFF1FEE9BFF1F809BFF1F6C
:10260000469DFF1F989BFF1FBC9DFF1F849BFF1FC4
:10261000509BFF1FAC9DFF1FA89BFF1FAD9DFF1F81
:102620003C9DFF1FF49CFF1FEE9CFF1F8C9BFF1F18
:10263000E89CFF1F4E9DFF1F829BFF1F5A9BFF1FA1
:10264000C49DFF1F449DFF1F8A9DFF1FFC9BFF1F12
:10265000C59DFF1FC19DFF1F3C9BFF1F5E9BFF1F72
:10266000769DFF1F5B9BFF1FB89BFF1F089DFF1FF1
:10267000109DFF1FFC9CFF1FB09BFF1FA99BFF1F0E
:10268000029B9C45BFF615AF8E4B1B88002B3FF479
:1026900010AFBBF1000F7FF4F1AE8B4B1B881BB169
:1026A000059B002B7FF4EAAE049B002B3FF401AFA7
:1026B000864B1A78002A7FF4FCAEDFF8888298F8FF
:1026C000006001221A70002E40F09183804B1B782D
:1026D000002B01F032817F4B1B78002B01F04381EE
:1026E0007D4B1B78002B7FF4E4AE7C4B1B78002BDA
:1026F0003FF4DFAEB9F8003079490A3BA9F8003061
:102700000A70D6E602F0A6FF764B1B7873B9764BBB
:102710001B785BB9754B1B7843B9754B1B782BB98C
:10272000744B1B7813B901F05BFE01E001F064FE0D
:1027300023682B60704B1B88012B7FF4F3AD6F4A2D
:102740006F4B11686F481A78A1F118032A2101FB19
:1027500003F10160002A00F0E1826B4A136899429C
:1027600000F37C8380F2868368480068D0F17F00A4
:1027700048BF0330801001301B1A994200F37A835E
:1027800013601946CCE2FEF7A1FD614B1B881B3B91
:102790009BB2022B05D85F4B1B7813B12B68012B22
:1027A00001D001F047FE23683360B0E5FFF766F81B
:1027B00023683360A5E5FEF7C1F9FEF7B3FD236892
:1027C000336098E5FEF732F9236833608DE5524AAD
:1027D00026681288B24204DB464B1B78002B00F0BF
:1027E00064834E4C4E48236807934E4B079900680C
:1027F0001B88091A994200F2AB80002B00F0A880D8
:10280000494B198800293FF45FAD484B48481B6885
:102810000088B342B8BF33469A4241F34580454BE6
:102820001A60DFF8248188F80010344FFEF7FEF8B4
:1028300038687F2840F342863F4B7F3883FB003265
:10284000C317C3EB620303EB4303A0EB83007330B6
:102850003A4B01931B883860002B40F04A87234B8A
:1028600000931B78002B00F07384354E3378002BD7
:1028700000F06E84DFF8D490DFF8BCA04FF0000BBE
:102880000CE003F17300C0B298F8001004F02AF9CC
:1028900033780BF1010B5B4540F35A843B6859F8E0
:1028A000040F1844A0F17F038AFB0321DA17C2EB5F
:1028B000610202EB42027F28A3EB8203E1DCFDF719
:1028C000E1FEE0E7EE9BFF1F049DFF1FE89CFF1F5A
:1028D000C19DFF1FC29DFF1FC39DFF1FC49DFF1F02
:1028E0005F9BFF1FFC9BFF1F449DFF1F8A9DFF1FD7
:1028F0003C9BFF1F6A9BFF1F4C9DFF1FB89DFF1F46
:10290000B79BFF1FE49BFF1F649BFF1F909DFF1F52
:10291000769DFF1F5E9BFF1FFA9BFF1FB09EFF1F50
:10292000B89BFF1FEC9BFF1F5C9BFF1F089DFF1FB9
:10293000A09DFF1F409BFF1FABAAAA2A949BFF1FCD
:102940008889FF1FE99CFF1FE29BFF1F6089FF1F13
:10295000554B56491B6808885549B342B8BF3346A2
:102960009A4200F38982534E09888342A8BF0346E6
:10297000336000297FF455AF9A42C8BF0B4640F33D
:102980008282801AB0F5804FAABF9B03C3EB8333CA
:10299000013093FBF0F0FEF72FF8C0F3C6100BF0F8
:1029A00075F8454B064618880BF070F84349074602
:1029B00030460BF0BFF8014638460BF0BBF8314605
:1029C0000AF0B0FF4FF07E5106460BF051FA002896
:1029D00040F05F873A4930460BF068FA002840F033
:1029E0001C8730460BF092FAC0B2DFF8F48088F80A
:1029F00000001AE7334B26681988B14274DD324B68
:102A00001B78002B70D1DFF8DC9099F800007F284C
:102A100040F3BE86A3F155337F3803F1004383FBB7
:102A20000032C317C3EB620303EB4303A0EB830045
:102A30007330264B01931B88C0B289F80000002B2D
:102A400040F00787224B00931B78002B00F067852E
:102A5000204E3378002B00F062851F4FDFF87C801A
:102A60004FF0000A0AE003F17300C0B204F062F80C
:102A700033780AF1010A534540F3518557F8043F72
:102A800099F800001844A0F17F0388FB0321DA17AE
:102A9000C2EB610202EB42027F28A3EB8203E2DC7D
:102AA000FDF7F0FDE1E700BF089DFF1FA09DFF1FA0
:102AB0005C9BFF1F409BFF1F489BFF1FCDCCCC3D65
:102AC0000000FE42FA9BFF1F6A9BFF1F949BFF1FA3
:102AD0008A9DFF1F8889FF1F6089FF1FABAAAA2A52
:102AE000E29BFF1F409DFF1FA24F38687F2840F3E5
:102AF000D181A14B7F3883FB0032C317C3EB620344
:102B000003EB4303A0EB83007330DFF8B49299F832
:102B100000A0824500F02882984B1B88002B43D1EF
:102B2000974A984812680088914205DC8242D4BFD7
:102B3000C1EB0203C1EB0003411AB1F5804FA6BF00
:102B40009B030131C3EB833393FBF1F0FDF754FF9B
:102B5000C0F3C6100AF09AFF8B4B064618880AF09D
:102B600095FF8A49804630460AF0E4FF0146404618
:102B70000AF0E0FF31460AF0D5FE4FF07E510646DE
:102B80000BF076F9002840F06186814930460BF061
:102B90008DF9002840F0308630460BF0B7F9C0B20E
:102BA000DFF8208288F80000BAF17F0F40F38184BB
:102BB0007148AAF17F0A80FB0A304FEAEA73C3EB3F
:102BC000600000EB4000AAEB80007330714B009373
:102BD0001B78C0B289F80000002B40F0E1836E4BF7
:102BE00003931B78002B40F0AE856C4B02931B784F
:102BF000002B40F051866A4B0193029B1B78002BFF
:102C00003AD0684B1B88182B17D099F80020134432
:102C1000A3F118007F2840F3F285574A973B82FBC7
:102C20000321DA17C2EB610202EB4202A3EB82033B
:102C300003F17300C0B203F07DFF5B4A5B4B127877
:102C400033F81230182B17D099F800201344A3F151
:102C500018007F2840F3DD85474A973B82FB03211C
:102C6000DA17C2EB610202EB4202A3EB820303F12B
:102C70007300C0B203F05EFF009B1B78002B00F0D6
:102C8000AE84019B464E1988002900F055853868AE
:102C90007F2840F35083384B7F3883FB0032C317C3
:102CA000C3EB620303EB4303A0EB83007330386094
:102CB000002940F0E984009B1B78002B00F05F8125
:102CC0003B4E3378002B00F05A81DFF8FCA0DFF890
:102CD000F4804FF0000B0CE003F17300C0B298F8E1
:102CE000001003F0FFFE33780BF1010B5B4540F35E
:102CF00046813B685AF8040F1F4A1844A0F17F032D
:102D000082FB0321DA17C2EB610202EB42027F2849
:102D1000A3EB8203E0DCFDF7B5FCDFE7254B196090
:102D2000254B1B68A92202FB03F3002BBCBF03F554
:102D30007F533F339B13543B194481F30C012820EC
:102D400007F02CFFFFF7EEBA144E1C481149124A47
:102D5000337003700B7003E493424FF0000B80F26A
:102D60009C800123CDF800B0CDF814B00493FFF798
:102D700048BB00BFB89DFF1FABAAAA2A5C9BFF1FE0
:102D8000409BFF1FA09DFF1F489BFF1FCDCCCC3D4C
:102D90000000FE428A9DFF1F3C9BFF1FFC9BFF1F04
:102DA000949BFF1F789BFF1FA29BFF1F549DFF1F3B
:102DB0008889FF1F649BFF1FC089FF1F449DFF1F61
:102DC000409DFF1FE29BFF1F6089FF1F924B1B78F6
:102DD000002B7FF46EAB039B904A243B83F34703A5
:102DE000D9B25B20136003F055FE98F80060032E03
:102DF00030D1DFF8808298F80030002B40F0368622
:102E0000874F3B78002B40F02486834E3378002B8D
:102E100040F01286834B1B78002B40F00086824ADC
:102E20001380824B1B78002B40F0EC85804B7F2277
:102E30001A8098F800306BB93B785BB933784BB99E
:102E40007C4A7F210720138003F024FE7F210B2082
:102E500003F020FE784B1F68FFF72BBB7748006814
:102E6000D0F17F0048BF033003EBA0030133994248
:102E7000BFF686AC116053E7714B09881A600029D0
:102E80007FF4CFAC13469842D4BFC2EB0003C2EB31
:102E9000030376E5FDF7F6FB37E60123CDF810B026
:102EA000CDF800B00593FFF7ACBA01232B60654C59
:102EB000FFF70ABA644B6A20198803F06FFF3B786A
:102EC0003370FFF701BA614B1B78002B3AD0604B8F
:102ED0001B88182B17D099F800201344A3F1180071
:102EE0007F2840F3ED845B4A973B82FB0321DA178E
:102EF000C2EB610202EB4202A3EB820303F1730017
:102F0000C0B203F017FE544A544B127833F8123013
:102F1000182B17D099F800201344A3F118007F282C
:102F200040F3D2844B4A973B82FB0321DA17C2EB72
:102F3000610202EB4202A3EB820303F17300C0B211
:102F400003F0F8FD019B1B88002B00F08C84444BA0
:102F50001B78002B40F08184424B394A198826683F
:102F60000020012310602B60B142364CBFF6ACA9A3
:102F700022683D4B0892089A1A60FFF7A5B9039B97
:102F80001B78002B7AD03B68A3F10C007F2840F31C
:102F9000F28330488B3B80FB0320DA17C2EB6000E2
:102FA00000EB4000A3EB800303F17300DFF8C08067
:102FB000C0B298F8001003F095FD009B1B78002B21
:102FC0005CD02A4E3378002B58D0DFF8ACA04FF0FD
:102FD000000B0BE003F17300C0B298F8001003F08F
:102FE00081FD33780BF1010B5B4547DD3B685AF8F7
:102FF000040F184A1844A0F18B0382FB0321DA174F
:10300000C2EB61020C3802EB42027F28A3EB820381
:10301000E0DCFDF737FBDFE7C49DFF1F7C9BFF1F54
:10302000C39DFF1FC29DFF1FF29BFF1FC59DFF1F7A
:103030005C9BFF1F389DFF1F509BFF1F909DFF1F34
:10304000409BFF1FB09EFF1F889BFF1FFC9BFF1F25
:10305000789BFF1FABAAAA2AA29BFF1F549DFF1FAC
:10306000449DFF1FFA9BFF1F509EFF1F8889FF1F73
:10307000E29BFF1FC19DFF1F6089FF1F029B1B7802
:10308000002B3AD0AD4B1A88182A18D03B6813444D
:10309000A3F118007F2840F3B683A94A973B82FB2F
:1030A0000321DA17C2EB610202EB4202A3EB8203B7
:1030B00003F17300A34BC0B2197803F013FDA249CA
:1030C0000B78022B00F253830133DBB20B701A46EC
:1030D0009E4830F81260182E40F090820422032B94
:1030E00003F10106F3B208BF002330F81360182E75
:1030F00040F08382013AF2D10B70019B1B88002BB8
:1031000000F0CB82009B1B783BB9039B1B7823B953
:10311000029B1B78002B00F0E0838D4B1B78002B6B
:1031200000F0D6808B490B78082B00F2D1808A48BA
:103130003A680068894E0133DBB25F1E101A46F808
:1031400027000B70864B2668198889F800200BE74A
:103150007F4B1B78002B40F0C1823B68814A12787C
:10316000002A45D0A3F10C007F2840F30A83744A5B
:103170008B3B82FB0321DA17C2EB610202EB4202B6
:10318000A3EB820303F17300C0B298F8001003F0C0
:10319000A9FC009B1B7853B36E4E33783BB3DFF82A
:1031A000FC91DFF89CA14FF0000B0BE003F17300E2
:1031B000C0B298F8001003F095FC33780BF1010BC6
:1031C0005B4514DD3B6859F8040F1844A0F18B03EC
:1031D0008AFB0321DA17C2EB61020C3802EB4202D0
:1031E0007F28A3EB8203E1DCFDF74CFAE0E73B68C4
:1031F0005D4A1278002A3DD0504A1288182A18D009
:103200001344A3F118007F2840F30D834C4A973BE9
:1032100082FB0321DA17C2EB610202EB4202A3EB4D
:10322000820303F17300C0B298F8001003F05AFC57
:103230003B6845490A78022A00F2A6820132D2B2DE
:103240000A701646414830F816E0BEF1180F40F0FB
:10325000F0810426032A02F1010E5FFA8EF208BF04
:10326000002230F812E0BEF1180F40F0E181013E7B
:10327000F0D10A70019A1288002A00F041823B497D
:1032800003220B702A60FFF71FB8394F3B78002BE1
:103290003FF476A9374E307801F01CF9364B1B7895
:1032A000002B00F0918233887E2B00F28D82334A0E
:1032B0000133108899B23180002800F09582C9B29C
:1032C000C0B22F4E03F0E6FB3B783370FEF7FCBF35
:1032D0003A6837E7DBB21846137003F0B9FB294BA5
:1032E0001B491A461F4B184600230B703B70137086
:1032F0000370FFF757B80123FFF796B880262249DD
:10330000224B234A09881B8812680B44B2EB630FD7
:10331000BFF6CFA8164B1B78002B40F0FE81B9F802
:1033200000301C4AB3423FF4C4A81B4B1680012254
:103330001A70FFF7BEB8FDF7A5F9B8E4789BFF1F38
:10334000ABAAAA2AE29BFF1FA29BFF1F549DFF1F4F
:10335000449DFF1F8889FF1F609BFF1F6489FF1F1B
:10336000FA9BFF1F3C9BFF1FFC9BFF1F409DFF1F05
:103370005E9BFF1F889BFF1FC69DFF1FCC9BFF1FEF
:103380005B9BFF1F8A9DFF1FEE9CFF1FF49CFF1F8E
:103390008C9BFF1F109DFF1F5F9BFF1F6089FF1FFE
:1033A000C14B01931B88002B40F06C83BF4B0393F0
:1033B000BF4B0293BF4E33786BB3DFF81483DFF853
:1033C000F8A24FF0000B09E003F17300C0B203F064
:1033D000B1FB33780BF1010B5B451CDD58F8043F62
:1033E00099F800001844A0F17F038AFB0321DA1743
:1033F000C2EB610202EB42027F28A3EB8203E3DC13
:10340000FDF740F9E2E7AA4B029303F093FB009B20
:103410001B78002BCED1039B1B78002B3FF4EDAB28
:1034200099F80030A3F10C007F2840F3A781A2484F
:103430008B3B80FB0320DA17C2EB600000EB4000FF
:10344000A3EB800303F17300C0B203F073FB009B96
:103450001B78002B00F08081964E3378002B00F013
:103460006582DFF86C82DFF850A24FF0000B0AE0B3
:1034700003F17300C0B203F05DFB33780BF1010B75
:103480005B457FF7BAAB58F8043F99F80000184441
:10349000A0F18B038AFB0321DA17C2EB61020C381F
:1034A00002EB42027F28A3EB8203E1DCFDF7EAF89E
:1034B000E0E75046FDF7E6F8FFF788BBFDF7E2F8D6
:1034C000FFF7C6B9002008707C49087840B17C49F4
:1034D00000910978002900F0A981009F002139702E
:1034E0007849097800297FF420A8002E67D10028A8
:1034F00065D1754E724F96F800E06C4E03966C4E97
:1035000002966A4E71493070694E009708703870A3
:103510003070BEF1000F7FF41AA8FFF721B8634B9B
:103520001B78002B3FF4CFAC99F80030A3F10C00CE
:103530007F2840F3C281604A8B3B82FB0321DA176C
:10354000C2EB610202EB4202A3EB820303F17300C0
:10355000C0B203F0EFFA009B1B78002B3FF4B3AC32
:10356000544E3378002B3FF4AEAC594FDFF848810E
:103570004FF0000A0AE003F17300C0B203F0DAFA78
:1035800033780AF1010A53457FF79DAC57F8043FA1
:1035900099F800001844A0F18B0388FB0321DA1787
:1035A000C2EB61020C3802EB42027F28A3EB8203DC
:1035B000E1DCFDF767F8E0E703980021017042497C
:1035C000097800293EF4CCAF3949029109780029E5
:1035D00000F08881029800210170FEF7C1BF039BB3
:1035E0001B78002B7FF44DAB029B1B78002B7FF4E4
:1035F00048AB019B1988FFF74ABB0B703B681E4420
:10360000A6F118007F2840F301812B4B973E83FBE6
:103610000632F317C3EB620303EB4303A6EB830607
:1036200006F173002B4BC0B2197803F05BFA64E526
:103630000A707344A3F118007F2840F3F1801E4AFA
:10364000973B82FB0321DA17C2EB610202EB4202D5
:10365000A3EB820303F17300C0B298F8001003F0EB
:1036600041FA3B6806E6243B002BB9F8000040F322
:103670002F8198423EF4F5AE9BB21748A9F800306E
:1036800001230370FEF7EDBEDFF84880C0B298F862
:10369000001003F027FAFFF70EBB0E4B38781978AD
:1036A00003F020FA2EE500BF949BFF1F3C9BFF1FF9
:1036B000FC9BFF1F8889FF1FABAAAA2AC59DFF1F7D
:1036C0008A9DFF1FC19DFF1F5E9BFF1F449DFF1F23
:1036D0006089FF1FE29BFF1F5F9BFF1F7F21402030
:1036E00003F0D8F9B349B44A3B680B60002111706C
:1036F00034E5C0B298F8001003F0F4F9FFF7AFB862
:10370000D8B298F8001003F0EDF93B68B7E5AB4B81
:10371000DFF8ECE21978FEF7A4BE4B2E40F3A98047
:103720001836802EB9F80030A54AA8BF8026B342CB
:103730007FF4FBADFEF7BDBE99F8000003F0FAF987
:103740003188FFF7A4BA9F4B01931B88002B7FF4AD
:103750005AAE9D4B029363E6029B1B78002B7FF4CD
:1037600050AA039B1B78002B7FF48BAA41E7002211
:1037700013460A70ACE4FCF785FF17E4FCF782FF00
:1037800062E6FCF77FFFFFE4002216460A7059E567
:10379000FCF778FFFFF74DB98C4E307800F09AFEB9
:1037A0008B4B1B781BB133887E2B40F2A780894B53
:1037B0001B7823B13388854A002B40F0AB80864EBE
:1037C0003B783370FEF780BD824B1B78002BF6D020
:1037D00033887E4A002BF2D08049013B088899B299
:1037E000118000287FF46BADC8B27B4E03F0C6F9A0
:1037F0003B783370FEF768BD7F20FFF7D1B9FCF747
:1038000041FFFFF717BAFCF73DFF53E4FCF73AFF1F
:1038100008E7FCF737FFFFF72CBA7F20FFF7E5B882
:10382000FCF730FF18E7FCF72DFFFCE4664F6C490E
:1038300002974FF0000C81F800C0009F02994FF0F2
:10384000010E87F800E081F800C049E60120FFF78B
:10385000A7B903F06FF9FFF7F5B80021402003F096
:1038600019F9FFF779BB99F8000003F063F9FFF746
:103870006EBB243E002EB9F800303ADDB3423EF470
:1038800018AEB6B2574BA9F8006001221A70FEF7C5
:1038900010BE0120FFF7A9B84A4B01931B88002BEB
:1038A0007FF4B3ADFFF7A9B94F4A8342A8BF0346DF
:1038B0001360FEF7B6BF16462CE5FCF7E3FE47E6BD
:1038C000FCF7E0FEFFF71CBBFCF7DCFEFFF737BBA5
:1038D00001283EF4C6AD0123CFE699F8000003F0BD
:1038E00029F91AE44148009041483D490390FEF708
:1038F0002EBE012B3EF4DDAD0126C3E701339BB2A2
:103900003380D9B20520344E03F0C4F83B783370CD
:10391000FEF7DABC013B9BB2D9B205202E4E1380D4
:1039200003F0B8F83B783370FEF7CEBC029B1B78EF
:10393000002B7FF466A9FFF7A4B92E4B1B782BB39D
:103940002D4B1B78002B7EF4B4AD2C4B1B78002B39
:103950003EF4AFADB9F8003022490A33A9F800307F
:103960000A70FEF7A6BD244B1B78002B7EF4A1AD98
:10397000224B1B78002B3EF49CADB9F8003019495E
:10398000013BA9F800300A70FEF793BD1A4B1B7873
:10399000002B7FF41BAA194B1B78002B3EF489AD3A
:1039A000B9F800300F490133A9F800300A70FEF76A
:1039B00080BD00BF609BFF1F8889FF1FAD9DFF1F5B
:1039C000109DFF1F949BFF1FFC9BFF1F889BFF1FE9
:1039D000C69DFF1FC59DFF1F5B9BFF1FCC9BFF1F4D
:1039E000449DFF1F5F9BFF1F409BFF1F8A9DFF1F82
:1039F0003C9BFF1FC29DFF1FC39DFF1FC49DFF1F58
:103A0000A99BFF1F224B00227F2107201A8003F071
:103A100041F87F210B2003F03DF8FFF70ABA1D4B58
:103A200001227F2107201A8003F034F87F210B2028
:103A300003F030F8FFF7F5B9174B04227F21072078
:103A40001A8003F027F800210B2003F023F8FFF77A
:103A5000E1B9114B02227F2107201A8003F01AF8E6
:103A60007F210B2003F016F8FFF7CFB90A4B002196
:103A700007201E8003F00EF87F210B2003F00AF8C8
:103A8000FFF7BEB9054B0393054B0293BDE400BF9E
:103A90005C9BFF1FF29BFF1F389DFF1F3C9BFF1F7E
:103AA000FC9BFF1F38B506F08FFD0E4804F0C6FCE6
:103AB0000D4804F0C3FC0D4804F0C0FC00234FF097
:103AC0007E5201210A48FCF7D1FC0A4B0A4A0B49F5
:103AD000802400251C7118461D60BDE838400AF09E
:103AE00035BA00BF709BFF1F9C9BFF1FF89BFF1FF9
:103AF000149DFF1F949DFF1F1C89FF1F29060000B6
:103B000043682A20198803F049B900BF10B504465C
:103B100022206368198803F041F9E368242019889A
:103B2000BDE8104003F03AB910B504460A206368B6
:103B3000198803F033F9E3680C201988BDE81040B8
:103B400003F02CB910B5044606206368198803F009
:103B500025F9E36808201988BDE8104003F01EB974
:103B600010B5044602206368198803F017F9E3686A
:103B700004201988BDE8104003F010B970B50E4C50
:103B800084B01225042201230646039002932046A6
:103B90008DE824001423102105F054FE0622092389
:103BA000029303960195204600921423102105F0FC
:103BB00049FE04B070BD00BFEC9DFF1F2DE9F04130
:103BC000224D82B0012602B284B2009228460196AC
:103BD0007823192105F07CFD04F10C0212B28DE866
:103BE00044002846A7197823192104F1020805F09A
:103BF0006FFD3FB20FFA88F819233A462846194656
:103C00000196CDF8008005F063FD78233A462846FA
:103C10001946CDF80080019604F10A070B3405F02F
:103C200057FD3FB224B278233A46284619468DE81C
:103C3000500005F04DFD192300943A4601962846A0
:103C4000194605F045FD02B0BDE8F081EC9DFF1F6F
:103C50002DE9F0411E4682B01446002A6AD0099B25
:103C60004D4A00EBC305012C6F8929896868A7EBD1
:103C7000010382FB03E21A444FEAE373C3EBA2138E
:103C800002887BD0042C38D112FA83F3994203DCEA
:103C90009F423946A8BF1946089A0180B6F90030FC
:103CA000BDF920803D48971D4FF0000E3FB21946E8
:103CB00042460097CDF804E005F00AFD29896A899B
:103CC0006B68521A1B885C2AA3EB010359DD03EBD6
:103CD00043030132C3EB431393FBF2F303F11B02E3
:103CE00013B20120328019464246019000972B48BA
:103CF00005F0EEFC2A4B00221A702A4B022CB3F975
:103D0000001045D0082C31D100221A8091422DD0CC
:103D1000089AB6F9003021480632012412B2009206
:103D200019460194BDF9202005F0D2FC204602B0CE
:103D3000BDE8F0811C4D1D4A2B681268CB1A9342D6
:103D40000F4617D9164A338811781448012918BF2D
:103D500001241470089A06321BB212B28DE81400C6
:103D60001946BDF9202005F0B3FC2F60012002B0F8
:103D7000BDE8F081204602B0BDE8F0819BB2D31AC5
:103D800084E75C2101FB03F393FBF2F21B32A7E70C
:103D90004A1C12B21A80B9E7C94216B2EC9DFF1F45
:103DA000729EFF1FD49DFF1F509EFF1FBCFF00008F
:103DB00030B583B000230C4605B2009326225B2366
:103DC0001C210C4805F0D4F9294601232622094874
:103DD00004F0DEFC002C24B205DB21460123262260
:103DE000044804F0D5FC044A044B15801C8003B041
:103DF00030BD00BFEC9DFF1F268AFF1F288AFF1FD2
:103E0000F0B59B4C237883B01BB19A4B4FF6FF72F1
:103E10001A80994BB3F90030C3B9984A954B106892
:103E2000B3F9002080F30C005B2303FB00F00013C8
:103E30001C3082425ED04FF0FF31FFF7B9FF90484F
:103E400005F0FAF90023237003B0F0BD012B36D042
:103E5000022B6ED0032B53D0042BF3D12522002547
:103E60008DE8240076231C218548864E864F05F078
:103E70002FFC17E0B0F5AF7FA8BF4FF4AF7032381A
:103E800003FB00F387FB0321DB17C3EB61111C313C
:103E900009B201231D442522794804F079FC0C2D38
:103EA00000F08480E9B2794804F030FB56F8042B26
:103EB000801A31284FF05B03DCDC1C21E9E7744BEE
:103EC0001A68B2F52F7F32DB41F25C239342A8BF20
:103ED0001346A3F52F735B226E4802FB03F380FBAE
:103EE0000320DB17C3EBA0201C30624BB3F900307A
:103EF0008342A0D1684BB3F9003001339BD1A1E7D5
:103F0000664B1B68B3F5FA7F11DBB3F57A6FA8BF78
:103F10004FF47A63A3F5FA7261485B2303FB02F363
:103F200080FB0320DB17C3EB20201C30DDE71C20C7
:103F3000DBE75C4B1B68B3F5FA7F33DBB3F57A6FD5
:103F4000A8BF4FF47A63A3F5FA7255485B2303FBCD
:103F500002F380FB0320DB17C3EB20201C30524B05
:103F60001B68B3F5FA7F1FDBB3F57A6FA8BF4FF478
:103F70007A63A3F5FA724A495B2303FB02F381FBE0
:103F80000321DB17C3EB21211C313A4BB3F900307D
:103F900083427FF452AF404BB3F900308B427FF441
:103FA0004CAF4FE71C20DAE71C21EEE72622002564
:103FB0008DE8240076231C2131483C4E324F05F019
:103FC00087FB16E0B0F5AF7FA8BF4FF4AF70323873
:103FD00003FB00F387FB0321DB17C3EB61111C31EB
:103FE00009B201231D442622254804F0D1FB0C2DE3
:103FF0000CD0E9B22E4804F089FA56F8042B801A46
:1040000031284FF05B03DDDC1C21EAE72722002585
:104010008DE8240076231C211948264E1A4F05F0FE
:1040200057FB17E0B0F5AF7FA8BF4FF4AF70323841
:1040300003FB00F387FB0321DB17C3EB61111C318A
:1040400009B201231D4427220D4804F0A1FB062DCF
:104050003FF4F5AEE9B2184804F058FA56F8042BCC
:10406000801A31284FF05B03DCDC1C21E9E700BF3C
:10407000CA9DFF1F268AFF1FD09DFF1F489DFF1F5F
:10408000EC9DFF1FDC89FF1F4B48371B9C9BFF1FCC
:104090004C9BFF1FD3058541288AFF1F8C9BFF1F68
:1040A000011FB812989BFF1FBC9DFF1F3089FF1F87
:1040B000F89BFF1F0C8AFF1F709BFF1F2DE9F04F1D
:1040C000DFF8EC82B74CB8F900604D7854F8264020
:1040D00087B08246039305B10D78DFF8FCB2002A61
:1040E00034D19BF800308BBBAF4EB6F900000028EE
:1040F00000F0CE80012800F02481012032232A46DE
:10410000019000935146A94B2046FFF7A1FD0025E1
:104110000746B6F90030022B40F3F48000233380C9
:10412000B8F90030A24A002BC0F2F880042BC4BFBB
:1041300000231380039B002B40F0F680002D0CBF62
:1041400038464FF0FF3007B0BDE8F08F964EE36879
:104150002268984804930027059237808BF80070F6
:1041600004F05EFF1120FFF729FD4FF0010919232C
:104170002821CDF804900091242219468D4805F09D
:10418000A7FA782328212422CDF8049000918948A9
:10419000194605F09DFA4946864805F02FFE022291
:1041A0001921844805F026FEDDF8149048460AF0EF
:1041B000A7FC494602467F4805F0B6FF7D4805F05A
:1041C000C9FF394614227B4805F014FE03227A49C0
:1041D000784805F0A9FF774805F0BCFF394623224F
:1041E000744805F007FE03227449724805F09CFFED
:1041F000704805F0AFFF049B002B72D10123704A79
:1042000018461370FFF7BAFC208963896768191A8A
:104210005C293A885BDC131A5C2202FB03F292FBF6
:10422000F1F31B33674A6348138001271BB21A223C
:1042300019468DE88400142205F04AFA049BDBB18C
:10424000218A638AE768581A5C283A886FDD521A17
:1042500002EB4202C2EB4212431C92FBF3F31B330C
:10426000524A54481380012738221BB28DE884003B
:104270001946322205F02CFA534A544BB6F9000085
:10428000012111704FF6FF721A8000287FF432AFBF
:10429000DFF848914E4AD9F800301268C3EB0A03A0
:1042A00093424CD9464B1A78012A18BF0120187046
:1042B0000127FFF763FCC9F800A0012D4ED0042DA3
:1042C00059D0022D60D0082D64D0002521E7121AA4
:1042D00002EB4202C2EB42124B1C92FBF3F31B3384
:1042E000A0E72F20FFF76AFC39463222314805F05B
:1042F00081FD032237492F4805F016FF2D4805F0B0
:1043000029FF7BE77FF40CAFE368002B3FF406AF97
:10431000B8F90030264A002BBFF608AF04231380FB
:10432000039B002B3FF40AAFFFF76AFD06E7511A23
:104330005C2202FB01F292FBF0F31B3390E707468D
:10434000BBE7002714238DE888002A4651461D4B01
:104350002046FFF77DFC3D460746DAE6B8F8003018
:104360008BF800500133A8F80030636983B1002551
:1043700020469847CDE6B8F800300122013BA8F866
:1043800000308BF80020F0E7012333800025C7E6DA
:104390001D46BEE66369002232804FF0FF35002BD8
:1043A000E6D1BDE62C8AFF1FD49DFF1FCE9DFF1FC7
:1043B000D09DFF1FEC9DFF1F64F4000068F4000017
:1043C000729EFF1FCC9DFF1FCA9DFF1F268AFF1FE5
:1043D000BCFF00006CF40000D29DFF1F509EFF1F29
:1043E00001210D2006F06ABD00210D2006F066BDFA
:1043F00001460D2006F062BD08B50D2006F064FDF3
:10440000B0FA80F149090D20BDE8084006F056BD1C
:1044100010B5002144080D2006F050FD204606F09E
:1044200089FD0D20012106F049FD2046BDE8104020
:1044300006F080BD08B5214A214B128818688242D7
:1044400034DA204B1B88991A8342A8BF0346B1F582
:10445000F87FA3EB020321DAC3EB031303EB43134F
:1044600093FBF1F105310A2006F098FB164B197801
:10447000F1B1164B16491B6883F30703C3EB031313
:1044800003EB431381FB03211944DB17C3EBA11199
:1044900005310920BDE8084006F080BBC3EB43139B
:1044A0001B01013193FBF1F10531DCE70021DAE773
:1044B0000920BDE8084006F071BB00BFFA9BFF1F52
:1044C000409BFF1FA09DFF1FB79BFF1F909DFF1FDD
:1044D000090402817F2838B5A8BF7F200D4D4FF415
:1044E000FA7303FB00F485FB04232344E117C1EBBB
:1044F000A3110A2006F052FBA4F578400C3885FB86
:1045000000310144C017A0EBA111BDE838400920DB
:1045100006F044BB09040281024B4E20198802F0C8
:104520003DBC00BF949BFF1F024B4420198802F042
:1045300035BC00BF789BFF1F024B1020198802F08A
:104540002DBC00BFFC9CFF1F024B2C20198802F0E1
:1045500025BC00BF6C9BFF1F024B1E20198802F078
:104560001DBC00BF689BFF1FC3680E20198802F0A6
:1045700015BC00BF024B2820198802F00FBC00BFF9
:10458000509DFF1F024B6420198802F007BC00BF3A
:104590004C9DFF1F024B5A20198802F0FFBB00BF41
:1045A000549BFF1F024B1620198802F0F7BB00BF77
:1045B0005C9BFF1F024B2E20198802F0EFBB00BF4F
:1045C000EC9BFF1F024B3020198802F0E7BB00BFB5
:1045D000489BFF1F024B1820198802F0DFBB00BF69
:1045E000FE9BFF1F024B1A20198802F0D7BB00BFA9
:1045F0009E9BFF1F024B1C20198802F0CFBB00BFFF
:10460000969BFF1F024B6620198802F0C7BB00BFB4
:10461000889DFF1F024B7220198802F0BFBB00BFAC
:10462000A49DFF1F024B2020198802F0B7BB00BFDA
:10463000869DFF1F024B3220198802F0AFBB00BFDE
:10464000769DFF1F024B6820198802F0A7BB00BFB0
:10465000CC9BFF1F024B6C20198802F09FBB00BF50
:10466000449BFF1F024B6E20198802F097BB00BFCE
:10467000C89DFF1F024B5220198802F08FBB00BF5C
:104680006089FF1F024B5020198802F087BB00BFD2
:10469000D489FF1F024B5420198802F07FBB00BF52
:1046A000D689FF1F024B5C20198802F077BB00BF40
:1046B000248AFF1F024B5E20198802F06FBB00BFE7
:1046C0002C89FF1F024B6020198802F067BB00BFD6
:1046D000EA9CFF1F024B5620198802F05FBB00BF07
:1046E000E09BFF1F38B5094D4624204602F070FBC1
:1046F00035F8021B00B28842204601D002F04EFB82
:104700000234A4B24E2CF0D138BD00BF549DFF1F1F
:10471000064B074A10B41C88064B0846002C14BFF1
:1047200011461946042210BC0AF0A8BAB09BFF1F1C
:1047300068FB00006CFB0000064B074A10B41C88A5
:10474000064B0846002C14BF11461946042210BC23
:104750000AF094BAEE9BFF1F68FB00006CFB0000A0
:10476000064B074A10B41C88064B0846002C14BFA1
:1047700011461946042210BC0AF080BA4E9DFF1F54
:1047800068FB00006CFB0000064B074A10B41C8855
:10479000064B0846002C14BF11461946042210BCD3
:1047A0000AF06CBA429DFF1F68FB00006CFB000022
:1047B000064B074A10B41C88064B0846002C14BF51
:1047C00011461946042210BC0AF058BAF29BFF1F8A
:1047D00068FB00006CFB0000F0B52B4E2B4FDFF8A0
:1047E000C4E005460FCE87B06C460FC496E80300C0
:1047F0003B68274A274F44F8040B40F6CC308342ED
:10480000C8BF3A46BEF800602180012E1188927818
:10481000ADF80D108DF80F202AD032D340F6CA0221
:10482000022E18BF00229A4226DCA3F698031A49EA
:104830001A4AC3EB031381FB03011944DB17C3EBD3
:104840006123243382FB0321DA17C2EBA10202EBBE
:104850008201A3EB4103303330328DF813308DF8F1
:1048600011206946284616220AF008FA07B0F0BD62
:1048700040F698029A42D8DD094B1868CDF811002D
:10488000EFE740F6FC02CEE780FB0000609DFF1FD3
:1048900074FB000070FB00003B773B986766666620
:1048A00078FB0000DE9CFF1FF8B5174C174E2278EE
:1048B000174D33782F888E46003218BF01220146EB
:1048C0007046FFF7FBFB002398423370237015DB23
:1048D00014BF012000202B889F420ED040F23A7274
:1048E000A3F5AF730B490C4C02FB03F381FB0312DE
:1048F000DB17A3EB621332332360F8BD07490122B3
:1049000018460A702270E6E7D08AFF1FE59DFF1F58
:104910009C9DFF1FB5814E1BC489FF1F689EFF1F12
:10492000014B187802F0D2B94C9EFF1F014B18784A
:1049300002F0E6B9E48FFF1F134BB3F9003030B536
:1049400083EAE374A4EBE374002BA0B218DB012329
:1049500000E0134603EB830252009442F9DA0B4D58
:1049600090FBF3F285FB03E403FB1200DB1730320C
:10497000D3EBA40380B201F8012BF1D10B7030BD51
:104980002D230B700131E2E7E48FFF1F6766666637
:10499000144BB3F9003070B583EAE375A5EBE3750A
:1049A000002BACB21ADB012300E0034603EB8300CB
:1049B00040008542F9DA0C4E94FBF3F086FB03E5E8
:1049C00003FB1044DB173030D3EBA503A4B201F88E
:1049D000010BF1D105480B70106070BD2D230B70D9
:1049E0000131E0E7549BFF1F6766666698FB000095
:1049F000134BB3F9003030B583EAE374A4EBE374EE
:104A0000002BA0B218DB012300E0134603EB830266
:104A100052009442F9DA0B4D90FBF3F285FB03E46C
:104A200003FB1200DB173032D3EBA40380B201F892
:104A3000012BF1D10B7030BD2D230B700131E2E75A
:104A40006089FF1F67666666134BB3F9003030B5A7
:104A500083EAE374A4EBE374002BA0B218DB012318
:104A600000E0134603EB830252009442F9DA0B4D47
:104A700090FBF3F285FB03E403FB1200DB173032FB
:104A8000D3EBA40380B201F8012BF1D10B7030BD40
:104A90002D230B700131E2E7D489FF1F676666663C
:104AA000134BB3F9003030B583EAE374A4EBE3743D
:104AB000002BA0B218DB012300E0134603EB8302B6
:104AC00052009442F9DA0B4D90FBF3F285FB03E4BC
:104AD00003FB1200DB173032D3EBA40380B201F8E2
:104AE000012BF1D10B7030BD2D230B700131E2E7AA
:104AF000D689FF1F67666666134BB3F9003030B581
:104B000083EAE374A4EBE374002BA0B218DB012367
:104B100000E0134603EB830252009442F9DA0B4D96
:104B200090FBF3F285FB03E403FB1200DB1730324A
:104B3000D3EBA40380B201F8012BF1D10B7030BD8F
:104B40002D230B700131E2E7248AFF1F676666663A
:104B5000134BB3F9003030B583EAE374A4EBE3748C
:104B6000002BA0B218DB012300E0134603EB830205
:104B700052009442F9DA0B4D90FBF3F285FB03E40B
:104B800003FB1200DB173032D3EBA40380B201F831
:104B9000012BF1D10B7030BD2D230B700131E2E7F9
:104BA0002C89FF1F67666666054B1B881BB9054B82
:104BB000186808607047044B18680860704700BFA9
:104BC000949BFF1FA0FB00009CFB0000164B1B8862
:104BD0000BB31BB230B583EAE374A4EBE374002B90
:104BE000A0B21CDB012300E0134603EB830252005A
:104BF0009442F9DA0D4D90FBF3F285FB03E403FBDD
:104C00001200DB173032D3EBA40380B201F8012B82
:104C1000F1D10B7030BD064B1868086070472D232A
:104C20000B700131DEE700BF689BFF1F6766666699
:104C30006CFB0000164B1B880BB31BB230B583EA2C
:104C4000E374A4EBE374002BA0B21CDB012300E0AF
:104C5000134603EB830252009442F9DA0D4D90FBA8
:104C6000F3F285FB03E403FB1200DB173032D3EBD6
:104C7000A40380B201F8012BF1D10B7030BD064BBB
:104C80001868086070472D230B700131DEE700BF04
:104C90007A9DFF1F676666666CFB0000164B1B88DB
:104CA0000BB31BB230B583EAE374A4EBE374002BBF
:104CB000A0B21CDB012300E0134603EB8302520089
:104CC0009442F9DA0D4D90FBF3F285FB03E403FB0C
:104CD0001200DB173032D3EBA40380B201F8012BB2
:104CE000F1D10B7030BD064B1868086070472D235A
:104CF0000B700131DEE700BF5C9BFF1F67666666D5
:104D0000A4FB0000174B1B881BB31BB270B583EAD2
:104D1000E375A5EBE375002BACB21EDB012300E0CD
:104D2000034603EB830040008542F9DA0E4E94FB04
:104D3000F3F086FB03E503FB1044DB173030D3EBC5
:104D4000A503A4B201F8010BF1D108480B70106063
:104D500070BD074B1868086070472D230B70013138
:104D6000DCE700BFEC9BFF1F676666667CFB00000C
:104D70006CFB0000164B1B880BB31BB230B583EAEB
:104D8000E374A4EBE374002BA0B21CDB012300E06E
:104D9000134603EB830252009442F9DA0D4D90FB67
:104DA000F3F285FB03E403FB1200DB173032D3EB95
:104DB000A40380B201F8012BF1D10B7030BD064B7A
:104DC0001868086070472D230B700131DEE700BFC3
:104DD000489BFF1F676666666CFB0000164B1B88CE
:104DE0000BB31BB230B583EAE374A4EBE374002B7E
:104DF000A0B21CDB012300E0134603EB8302520048
:104E00009442F9DA0D4D90FBF3F285FB03E403FBCA
:104E10001200DB173032D3EBA40380B201F8012B70
:104E2000F1D10B7030BD064B1868086070472D2318
:104E30000B700131DEE700BF889DFF1F6766666665
:104E40006CFB0000164B1B880BB31BB230B583EA1A
:104E5000E374A4EBE374002BA0B21CDB012300E09D
:104E6000134603EB830252009442F9DA0D4D90FB96
:104E7000F3F285FB03E403FB1200DB173032D3EBC4
:104E8000A40380B201F8012BF1D10B7030BD064BA9
:104E90001868086070472D230B700131DEE700BFF2
:104EA000A49DFF1F676666666CFB0000174B1B889E
:104EB0001BB31BB270B583EAE375A5EBE375002B5A
:104EC000ACB21EDB012300E0034603EB830040008D
:104ED0008542F9DA0E4E94FBF3F086FB03E503FB03
:104EE0001044DB173030D3EBA503A4B201F8010B5B
:104EF000F1D108480B70106070BD074B186808604E
:104F000070472D230B700131DCE700BF869DFF1F2A
:104F100067666666A8FB00006CFB0000074B1B88F9
:104F2000022B06D0012B0CBF054B064B18680860FE
:104F30007047054B18680860704700BFEA9CFF1F68
:104F4000B0FB0000B4FB0000ACFB0000054B1B886D
:104F50001BB1054B186808607047044B186808605F
:104F6000704700BFE09BFF1FBCFB0000B8FB0000C8
:104F700008B5702001F02CFF044B1988884204D03A
:104F80007020BDE8084001F009BF08BDDE9CFF1F8E
:104F900008B5742001F01CFF044B1988884204D026
:104FA0007420BDE8084001F0F9BE08BD6C9DFF1FEC
:104FB00038B5FCF7C9FC0D4B1B7833B90C4B1020EE
:104FC000198801F0EBFE012038BD0A4D0A4C2B7800
:104FD0002288B3FA83F382F008025B09114642206B
:104FE0002B70228001F0DAFE002038BD5E9BFF1F8F
:104FF000FC9CFF1FE29CFF1FA29DFF1F184B1A88FD
:1050000052B3184A128830B50A80B3F90030002B29
:1050100083EAE374A4EBE374BCBF2D238B70A0B2CE
:10502000ACBF02310331012300E0134603EB8302DE
:1050300052009442F9DA0C4D90FBF3F285FB03E445
:1050400003FB1200DB173032D3EBA40380B201F86C
:10505000012BF1D10B7030BD044B1868086070470C
:105060009E9BFF1FC0FB0000676666666CFB00002E
:1050700010B40A4B0A4C0A4693E8030083B0238815
:1050800002AC04E9030004EB8303104653F8081C48
:10509000052203B010BC09F0F1BD00BFF4F400001C
:1050A0004C9DFF1F30B40A4B0A4D0C4693E8070095
:1050B00084B02B8804AD05E9070005EB8303204687
:1050C00053F80C1C042204B030BC09F0D7BD00BF5B
:1050D000FCF40000DE9CFF1FF0B40C4D0C4F0E469C
:1050E0000FCD8CB001AC0FC40FCD0FC495E80700F5
:1050F0003B8884E807000CAA02EB8303304653F890
:105100002C1C04220CB0F0BC09F0B8BD08F500005E
:10511000389DFF1FF0B40A4D0A4F0E460FCD86B0E2
:1051200001AC0FC42A683B88226006AA02EB830305
:10513000304653F8141C042206B0F0BC09F09EBDA2
:1051400034F50000FE9BFF1FF0B40A4D0A4F0E46D7
:105150000FCD86B001AC0FC42A683B88226006AA36
:1051600002EB8303304653F8141C0C2206B0F0BC4B
:1051700009F084BD48F50000969BFF1FF0B40A4D6E
:105180000A4F0E460FCD86B001AC0FC42A683B888B
:10519000226006AA02EB8303304653F8141C042253
:1051A00006B0F0BC09F06ABD5CF500006C9DFF1F05
:1051B000164B1B880BB31BB283EAE370A0EBE370C2
:1051C000002B30B584B21DDB012300E0134603EB56
:1051D000830252009042F9DA0D4894FBF3F280FB0F
:1051E00003E503FB1244DB173032D3EBA503A4B273
:1051F00001F8012BF1D10B7030BD0846042205499E
:1052000009F03CBD2D230B700131DDE7CC9BFF1F66
:1052100067666666C4FB0000F0B40A4D0A4F0E468E
:105220000FCD86B001AC0FC42A683B88226006AA65
:1052300002EB8303304653F8141C042206B0F0BC82
:1052400009F01CBD70F50000449BFF1F70B53C4D7C
:105250002B780646002B35D11C4673780BB92046B7
:1052600070BDFCF771FB374A374B384812783178FC
:105270001B78007802EB43034A1E03EB80030E2ADF
:10528000EDD801A050F822F0F152000013530000B5
:105290005F520000F15200005F5200005F520000B8
:1052A0005F520000DF5200005F5200005F520000BA
:1052B0005F5200005F5200005F5200005F5200002A
:1052C000DB520000AE21224803F05AFC204803F0D4
:1052D000A7FE00232B700124BFE706F03DF9AF21A4
:1052E0001B4803F04DFC1B4A012313702B70B6E7DB
:1052F00083B91948038804294FF6FF7103F1FF327F
:105300000CBF01230B46134403F07F0301330380DA
:105310000FE073B1013B114A32F813304BB10E4E1E
:105320000F481049104A33800123002606700B7085
:105330001370084A0221012311702B70204670BDA2
:10534000D08AFF1F8B9DFF1F849DFF1F8C9DFF1F19
:10535000EC9DFF1F689EFF1F109DFF1FD09CFF1F2D
:10536000C49BFF1F5F9BFF1F749EFF1F10B5064B62
:10537000064C1A882046012101F0FEFC21884220BB
:10538000BDE8104001F00ABDB09BFF1FA29DFF1FAA
:1053900010B5064B064C1A882046022101F0ECFCA1
:1053A00021884220BDE8104001F0F8BCEE9BFF1FB1
:1053B000A29DFF1F10B5064B064C1A8820460521FA
:1053C00001F0DAFC21884220BDE8104001F0E6BC83
:1053D0004E9DFF1FA29DFF1F10B5064B064C1A885D
:1053E0002046002101F0C8FC21884220BDE8104081
:1053F00001F0D4BC429DFF1FA29DFF1F08B51220E3
:1054000001F0E6FC054B1988884206D0122001F015
:10541000C5FCBDE8084001F0D9BB08BD389DFF1FA1
:1054200008B5582001F0D4FC054B1988884206D0F5
:10543000582001F0B3FCBDE8084001F0C7BB08BD2F
:105440007A9DFF1F08B5142001F0C2FC054B198896
:10545000884206D0142001F0A1FCBDE8084001F00C
:10546000B5BB08BDF29BFF1FF0B480EAE075A5EB69
:10547000E0750028ACB21FDB1DBF2B230B704E1C48
:105480000E46012300E0134603EB830252009542CF
:10549000F9DA0B4F94FBF3F287FB030503FB12448D
:1054A000DB173032D3EBA503A4B206F8012BF1D100
:1054B00033700846F0BC70472D230B704E1CE0E79C
:1054C00067666666084B188828B10D2807D00D3826
:1054D00000B2FFF7C9BF054A106808607047044A68
:1054E00010680860704700BFC89DFF1F6CFB00007C
:1054F000C8FB0000174B18880C2813D0192815D0AA
:105500001A2817D01B2819D01C281BD01D281DD0E5
:105510001E2803D00C3800B2FFF7A6BF0E4A106851
:10552000086070470D4A1068086070470C4A1068A0
:10553000086070470B4A1068086070470A4A106894
:1055400008607047094A106808607047084A106888
:1055500008607047769DFF1FE4FB0000CCFB000055
:10556000D0FB0000D4FB0000D8FB0000DCFB0000F7
:10557000E0FB0000034B1888A0EB8000400000B265
:10558000FFF772BF4C9EFF1F024B1888033800B212
:10559000FFF76ABF509DFF1F024B18880C3800B2FE
:1055A000FFF762BF589BFF1F024B1888183800B2E4
:1055B000FFF75ABF789BFF1FC3681888183800B2DE
:1055C000FFF752BF30B5134C85B001252B463C2266
:1055D00002212046009503F049FB204603F020FD00
:1055E00000224021802320460191009311460A4B5E
:1055F000029504F0C3F9204603F01EFE074808494F
:10560000084A0023036083800B608B8013609380C3
:1056100005B030BDEC9DFF1F10F70000D89DFF1FA7
:105620006C9EFF1F589EFF1F10B500EBC00000F1DD
:105630000F02D2B293B284B09C1E981C3D230391FA
:105640008DE819003921024804F0FCF804B010BDBF
:10565000EC9DFF1F014B01221A707047E59DFF1F53
:10566000F0B585B0634C644B0293644A0192042305
:105670000093634E634B644F644D2046402280216B
:1056800003F0FCF82046624A6249634C08F05EFC75
:10569000B761624FF761624FAF61624FEF61624F76
:1056A000A7616248624FE761624F87616249634F59
:1056B000C761634F8F61634A634FCF61634F9761E7
:1056C000634B644FD761644F9F61644E644FDF61E9
:1056D000644FB761644D654FF761654FAF61654CCD
:1056E000654FEF61654F6648A761664FE761664F9A
:1056F00066498761664FC761664F674A8F61674F2A
:10570000CF61674F674B9761674FD761674F684EAF
:105710009F61684FDF61684F684DB761684FF761FF
:10572000684F694CAF61694FEF61694FA761694884
:10573000694FE761694F876169496A4FC7616A4F7D
:105740008F616A4A6A4FCF616A4F97616A4B6B4FAC
:10575000D7616B4F9F616B4E6B4FDF616B4FB761D2
:105760006B4D6C4FF7616C4FAF616C4C6C4FEF61E0
:105770006C4FA7616C486D4FE7616D4F87616D4954
:105780006D4FC7616D4F8F616D4A6E4FCF616E4F28
:105790006E4B97616E4FD7616E4F6F4E9F616F4F2B
:1057A000DF616F4F6F4DB7616F4FF7616F4F704C97
:1057B000AF61704F70487149EF61714F714DA761D2
:1057C000E561714F714D724CDFF8E8E1714A724B3F
:1057D0008761C5618C61714EC1F81CE0704F714DDD
:1057E000714C724872499761D5619C61D861B16012
:1057F00005B0F0BDEC9DFF1FA0860100801A0600D9
:10580000348DFF1F2490FF1F99550000688EFF1FE5
:105810001C89FF1FD5880000D88DFF1F6945000037
:10582000895500007545000011470000148CFF1FCA
:105830006D53000039470000C88CFF1F91530000D2
:1058400061470000E88FFF1FB55300007150000052
:10585000808CFF1F8545000089470000108DFF1FC9
:10586000D953000075550000EC8CFF1F2149000042
:1058700039490000448EFF1F2D490000A55000004B
:10588000CC8BFF1F714F0000D9500000D08EFF1F3E
:10589000FD530000354C00005C8CFF1F21540000BC
:1058A00091490000888BFF1F95450000B14700001B
:1058B0003C8FFF1F455400009D4C0000388CFF1F9B
:1058C000A5450000054D0000588DFF1FB54500009F
:1058D000754D0000F88AFF1FC545000015510000F6
:1058E000A48CFF1FD5450000FD4F0000208EFF1F38
:1058F000E545000049510000C08FFF1FF54500003D
:10590000DD4D0000B48DFF1F05460000454E000030
:105910001C8BFF1F154600007D510000F48EFF1FF9
:10592000914F0000AD4E0000FC8DFF1F254600008A
:10593000F5540000408BFF1F35460000B1510000B8
:10594000D48AFF1F4546000019520000408AFF1FFD
:1059500055460000C5540000908FFF1F65460000AB
:10596000F1490000F08BFF1F75460000494A000016
:10597000AC8AFF1F85460000648BFF1F8C8EFF1FC3
:10598000A14A000095460000F94A0000A546000023
:10599000514B0000888AFF1F648AFF1FB48FFF1FCE
:1059A0001D4F0000C54600004D4F0000D5460000C9
:1059B0006D5F0000B5460000F0B5461C83B00D4693
:1059C0000127032336B22AB2044631468DE8880007
:1059D0002448ADB203F0CCFE0C23AA1C12B20093F3
:1059E0000197052321B21F4803F0C2FE1E4A1F4B38
:1059F00012881B68BA422AD023D3022A10D11C4C29
:105A0000A3F6CA0384FB03241C44DB17C3EB241452
:105A10000A2CA8BF0A2424EAE474A2B223B202E04A
:105A200000231A461C460D35AA1A01200093019046
:105A300012B2314603230B4803F018FE204603B090
:105A4000F0BD0C4CA3F6FC0384FB0324DDE7084CFB
:105A5000A3F6980384FB03241C44DB17C3EBE40484
:105A6000D6E700BFEC9DFF1FDE9CFF1F609DFF1F60
:105A7000898888881F85EB512DE9F0438FB283B068
:105A8000DFF84C80BD1D461D2DB204B236B24FF07A
:105A900001090AB22346314640460095CDF80490EC
:105AA00003F016FE2A463346214640468DE8200282
:105AB00003F00EFE07F10C020095334612B22146A8
:105AC000CDF80490404603F003FE03B0BDE8F08338
:105AD000EC9DFF1F2DE9F043804685B0002956D18B
:105AE0000121304804F08AF92F4998F8062098F8E7
:105AF000083011F80290994522DA4FEA89064D469E
:105B00000C24D8F80C3027489B595F6822B200213A
:105B100004F070F9384608F0F3FF39460246214890
:105B200004F002FB1F4804F015FB98F8083001351B
:105B30000934AB42A4B206F1040601DD422CE0D1E7
:105B4000B9F1000F13D109F1060999450CDA3C238C
:105B500001213B22039102930093019239233F22BA
:105B60003A21104803F06EFE05B0BDE8F0830F2324
:105B700001213B22039102930093019239230C22CD
:105B80003A21084803F05EFE98F80830DBE7002170
:105B90003423009301913F230C22024803F066FD59
:105BA0009EE700BFEC9DFF1F6C9EFF1F10B5104CC1
:105BB0000121204604F028F92046012104F01EF9B5
:105BC00020463422552104F015F9204602220949C5
:105BD00004F0AAFA20460522074904F0A5FA204657
:105BE00004F0B8FA2046BDE8104003F025BB00BF22
:105BF000EC9DFF1FE8FB0000ECFB000070B50D46BC
:105C0000064608F07DFF00EB40008400002D36D0F2
:105C1000284608F075FF00EB4000400023185B1099
:105C200003F16001091A282209B21748C3F1600480
:105C300004F0E0F80121144804F0E0F8284608F0E8
:105C40005FFF29460246104804F06EFA0E4804F041
:105C500081FA02210C4804F0D1F821B221220A482D
:105C600004F0C8F8304608F04BFF314602460648BB
:105C700004F05AFA0448BDE8704004F06BBA6410AE
:105C8000C4F16004E5E700BFEC9DFF1F10B50D4BAC
:105C90001B5C51F82340237884B013B1012004B079
:105CA00010BD04AA01A942F8103D2046A3699847F7
:105CB000A38A9B07F2D401A80099FFF79FFF012058
:105CC00004B010BDD89DFF1F2DE9F04F2F4DDFF818
:105CD000CCB0DFF8C4A0DFF8C8900FCD91B003AC12
:105CE0000FC40FCD0FC40FCD0FC42B682360002548
:105CF000A8462F462E4600E09846BAF800302449C0
:105D00005BF8232028461123FAF760FE00EBC0045D
:105D100000EB840089FB00340444C017C0EB6434FA
:105D2000C4F13C00C6F13C0207F14101012600B27A
:105D300008F1410300901BB2019612B209B2154856
:105D400003F0C6FC08EB060305F211153C2B2646B2
:105D5000ADB24746D0D134226B210E4804F04AF848
:105D600000210C4804F04AF80B4B1B8810AA02EBE8
:105D7000830353F8344C204608F0C2FE024605481F
:105D8000214611B0BDE8F04F04F0CEB984F5000013
:105D90008CF10000EC9DFF1F6C9BFF1FA4F0000026
:105DA00009000280214B70B5B3F9003083EAE37437
:105DB000A4EBE374002B82B0A1B22FDB68466D46E2
:105DC000012300E0134603EB830252009442F9DA08
:105DD000174E91FBF3F286FB03E403FB1211DB1772
:105DE0003032D3EBA40389B205F8012BF1D1194667
:105DF0002B70FFF703FF0F4B1B786BB101210E488F
:105E000003F0FCFF332274210B4803F0F3FF01225F
:105E10000A49094804F088F902B070BD2D238DF8B5
:105E200000300DF101056846CAE700BFFC9CFF1F6A
:105E300067666666E29CFF1FEC9DFF1F7CFF00000B
:105E400010B5424C424882B003F0EAF82378C3B957
:105E500006213F4803F0D2FF2378012B37D90A22CD
:105E6000022B11463A486BD003F0C4FF3949032294
:105E7000374804F059F9364802B0BDE8104004F044
:105E800069B9354B1A7801210523002A35D10191D2
:105E9000009311462E4803F06BFC304B1A78002A11
:105EA00036D0052301220192009300220A212848BE
:105EB00003F0DCFB2A4B1A78002A35D10121052397
:105EC000019100931421224803F052FCC0E7254CB5
:105ED0002388092B32D9632B8CBF0A211F210A2268
:105EE0001B4803F087FF2188194804F083F91848FC
:105EF00002B0BDE8104004F02DB9002201910093DA
:105F00001146134803F0B2FB144B1A78002AC8D18B
:105F100005230121019100930A210D4803F028FC7B
:105F20000F4B1A78002AC9D0012205230192009351
:105F300000221421064803F099FB89E73021CEE7BF
:105F400003F058FF0322084992E700BF749EFF1F29
:105F5000EC9DFF1FF8FB00008B9DFF1F849DFF1F22
:105F60008C9DFF1F109DFF1FF4FB0000F8B56D4DC9
:105F7000287840B96C4B1B6899425CD36B4A01236B
:105F800013702B70F8BD0C4600266948664F03F06D
:105F900047F804F6AC53324665483B6031212E7019
:105FA00003F028FF01216248624D03F02DFF3146C6
:105FB0005F4803F023FF05225F495D4804F0B4F811
:105FC0005B4804F0C7F80C221021594803F012FF77
:105FD0000B225A49564804F0A7F80522584954485C
:105FE00004F0A2F8524804F0B5F8564B50481C682B
:105FF000A4F69803C3EB031385FB03251D4410216E
:10600000DB172022C3EB652503F0F4FE40F6CC330A
:106010009C4205F124054FF022014FF004000BDCF7
:10602000FFF7CAFC484B1C88064674B3012C46D0C7
:10603000022C41D00120F8BDFFF71EFD0922434983
:106040003B4804F071F82A221021394803F0D2FEAF
:106050003F4C374884FB0534EB17C3EBA4042146BF
:1060600004F0C8F801223B49314804F05DF804EB24
:106070008401A5EB41012E4804F0BCF80122364909
:106080002B4804F051F80120F8BD3449102228486B
:1060900004F04AF8264804F05DF82A22102124482A
:1060A00003F0A8FE3146224804F0A4F807222C4948
:1060B0001F4804F039F8CBE70C222A49E7E70C2205
:1060C00029491B4804F030F8194804F043F82A2203
:1060D0001021174803F08EFE314615481C4E04F07F
:1060E00089F807221E49124804F01EF886FB05367F
:1060F000EB17C3EBA60631460D4804F07BF82246A9
:1061000014490B4804F010F806EB8601A5EB410199
:10611000074804F06FF822460F49054804F004F8D8
:106120002046F8BDD08AFF1F549EFF1F689EFF1FA8
:10613000EC9DFF1F3B773B98FCFB000004FC00003C
:10614000ECFB0000609DFF1FDE9CFF1F10FC0000A9
:1061500067666666F0000100600001001CFC00003C
:1061600030FC000048FC000038FC00002DE9F04144
:10617000754C2278002A05460F4614BF4FF00108DF
:106180004FF000084ED1714E3368CB1AB3F5FA6F59
:1061900004D86B78A3B94046BDE8F0816C4B6D48DC
:1061A0006D49DFF8D0E11A7001230370098823706C
:1061B00026208EF8002000F0F1FD6B78002BEAD04D
:1061C0003760FBF7C1FB654A654B66491278287852
:1061D0001B78097802EB4303421E03EB81030E2A6E
:1061E000D9D801A151F822F0D9620000A5620000BF
:1061F00097610000D962000097610000976100007C
:10620000976100008D620000976100003F6200000E
:10621000976100009761000097610000976100009E
:106220003B620000AF215048484E02F0A9FCFFF746
:1062300007FE002337602370ABE705F08DF94A486D
:1062400002F0EEFE0221484803F0D8FD0F22232180
:10625000454803F0CFFD05224449434803F064FF5D
:10626000414803F077FF1E2223213F4803F0C2FD7F
:1062700005223F493C4803F057FF3B4803F06AFFC3
:10628000394802F0D9FF00F0ADFC84E7394D2B7896
:10629000012B50D9304B2620198800F07FFD0023B8
:1062A0002B7078E7002B3FF476AF013B324A32F88F
:1062B0001330002B3FF46FAF274C304825492D4A4F
:1062C00023804FF001080023037081F8008082F8DA
:1062D0000080FFF7B5FD5EE793B1013B264A32F837
:1062E000131019B31C4B254D1A4C224A1980002655
:1062F000012326202E702370137000F04FFD15E04F
:10630000154C1E4922880B7004284FF6FF7002F1CD
:10631000FF310CBF012202460A440E4E154D02F019
:106320007F0201320121228031702B70FFF788FD3E
:106330004FF001082FE70649064A012300200870A4
:1063400013702370A6E700BFD08AFF1F649EFF1F53
:10635000689EFF1F5F9BFF1F109DFF1F8B9DFF1FF0
:10636000849DFF1F8C9DFF1FEC9DFF1F58FC0000AC
:1063700060FC0000749EFF1FD09CFF1FC49BFF1F8A
:106380002DE9F04F05468BB00F46AD48012116466A
:1063900003F03AFDAA8812F0010440F0B080DFF863
:1063A000CC8298F80030002B7DD1AB79A54AD15C26
:1063B000A1B9DFF8BCA279781AF8039041B3397813
:1063C0000139072900F2B780DFE811F0F10054012C
:1063D000B5006C01B500B500B500E9007C78002C73
:1063E00000F0CA800139EC68387854F82170FC68F4
:1063F000411EB4F80080072900F2A780DFE811F001
:1064000074015901A5006C01A500A500A5009F001D
:10641000DFF854A2DAF80020B21AB2F5967F75D9E7
:10642000894A107801281ABF012010701170874A1C
:1064300018BF0146D05CC0EB0900C0B2FFF7F4F80A
:106440000124CAF80060AB889B0770D57B78002BCD
:106450006DD0FBF779FA7E4B7E4A7F481B78127825
:1064600039780078022515FB02330A2903EB8003F3
:1064700000F04E810C295AD1002B58D003F119009D
:10648000764E774A013B0021400080B226F8131077
:106490000123157088F8003000F080FC714B032256
:1064A00020461A702FE0664802F0BAFD01216448C8
:1064B00003F0A4FC62482246214603F09BFCAB8813
:1064C000580725D42C68204608F01AFB21460246BE
:1064D0005B4803F029FE5A4803F03CFE09220123E1
:1064E0008DE80C0000217F23554803F0F1F80021CE
:1064F0002846FFF7EFFA002388F8003055E7AB682D
:106500003146384698470BB0BDE8F08F0846FAE7A9
:106510002B6804A8984704A808F0F2FA04A90246D8
:10652000474803F001FE464803F014FED6E7204634
:106530000BB0BDE8F08F00240AF8039083E7002138
:10654000D1543846FB699847FC68A4F800800027BE
:1065500025223C238DE8840041211822384803F08D
:1065600085F8E968A879FFF791FB374A3E4B177029
:106570001E600BB0BDE8F08F3B490A68B21AB2F555
:10658000967FD4D9304F0E603E78012E00F0B48053
:10659000E968184601233B70FFF778FBB3E7304A00
:1065A000E9791170012288F800200024C4E72A7AD2
:1065B000013A4A45BFDD09F10104E4B2A145BAD070
:1065C000224E16F803B0CBEB0900C0B20021FFF752
:1065D0002BF82B7A052BD9461BD9CBEB0402042AC6
:1065E00040F3AE80A4F1040BBBF1000FC0F2B08009
:1065F000063B5B45A8BF5B465FFA83F9AA7913485F
:10660000B15C994205D000F8029001212846FFF7BD
:1066100061FAC9EB0400C0B201210B4EFFF704F888
:1066200000213423019100930548317040230B224F
:106630003F21A14603F01AF80124AB797CE700BFA3
:10664000EC9DFF1F589EFF1F729EFF1F6C9EFF1F39
:106650008B9DFF1F849DFF1F8C9DFF1FD09CFF1FE4
:10666000689EFF1F749EFF1F509EFF1FD08AFF1F52
:10667000D89DFF1F0FFA89F1E868604C50F821603F
:106680002168049134785E4904980860002C71D028
:10669000012C7FF450AF5B4A317A88F800401170CA
:1066A000002449E7B9F1000F50D009F1FF34E4B2FA
:1066B00084E7B98A01F0040189B200293FF440AFB0
:1066C0003B6A03929847039A00283FF43DAFAB79A9
:1066D000FC680021D15438E77B8A43453CD908F156
:1066E00001081FFA88F830E73B8A43453BD208F19E
:1066F000FF381FFA88F828E725238DE8180042485C
:106700003C703C231822412102F0B0FF3046FAE6EB
:10671000002B3FF40CAF3D4A3D4E1188394A03F13E
:106720001900013B400080B226F81310012388F8BD
:106730000030157000F032FB364B20461D70E2E64B
:10674000002A3FF755AF04F1FF3B4DE74C46F3E617
:106750004FF000094B4651E7BB8ADA077FF5F5AEEB
:10676000B7F81080F1E6BB8AD9077FF5EEAEB7F82F
:106770001280EAE62849C85CC0EB090009F1010E65
:10678000C0B201214FF0340B02F803E0FEF74CFFDA
:10679000B6681D48019440230B223F210124CDF807
:1067A00000B002F063FF40230B223F211648CDF8D2
:1067B00000B0019402F0DCFF2146134803F01EFBF9
:1067C000304608F09DF9A0EB800000F15F0109B2AE
:1067D0000F220D4803F00EFB304608F091F93146C8
:1067E0000246094803F0A0FC074803F0B3FCE9683F
:1067F000A879FFF74BFAAB799EE600BFB09EFF1F6A
:10680000509EFF1F689EFF1FEC9DFF1F109DFF1FE6
:10681000D09CFF1F749EFF1F6C9EFF1F2DE9F04749
:10682000DFF808926D4B99F800601B68DFF800A252
:1068300082B0003601934FF0030018BF0126019F7C
:106840009AF8008004F040FB0546042004F03CFB6D
:106850000446052004F038FB800040EA440406208A
:1068600004F032FB2C4364B25D4944EAC0000A786C
:1068700080F00F03DBB29A425A4A3CD017600022E4
:1068800059480B7003788DF800808DF8012053B3C0
:10689000564A12684EF66021BA1A8A4219D8022B5B
:1068A00059D0012B5FD0062B48D0032B63D0042B8B
:1068B00069D0052B77D0072B7DD0082B00F0838083
:1068C000092B68D016B14A4802F0B6FC02B0BDE808
:1068D000F087484A484C002301212370037013605D
:1068E000938089F800103A4669464448FFF748FD0E
:1068F0003043C6B2E6E71268BA1A1E2A6BD99AF874
:106900000020934222D0394C3D488AF80030012BB8
:10691000276082EA030207609846B1D0042BAFD10A
:1069200037480068381AB0F5C87FA9D9354C2068B7
:10693000381A3228A4D927601A46A1E73A46694690
:106940003148FFF71DFD3043C6B2BBE7012B4FF0C6
:106950000002E3D1E4E73A4669462C48FFF710FD10
:106960003043C6B2AEE73A4669462948FFF708FD0C
:106970003043C6B2A6E73A4669462648FFF700FD0F
:106980003043C6B29EE73A4669462348FFF7F8FC13
:106990003043C6B296E73A4669462048FFF7F0FC16
:1069A0003043C6B28EE73A4669461D48FFF7E8FC19
:1069B0003043C6B286E73A4669461A48FFF7E0FC1C
:1069C0003043C6B27EE73A4669461748FFF7D8FC1F
:1069D0003043C6B276E7002252E700BFB09EFF1FE9
:1069E000759EFF1FE09DFF1F689EFF1F609EFF1F9B
:1069F000EC9DFF1F589EFF1F739EFF1FBCF60000FB
:106A0000789EFF1FE89DFF1F10FB000080F600002E
:106A1000E0F50000C4F5000014F60000D0F5000019
:106A200024F6000064F60000B48FFF1FD08AFF1F19
:106A3000E49DFF1F28B11028044BA8BF1020186048
:106A40007047024B01201860704700BF7C9EFF1FFB
:106A500038B50F4D2B78013B01381B02C4B203F44B
:106A60007063200443F4404343F00C0300F4FE0041
:106A7000184305F091FB2868013860F03F00C0B270
:106A800004F0B8FB2046BDE8384004F0B3BB00BFBB
:106A90007C9EFF1F70B5124D2B78013B1B0203F447
:106AA0007063064643F430430806320400F0FE40AB
:106AB00043F00B03034302F4FE0018430C4605F0B9
:106AC0006BFB2868013860F04F00C0B204F092FB05
:106AD000304604F08FFB2046BDE8704004F08ABBCE
:106AE0007C9EFF1F70B5124D2B78013B1B0203F4F7
:106AF0007063064643F410430806320400F0FE407B
:106B000043F00903034302F4FE0018430C4605F06A
:106B100043FB2868013860F06F00C0B204F06AFBE4
:106B2000304604F067FB2046BDE8704004F062BBCD
:106B30007C9EFF1F38B5104D2B78013B1B0203F4E0
:106B40007063044643F41043000443F0090300F467
:106B5000FE00184305F020FB2868013860F06F0044
:106B6000C0B204F047FB204604F044FB0020BDE81F
:106B7000384004F03FBB00BF7C9EFF1F38B50E4D70
:106B80002B78013B1B0203F47063044643F450432B
:106B9000000443F00D0300F4FE00184305F0FCFA76
:106BA0002868013860F02F00C0B204F023FB2046B3
:106BB000BDE8384004F01EBB7C9EFF1F08B50020D6
:106BC00005F0B4FB0028FAD108BD00BF08B5642168
:106BD0000720FFF75FFF7F210B20BDE80840FFF78C
:106BE00059BF00BF10B500217B20FFF753FF0024E1
:106BF000E0B2FFF79FFF0134022004F09BF9802CE4
:106C0000F6D110BD10B504464FF4406004F0A2FA6E
:106C100004F0FAFA2CB1102C044BA8BF10241C600D
:106C200010BD024B01241C6010BD00BF7C9EFF1FE5
:106C300010B5044641F0E00004F0DCFA04F07F00F7
:106C400004F0D8FAC4F3C610BDE8104004F0D2BA7C
:106C500038B5134D2B78044641F6FF72A0F500506D
:106C6000824203F1FF33A8BF02461B0202F5005225
:106C700003F47063100443F4604343F00E0300F424
:106C8000FE005204184302F0FE42104305F084FA5D
:106C9000296801392046C9B2BDE83840FFF7C8BFAE
:106CA0007C9EFF1F38B504460D46F02004F0A2FA82
:106CB00035B1254414F8010B04F09CFAAC42F9D12B
:106CC000F720BDE8384004F095BA00BF00B50B4B83
:106CD00083B00246998818680090032AADF8041022
:106CE00002D903B05DF804FB684606218DF8052043
:106CF000FFF7D8FF03B05DF804FB00BF20000100E0
:106D000000B50B4B024683B0186899880090131F9A
:106D10004C2BADF8041002D903B05DF804FB6846B3
:106D200006218DF80520FFF7BDFF03B05DF804FBD9
:106D300028000100030203F4FE43C0F3C610184309
:106D4000704700BF03784078DB0103F47E5300F006
:106D50007F001843704700BF82B002AA114642F874
:106D6000040D002012F8013B03F07F03914243EA37
:106D70000020F7D102B07047003210B403884FF002
:106D8000010404FA01F418BF012202FA01F123EA16
:106D900004020A43028010BC704700BF70B5CEB237
:106DA0000C46054603F058FC864203D0314628467F
:106DB00003F06CFC0135284603F04EFC240A8442A3
:106DC00005D021462846BDE8704003F05FBC70BD89
:106DD00038B5054603F040FC4FF0000460F30704AB
:106DE000681C03F039FC60F30F24A0B238BD00BF6B
:106DF000F8B504460020FFF7EBFF002C00F0CD8330
:106E00004FF4AF610220FFF7C9FF4FF47A6104200D
:106E1000FFF7C4FF4FF496610620FFF7BFFF4FF462
:106E2000FA610820FFF7BAFF4FF4AF610A20FFF7BD
:106E3000B5FF40F6FC010C20FFF7B0FF4FF4966160
:106E40002220FFF7ABFF4FF416612420FFF7A6FFC7
:106E50007D212A20FFF7A2FF0C210E20FFF79EFFC5
:106E600001211020FFF79AFF02211220FFF796FF61
:106E700000211420FFF792FF00211620FFF78EFF5C
:106E800002211820FFF78AFF01211A20FFF786FF51
:106E900002211C20FFF782FF04211E20FFF77EFF46
:106EA00014212020FFF77AFF01212620FFF776FF2B
:106EB00003212820FFF772FF04212C20FFF76EFF2B
:106EC0000F212E20FFF76AFF00213020FFF766FF19
:106ED0000C213220FFF762FF00213420FFF75EFF14
:106EE00000213620FFF75AFF00213820FFF756FF18
:106EF00000213A20FFF752FF00213C20FFF74EFF10
:106F000000213E20FFF74AFF00214020FFF746FF07
:106F100000214220FFF742FF1F214420FFF73EFFE0
:106F200013214620FFF73AFF0E214820FFF736FFD6
:106F300011214A20FFF732FF0A214C20FFF72EFFD4
:106F400000214E20FFF72AFF06215020FFF726FFE1
:106F500002215220FFF722FF0C215420FFF71EFFD1
:106F600000215620FFF71AFF00215820FFF716FFD7
:106F700001215A20FFF712FF03215C20FFF70EFFCB
:106F80000A215E20FFF70AFF00216020FFF706FFBD
:106F900004216220FFF702FF01216420FFF7FEFEBB
:106FA00000216620FFF7FAFE0B216820FFF7F6FEAE
:106FB0007F216A20FFF7F2FE00216C20FFF7EEFE32
:106FC00000216E20FFF7EAFE00217020FFF7E6FEA9
:106FD00000217220FFF7E2FE00217420FFF7DEFEA1
:106FE00023210020FFF7DAFE0220FFF7F1FEB0F5C3
:106FF000805F034680F01184D24A04201380FFF79B
:10700000E7FEB0F5805F034680F0FE83CE4A06209F
:107010001380FFF7DDFEA0F52F739BB2B3F57A6FF7
:10702000024606D940F628210620FFF7B7FE40F6B3
:107030002822C64B08201A80FFF7CAFEA0F52F733E
:107040009BB2B3F57A6F024606D940F6E4410820B8
:10705000FFF7A4FE40F6E442BD4B0A201A80FFF77A
:10706000B7FEA0F5FA739BB240F6AC518B420246D4
:1070700006D94FF4AF610A20FFF790FE4FF4AF62DC
:10708000B44B0C201A80FFF7A3FEA0F5FA739BB255
:1070900040F6AC518B42024606D940F6FC010C206A
:1070A000FFF77CFE40F6FC02AB4B0E201A80FFF788
:1070B0008FFE1828034600F2A183A84A10201380EF
:1070C000FFF786FE431E9BB20F2B024604D9012117
:1070D0001020FFF763FE0122A14B12201A80FFF758
:1070E00077FE0A28034600F283839E4A1420138009
:1070F000FFF76EFE0128034604D900211420FFF794
:107100004DFE0023984A16201380FFF761FE7F286A
:10711000034600F26783954A18201380FFF758FE54
:107120000428034600F25883914A1A201380FFF77F
:107130004FFE0C28034600F249838E4A1C20138020
:10714000FFF746FE0428034600F23A838A4A1E20CF
:107150001380FFF73DFE0928034600F22B83874A80
:1071600020201380FFF734FE4628034600F21C83DC
:10717000834A22201380FFF72BFEA0F5FA739BB2FF
:1071800040F6AC518B42024606D94FF4966122205C
:10719000FFF704FE4FF496627A4B24201A80FFF723
:1071A00017FEA0F5FA739BB240F6AC518B42024633
:1071B00006D94FF416612420FFF7F0FD4FF4166254
:1071C000714B26201A80FFF703FE7F28034600F24A
:1071D000E5826E4A28201380FFF7FAFD0628034651
:1071E00000F2D6826A4A2A201380FFF7F1FDA0F14F
:1071F00032039BB2B3F5967F024604D97D212A2043
:10720000FFF7CCFD7D22634B2C201A80FFF7E0FDB9
:107210000C28034600F2B6825F4A2E201380FFF747
:10722000D7FD1E28034600F2A7825C4A3020138057
:10723000FFF7CEFD0928034600F26382584A322048
:107240001380FFF7C5FD1E28034600F25482554AFD
:1072500034201380FFF7BCFD7F28034600F24582EF
:10726000514C36202380FFF7B3FD7F28034600F200
:10727000368238206380FFF7ABFD7F28034600F29B
:1072800028823A20A380FFF7A3FD7F28034600F25F
:107290001A823C20E380FFF79BFD7F28034600F223
:1072A0000C823E202381FFF793FD7F28034600F2E6
:1072B000FE8140206381FFF78BFD7F28034600F2AB
:1072C000F0814220A381FFF783FD384D28804420C0
:1072D000FFF77EFD3028034600F2DD81344A462068
:1072E0001380FFF775FD3028034600F2CE81314C44
:1072F00048202380FFF76CFD3028034600F2BF8151
:107300004A206380FFF764FD3028034600F2B18114
:107310004C20A380FFF75CFD3028034600F2A381D8
:107320004E20E380FFF754FD0128034604D90021D5
:107330004E20FFF733FD00231F4A50201380FFF734
:1073400047FD3BE0FA9BFF1FA09DFF1FB29BFF1F65
:10735000749DFF1F469DFF1F809BFF1F589BFF1FB3
:10736000FC9CFF1F389DFF1FF29BFF1F5C9BFF1FB4
:10737000FE9BFF1F9E9BFF1F969BFF1F689BFF1F8F
:10738000869DFF1FF49CFF1FEE9CFF1F109DFF1F9B
:10739000509DFF1F9C9DFF1F6C9BFF1FEC9BFF1FC1
:1073A000489BFF1F769DFF1FD09CFF1FA29DFF1FC4
:1073B000789BFF1F549DFF1F949BFF1F431E9BB292
:1073C0000B2B024604D906215020FFF7E7FC0622CA
:1073D000CF4B52201A80FFF7FBFC0428034600F233
:1073E0003C81CC4A54201380FFF7F2FC431E9BB231
:1073F0001D2B024604D90C215420FFF7CFFC0C2290
:10740000C54B56201A80FFF7E3FC0128034604D938
:1074100000215620FFF7C2FC0023C04A58201380E9
:10742000FFF7D6FC7F28034600F21181BC4A5A20A0
:107430001380FFF7CDFC431E9BB2092B024604D9F3
:1074400001215A20FFF7AAFC0122B64B5C201A80CA
:10745000FFF7BEFC431E9BB2102B024604D903214A
:107460005C20FFF79BFC0322AF4B5E201A80FFF7E6
:10747000AFFC431E9BB21D2B024604D90A215E209D
:10748000FFF78CFC0A22A94B60201A80FFF7A0FCB2
:107490000228034600F2D580A54A64201380FFF736
:1074A00097FC0128034604D901216420FFF776FCEC
:1074B0000123A04A62201380FFF78AFCC31E9BB2FF
:1074C000012B024604D904216220FFF767FC042245
:1074D000994B66201A80FFF77BFC7F28034600F259
:1074E000AA80964A68201380FFF772FC7F28034623
:1074F00000F29B80924A6A201380FFF769FC7F2884
:10750000034600F28C808F4A6C201380FFF760FCEA
:10751000042803467DD88C4A6E201380FFF758FC60
:10752000192803466FD8894A70201380FFF750FC52
:107530000228034661D8864A72201380FFF748FC70
:107540000628034653D8834A74201380FFF740FC73
:10755000042846D82B88DFF81CE27F4F7F4A804DF5
:10756000804E814C814903F0010CAEF800C0C3F39A
:10757000400EA7F800E0C3F380071780C3F3C007ED
:107580007B4A2F70C3F30017C3F34015C3F3801376
:10759000378025800B801080F8BD4FF6FF7398422E
:1075A0003FF42EAC23283FF41FAD17287FF628ACFC
:1075B00019287FF691AC1B287FF6AEAC1C283FF44F
:1075C000C3AC1E287FF6C8AC1F283FF4CDAC2028E2
:1075D0003FF4E6AC21283FF4EFAC22287FF400AD65
:1075E000F2E474200021FFF7D9FB0020B2E700216C
:1075F0007220FFF7D3FB0023A5E700217020FFF7DF
:10760000CDFB002397E700216E20FFF7C7FB002387
:1076100089E700216C20FFF7C1FB00237BE77F2176
:107620006A20FFF7BBFB7F236DE70B216820FFF784
:10763000B5FB0B235EE700216620FFF7AFFB0023BD
:107640004FE700216020FFF7A9FB002324E700217A
:107650005820FFF7A3FB0023E8E602215220FFF7A2
:107660009DFB0223BDE60A214C20FFF797FB0A236E
:1076700056E611214A20FFF791FB112348E60E211F
:107680004820FFF78BFB0E233AE613214620FFF735
:1076900085FB13232BE61F214420FFF77FFB1F23CD
:1076A0001CE600214020FFF779FB002309E60021BA
:1076B0003E20FFF773FB0023FBE500213C20FFF792
:1076C0006DFB0023EDE500213A20FFF767FB002367
:1076D000DFE500213820FFF761FB0023D1E5002121
:1076E0003620FFF75BFB0023C3E500213420FFF7C2
:1076F00055FB0023B4E50C213220FFF74FFB0C2390
:10770000A5E500213020FFF749FB002396E500BFE7
:10771000D489FF1F6089FF1FD689FF1FE09BFF1FD1
:107720007A9DFF1F549BFF1F248AFF1F2C89FF1F78
:10773000EA9CFF1F4C9DFF1FA09BFF1F889DFF1F02
:10774000CC9BFF1F889BFF1F449BFF1FC89DFF1FF3
:10775000DE9CFF1FA49DFF1FB09BFF1FEE9BFF1F22
:10776000E29CFF1FEC9CFF1F4E9DFF1F049DFF1F0F
:107770006C9DFF1F429DFF1F0F212E20FFF70EFB68
:107780000F2352E504212C20FFF708FB042343E5D7
:1077900003212820FFF702FB032323E501212620F4
:1077A000FFF7FCFA012314E514212020FFF7F6FA75
:1077B0001423DDE404211E20FFF7F0FA0423CEE4B5
:1077C00002211C20FFF7EAFA0223BFE401211A205C
:1077D000FFF7E4FA0123B0E402211820FFF7DEFAF4
:1077E0000223A1E400211620FFF7D8FA002392E437
:1077F00002211220FFF7D2FA022376E40C210E2098
:10780000FFF7CCFA0C2358E44FF47A610420FFF719
:10781000C5FA4FF47A63FFF7F9BB4FF4AF6102206A
:10782000FFF7BCFA4FF4AF63FFF7E6BBF8B587206C
:1078300006F0C6FB204B214A054603CB1368C5F86A
:1078400003001A0C7620C5F807102B80AA70FFF7EA
:1078500071FA2E46002426F80B0FA0B2FFF7B8FAF3
:10786000FFF768FA0234762C26F8020FF5D16C1E69
:1078700005F182064FF0FF3014F8013F0827584009
:107880000F4B40F300017A1E0B4012F0FF0783EA12
:107890005000F5D1B442EFD1C043FFF75DFA3A464C
:1078A000C5F883008721284604F0C4FC2846BDE8BB
:1078B000F84006F08DBB00BF34000100300001002D
:1078C0002083B8EDF0B50E4B0E4C054693E807004B
:1078D00085B024682E88AD7801AB83E80700270CBB
:1078E000184600220B21ADF804408DF80670ADF863
:1078F0000C608DF80E5004F09DFC05B0F0BD00BF8B
:107900004000010030000100F0B5124B124D1E681E
:10791000124F0FCD87B06C460FC495E8030044F8B2
:10792000040B38683B79CDF80D00320C2320218000
:107930008DF802208DF81130ADF80060FFF7FAF9EC
:107940000022ADF80B001221684604F073FC07B06A
:10795000F0BD00BF300001004C000100ECFB000056
:10796000002004F0E3BC00BF02F02EBE70B5124C44
:1079700082B0002540230646294620460093019503
:107980008023202201F072FE20222946204602F0A8
:1079900031FA2046012102F037FA304607F0B0F8FC
:1079A00031460246204602F0BFFB204602B0BDE849
:1079B000704001F041BC00BFEC9DFF1FF0B586296F
:1079C00083B075D90546441E00F182064FF0FF30A2
:1079D00014F8012F08275040404A40F300017B1E55
:1079E0000A4013F0FF0782EA5000F5D1B442EFD10C
:1079F000C043FFF7B1F90146D5F883000190019A21
:107A0000914202D0B2F17F2F0BD105F10B00FFF7AD
:107A100099F976280BD03248FFF7A8FF002003B071
:107A2000F0BD3048FFF7A2FF384603B0F0BD05F1C6
:107A30000D00FFF787F9232840D1002440F6AC560B
:107A400013E004281AD0062821D008281FD00A28BD
:107A500028D00C2822D1A1F5FA7292B2B24201D8F4
:107A6000FFF79CF90234762C0ED004F10D00284467
:107A7000FFF768F9022C0146A0B2E2D1B1F5805FB0
:107A8000EED30234762CF0D1012003B0F0BDA1F585
:107A90002F7292B2B2F57A6FE4D8E1E7222801D0D2
:107AA000242811D1A1F5FA7292B2B242DAD8D7E7FE
:107AB0000D48FFF75BFF002003B0F0BD0B48FFF758
:107AC00055FF002003B0F0BD2A28C9D1A1F1320230
:107AD00092B2B2F5967FC5D8C2E700BF2083B8ED59
:107AE000900001007C00010064000100A40001007E
:107AF00003290CD970B5461C82B005460C463046A9
:107B000003222A4907F06AF810B102B070BD70472D
:107B10000B2C05D905222649281D07F05FF840B136
:107B20002448FFF723FF244802B0BDE87040FFF768
:107B3000C9BE05F10901032201A807F09FF801A8B9
:107B400003221E4907F04AF8D8B103221C4901A8B4
:107B500007F044F808B301A803221A4907F03EF8D9
:107B6000B0B91948FFF702FFA11E89B23046FFF7EE
:107B700025FF0028C9D0154802B0BDE87040FFF7C6
:107B8000F5BE1348FFF7F2FEFFF750FE1148F3E78A
:107B90001148FFF7EBFE1148C6E71148FFF7E6FE74
:107BA00002B0BDE87040FFF7AFBE00BF300001007B
:107BB000BC000100C4000100D8000100DC0001008D
:107BC000040101001C010100200101003401010039
:107BD000E0000100F4000100480101005C01010027
:107BE000080101002DE9F043174D2B6883B0814651
:107BF0000F469046F3B1154E34880A1992B21846D2
:107C00001146328006F05AFD28603A464946204423
:107C100002F06CFDB8F1000F09D031882868FFF739
:107C200067FF286806F0D4F900232B60338003B087
:107C3000BDE8F083054E01930846318006F0C0F997
:107C4000019B28601C46E0E7849EFF1F809EFF1F6B
:107C500010B51F4C4FF4FA70FCF7DAFB204601F028
:107C6000DFF900221146204602F0C4F82046012127
:107C700002F0CAF82046002102F0C0F80B22154994
:107C8000204602F051FA204602F064FA0F2212490F
:107C9000204602F049FA204602F05CFA0F4907221A
:107CA000204602F041FA204602F054FA204601F044
:107CB000C3FA0B4B0B4A1A604FF4FA70FCF7A8FB9F
:107CC000FFF722FE0848BDE81040FFF74FBE00BF97
:107CD000EC9DFF1F600101006C0101007C010100AF
:107CE0003CA0FF1FE57B00008401010000207047DD
:107CF00090F8392090F83800101A704790F8383012
:107D000090F839209A4205D95A1C034480F838204B
:107D1000187E70474FF0FF30704700BF90F8383042
:107D200090F839209A4286BF1B18187E4FF0FF301A
:107D3000704700BF704700BF38B50546B0F85E0019
:107D400090B195F85D301446C3F1210294420CD8ED
:107D500005F13B001844224602F0C8FC95F85D305E
:107D6000234485F85D30204638BD01201446287133
:107D7000EEE700BFB0F85E306BB190F85D30202BBD
:107D800007D8C218013380F85D30012082F83B101B
:107D90007047012303710020704700BF0023426930
:107DA00080F8383080F8393080F85C3080F85D3009
:107DB00080F85E3080F85F3006CA30B40D68046920
:107DC00043662A4383660A60A370426990F8613073
:107DD0001649146813441D7A5B7B01EBC5051B0231
:107DE0006D6803F4E06343F064032B6090F8623045
:107DF00013449D7CDB7D01EBC5011B02496803F444
:107E0000E06343F064030B6021685368194205D0B6
:107E1000036927225A70036904229A710369202298
:107E20005A71036980229A7030BC7047B80C010007
:107E300043690CCB12681A420CD0094B99420AD9FB
:107E4000084B9942036994BF1A220D225A700369A4
:107E500004229A717047036927225A70F7E700BF1E
:107E60007F1A06003F420F0010B50269D378DBB2DB
:107E7000D90604463DD510215806D17038D503F0F7
:107E8000040303F0FF02002B51D03D49626E002332
:107E90000B7084F85D30002A5BD0904794F85D3019
:107EA000002B56D02369D0229A70236994F83B2086
:107EB0001A712369012284F85C200222DA7010BD55
:107EC000304B84F860009C424AD02F4B9C4252D0E9
:107ED00094F8391013791F29DBB207D828480078A5
:107EE00020B16018013184F8391003760223D37071
:107EF00010BD5906C3D4917801F0100101F0FF00C4
:107F00000029DDD013F001031ED194F85C1094F821
:107F10005D00884281BF4B1C091984F85C3091F8E0
:107F20003B3013712369D0229A702269DEE72369FE
:107F300084F83920C0229A702369114A19790121E5
:107F400011700222DA7010BDC02393702269137978
:107F5000CCE70122002384F85D2084F83B30A1E7C0
:107F6000626994F86130094913440322187A02F0D7
:107F700043FD2269ACE7626994F861300449F3E794
:107F8000889EFF1F2490FF1F9090FF1FF17F00002D
:107F9000FD7F00000369DB7803F0200373B190F8E4
:107FA00060300133DBB2012B80F860301AD94269AE
:107FB00090F861301344187A02F09ABD70B54269A6
:107FC00003F0FF0590F8613013440446187A02F07C
:107FD0008FFDA36E5BB184F8385094F83900BDE88A
:107FE0007040184790F85F30002BE0D0704770BDAC
:107FF0000148FFF7CFBF00BF2490FF1F0148FFF7E4
:10800000C9BF00BF9090FF1F2DE9F047374FDFF841
:10801000E0903B68026982B006460093DDF800807C
:108020000021A025D3789B065BD53B680193019B7B
:10803000C8EB03030F2BF5D949B1102BF2D0002068
:108040009070336980229A7002B0BDE8F08772693F
:1080500096F8613013440521187A02F043FF7269E3
:1080600096F861301344012193F812A0504602F0B3
:1080700039FF09240021504602F020FF2B46013B26
:10808000FDD10121504602F019FF2B46013BFDD1E5
:10809000013CEFD1706996F8611001444FF4A07271
:1080A0000C7A4B7B09EBC4011B02496803F4E063C3
:1080B00043F064030B6096F862300344997CDB7DE7
:1080C00009EBC1011B02496803F4E06343F0640358
:1080D0000B60013AFDD13269D3789B064FF0010164
:1080E000A3D4012002B0BDE8F08700BFB09EFF1FFF
:1080F000B80C0100F0B503691222DA7002699378B6
:1081000003F0200385B004460D46002B5ED0B42357
:1081100093703C4922690B680093009E05E00B6850
:108120000193019B9B1B042B42D8D37803F02003BF
:1081300003F0FF00002BF2D094F85D30002B31D01B
:108140004FF0000E4FF0020C04EB0E0393F83B309F
:1081500013710B680393039F206907E09B060DD5FD
:108160000B680293029BDB1B052B28D8C378DBB27C
:1081700003F0020202F0FF06002AEFD080F803C0ED
:108180002669F378DBB2DF0632462DD49F062BD565
:10819000DB0731D40EF1010E94F85D305FFA8EFEEC
:1081A0007345D1D800201DBB002384F85E3004E065
:1081B0009070236980229A70042005B0F0BD86700B
:1081C0002369802204209A7005B0F0BD03F0FF06F9
:1081D000FFF71AFF10B9042005B0F0BD236984F839
:1081E0005F60B0229A7094E78023B3700420DAE7CE
:1081F00026698023B370D7E7BEF1000F0CBF0220C1
:108200000320F6E7B09EFF1F2DE9F0410669002527
:10821000122780F8385080F83950F770D0F810C025
:108220009CF802E00EF0200E88B004468846154601
:108230001E46BEF1000F49D0B4238CF80230784BB3
:1082400021691A680092DDF800E006E01A680192E0
:108250000198CEEB0000042830D8C87800F0200048
:1082600000F0FF070028F1D04FEA480242F0010277
:10827000D2B20A711A680292DDF808E0206906E0BD
:108280001A6803920399CEEB010105292AD8C17817
:1082900001F0020101F0FF070029F1D04FF0020CBC
:1082A00080F803C02269D17811F0110722D12DBBCB
:1082B000002E0CBFA0238023937003E08F702369EE
:1082C00080229A70384608B0BDE8F0810EF0FF07B2
:1082D000FFF79AFE0028F5D0236984F85F70B0227A
:1082E0009A70ACE787702369802238469A7008B08C
:1082F000BDE8F081802393700027E3E7012D75D05E
:10830000A021917021690A79BE4667464FF0A80CFA
:108310001A680492049805E01A680592059A121AE0
:10832000052A4AD8CA7802F0020202F0FF08002AA1
:10833000F2D0CF702169CA78D2B212F0100F08467D
:108340005AD1920658D5013DEDB2012D49D0BEF16A
:108350001F0F3BD90A79012DDAD11A680692069DC2
:1083600005E01A680792079A521B052A46D8C27878
:1083700002F0020202F0FF01002AF2D00223C370D1
:108380002269D378DBB2D9063AD49B0634D5B02320
:10839000BEF11F0F93703FD8226904EB0E031279D0
:1083A0001A760EF1010E5FFA8EFE16B12369802255
:1083B0009A7084F839E0774684E781F8028023696F
:1083C00080229A70774684F839E07BE704EB0E024E
:1083D00091F8048082F818800EF1010E5FFA8EFE8B
:1083E000B9E781F802C021690846B0E7A821917079
:1083F0002069BE460279B0E7774663E78170DEE721
:108400001021A023D170013BFDD12269937803F0A4
:10841000F7037746937055E723691B79C5E700BFDB
:10842000B09EFF1F0148FFF71FBD00BF2490FF1F34
:108430000148FFF719BD00BF9090FF1F704700BFB4
:1084400038B5144C037801225B000546204684F8B9
:108450003B3084F85E2084F85D20FFF78BFC2046DB
:108460000021FFF747FE0B4C2978012320461A46CE
:10847000FFF7CAFE0128F6D194F8383094F8392075
:108480009A4205D9E218013384F83830107E38BD9D
:10849000FF2038BD2490FF1F38B51B4C0378012204
:1084A0005B000546204684F83B3084F85E2084F863
:1084B0005D20FFF75FFC20460021FFF71BFE124CFA
:1084C0002978204601230222FFF79EFE0228F6D1DA
:1084D00094F8382094F839108A420FD2531CDBB23A
:1084E000A018994284F83830007E0AD92344023219
:1084F0001B7E84F8382040EA032038BD4FF6FF7019
:1085000038BD40F47F4038BD2490FF1F0C2901D9AD
:10851000002070470231490001F0FE01FFF7BCBFA7
:1085200070B50C4C0378164601255B00204684F894
:108530003B3084F85E5084F85D50FFF71BFC3146F9
:108540002046FFF717FC29462046BDE87040FFF79C
:10855000D1BD00BF2490FF1FF8B505460F46164653
:10856000412421463A462846FFF7DAFF611C0234CF
:10857000C9B232462846E4B2FFF7D2FF592CF0D1F7
:10858000F8BD00BF38B504460D463548FFF706FC78
:108590006322802120462570FFF7C2FF012002F0F0
:1085A000C9FC204600225E21FFF7BAFF20465D216C
:1085B000FFF746FF242801D0002038BD20460622C0
:1085C0000C21FFF7C9FF204601222B21FFF7A8FF4E
:1085D000204601222C21FFF7A3FF20460E222D2149
:1085E000FFF79EFF204600222E21FFF799FF20462D
:1085F00001222F21FFF794FF204605223021FFF7AB
:108600008FFF204601223121FFF78AFF20460022FA
:108610003221FFF785FF204600223321FFF780FF3C
:10862000204600223421FFF77BFF2046002235211F
:10863000FFF776FF204600225B21FFF771FF2046FF
:1086400010225C21FFF76CFF204620225D21FFF7FE
:1086500067FF20468F225E21FFF762FF012038BDB1
:108660002490FF1F10B4047F4160022CC26002D02E
:1086700010BC01F0D7BB836810BC184790E80C0011
:10868000F0B41C6859682568164F174E29432160BD
:10869000164D17491760D66015611160417A154A69
:1086A0005C180A3194F8244053F8215002EBC401BD
:1086B00049680D60017A5C1803EB8101247ECD6965
:1086C00002EBC40149680D60817A581803EB8103FD
:1086D00090F83000596B02EBC002F0BC536819608F
:1086E000704700BF01401F000110003801100078E2
:1086F00000001F80B80C0100704700BFF0B50C1ED1
:10870000BDF8146034DBB0F906701919B942C4BF62
:108710003B1B1BB2002BA6461CDD002A1146B8BF2E
:10872000D11D02F00705CC10826A012007FB04E18D
:10873000A840012E0A44C0B21ED00CD3022E09D18B
:10874000013B12FA83F3013A12F8011F41409A42A9
:108750001170F9D1F0BDC043013B12FA83F3C0B2EE
:10876000013A12F8011F014093421170F9D1F0BD96
:1087700023441BB20024C6E7013B12FA83F3013AFB
:1087800012F8011F01439A421170F9D1F0BD00BFE8
:10879000F8B50D1E0EDB14461F46064601F03AFBE7
:1087A000A84207DD002C05DB304601F037FBA04274
:1087B00001DCF8BDF8BD304601F02AFB022853D099
:1087C00003284BD0012806D16540F3886C406540F2
:1087D000013B5D1B2DB2012F03D02AD3022F14D0F1
:1087E000F8BD002C2246B6F90630B06AB8BFE21DCB
:1087F00042F3CF0202FB035504F00704435D01215D
:1088000001FA04F41C434455F8BD002C2246B6F985
:108810000630B06AB8BFE21D42F3CF0202FB035537
:1088200004F00704435D012101FA04F45C4044555F
:10883000F8BD002C2246B6F90630B06AB8BFE21D7A
:1088400042F3CF0202FB035504F00704435D01210C
:1088500001FA04F423EA04044455F8BD3389013BCA
:10886000591B25460CB2B6E7F18832890139013A25
:108870004D1B141B2DB224B2ADE700BF2DE9F04112
:10888000079E9DF91880089D04461F4600F0C0FF12
:108890000D4B0E480E4984F83380FF22002F08BF8D
:1088A0001F4684F82F20002384F8302084F83120DC
:1088B00084F832202060A665E56567626165236201
:1088C000A3622046BDE8F0812490FF1F1002010042
:1088D0000110013810B50446806A034B236008B1CB
:1088E00005F076FB204610BD10020100F8B5436A82
:1088F000DBB190F82C200125AA4083F83B2083F8B7
:108900005E5083F85D500446406A03680E461B685B
:1089100000219847606A036831461B6898472946DA
:10892000606ABDE8F840FFF7E5BBC26BC56C136831
:10893000046A23EA050313604CB122684FF0004338
:10894000D3625163D36A002BFCDA936BF8BD836B5F
:10895000466B0825802410E03768426C3A43326049
:108960001F68826C3A431A601A68876C013D22EADC
:1089700007024FEA54041A6007D02142ECD1326852
:10898000476C22EA07023260EAE7F8BD70B5044698
:10899000406A0D4600282BD0A16DFFF749FA002D43
:1089A00020460CBFA621A721FFF7A0FF606A20B1D7
:1089B000E16DBDE87040FFF73BBA216C226D08689D
:1089C000236A02430A6093B1DA7A82B1D00703D5F1
:1089D000224A99691160DA7A910703D5204AD96948
:1089E0001160DA7A520702D51E4A1B6A136070BD05
:1089F000236A002B2BD0D97A626DE1B172B6D97A95
:108A0000CE0706D51848D9680668314099610160DB
:108A1000D97A880706D51548196906683140D961A1
:108A20000160D97A4E0705D5114859690668314069
:108A30001962016062B61B68D968914207D00D487F
:108A400018600D49DA6042F0804018611960226CAC
:108A5000216D136823EA01031360A0E700E100E041
:108A600004E100E008E100E080E100E084E100E0F2
:108A700088E100E001403F0000003F80436A2DE9AB
:108A8000F04105460E469046002B3ED090F82C1043
:108A90000124A14083F83B1083F85E4083F85D40D9
:108AA000406A036800211B6808F1FF379847FFB24E
:108AB000B8F1000F23D03744A046013E686A16F88B
:108AC000011F03681B6898470134B742E4B216D00F
:108AD000202CF3D10121686AFFF70CFB95F82C20BC
:108AE0006B6A520083F83B2083F85E8083F85D80D8
:108AF000686A036800211B6898470124DEE7686AFA
:108B00000121BDE8F041FFF7F5BAC26BC16C1368F3
:108B100023EA010306EB080413604FF00048A64265
:108B20000ED02B6A16F801EB63B11A68C2F82C80DC
:108B3000C2F834E0D36A002BFCDAA642936BF0D182
:108B4000BDE8F081AB6BD5F834C008208021DCF89B
:108B500000206F6C1EEA010F14BF3A43BA43CCF8F1
:108B600000201A68AF6C3A431A601A68AF6C01387B
:108B700022EA07024FEA51011A60E8D1CFE700BFAD
:108B800070B50446406A0D46002828D0A16DFFF755
:108B90004FF920462946FFF7A9FE606A20B1E16D32
:108BA000BDE87040FFF744B9216C226D0868236A64
:108BB00002430A6093B1DA7A82B1D00703D5234A1F
:108BC00099691160DA7A910703D5214AD969116050
:108BD000DA7A520702D51F4A1B6A136070BD236AF6
:108BE000002B2BD0D97A626DE1B172B6D97ACE075B
:108BF00006D51948D9680668314099610160D97A6B
:108C0000880706D51548196906683140D9610160A1
:108C1000D97A4E0705D5124859690668314019625C
:108C2000016062B61B68D968914207D00D48186090
:108C30000D49DA6042F0804018611960226C216DA4
:108C4000136823EA01031360A3E700BF00E100E01B
:108C500004E100E008E100E080E100E084E100E000
:108C600088E100E001403F0000003F802DE9F04135
:108C7000044686B0806A9DF830801E460F46154631
:108C8000B4F90830002800F04281DA1D48BF03F132
:108C90000E02B4F90630D21003FB02F2002105F0F7
:108CA000BBFCB4F90820202A00F39280B4F9061026
:108CB000A34B0120203A733902EBD27201EBD17140
:108CC0004FF0200E029073208DE8014042F34F02D6
:108CD00041F34F01204600F051FE606A84F82D7088
:108CE000002800F04D81002D40F08A80B4F9083052
:108CF000202B14BF3D253C2584F82C50B8F1000FE3
:108D000040F0858006B394F93300002818DBC0B228
:108D1000012102F0E7F8012194F8330002F0CEF8C7
:108D2000012002F007F9002194F8330002F0C6F8A0
:108D30000A2002F0FFF8012194F8330002F0BEF897
:108D4000606A002800F08280A16DFFF771F80422AC
:108D50007C492046FFF792FE217A0139C9B22046AC
:108D6000FFF7C4FD784904222046FFF787FE94F9F7
:108D70002D30012B14BF142110212046FFF7B6FD22
:108D8000042272492046FFF779FEB4F90630802BA1
:108D900000F09280602B00F0A680D9212046FFF7DA
:108DA000A5FD94F92D30012B14BFF121222120467D
:108DB000FFF79CFD204606226549FFF75FFE606ACB
:108DC00050B3E16DFFF734F8012006B0BDE8F08143
:108DD000B4F906105F4B0120403A52394FF0400E73
:108DE000029002EBD272522001EBD1718DE801406A
:108DF00042F34F0241F34F01204600F0BFFD6CE704
:108E00006DB284F82C50B8F1000F3FF47BAFFEF741
:108E1000C5FF002E94D076E7216C226D0868236A86
:108E200002430A6073B1DA7A62B1D00703D54A4AC5
:108E300099691160DA7A91077CD4520702D5474AC2
:108E40001B6A1360012006B0BDE8F081236A002B85
:108E50002BD0D97A626DE1B172B6D97ACF0706D537
:108E60003F48D9680568294099610160D97A8E0721
:108E700006D53C48196905682940D9610160D97A4D
:108E80004D0705D5384859690568294019620160C0
:108E900062B61B68D968914207D0344818603449DB
:108EA000DA6042F0804018611960226C216D13680D
:108EB00023EA010313604AE7B4F90830202B00F0DD
:108EC0008680402B7FF469AF2A4920460322FFF7B2
:108ED000D5FD94F92D30012B14BFCF219F212046C1
:108EE000FFF704FD59E7B4F90830102B7FF455AFB4
:108EF000214920460322FFF7C1FD94F92D30012BB3
:108F000014BFAF2110212046FFF7F0FC45E7DA1D22
:108F100048BF03F10E02B4F90630D21003FB02F28F
:108F20001046059205F04CF8A06200283FF44DAFC2
:108F3000059AB3E6114AD9691160DA7A7DE700BF74
:108F400068020100480401004C04010050040100C3
:108F5000540401005C04010000E100E008E100E0CD
:108F600080E100E084E100E088E100E001403F00B2
:108F700000003F80640201001C07010004E100E0E2
:108F8000012194F83100244F01F0ACFF94F8320035
:108F9000012101F0A7FF94F9312094F9323057F8FC
:108FA0003220E26357F83330206A23640125E564F8
:108FB00025651A682A431A6078B1B8F1000F3FF4AA
:108FC00028AFFFF75BFB002E3FF4BAAE9BE604220E
:108FD00012492046FFF752FDDFE6294694F82F009C
:108FE00001F080FF294694F8300001F07BFF94F9EE
:108FF0002F2094F9303057F83220626357F833301D
:109000006564A5641A68A36322F001021A60002E49
:109010003FF496AE77E600BFB80C01006002010095
:10902000B0F90820D31D48BF02F10E03B0F90620A5
:10903000806ADB1002FB03F2002105F0EDBA00BFED
:10904000F0B50029BDF814502EDBB0F90660B1422E
:109050002ADA002A59DBB0F9087014461C44BC42D5
:10906000C4BFBB1A1BB2002B1EDDD2B2D408D0F88D
:1090700028E016FB041112F00702DBB20EEB01042C
:1090800021D0C2F10807FAB2374F9342BF5C0CD22D
:10909000C3EB020CFF2646FA0CF6012D07EA060781
:1090A0003FD005D3022D36D0F0BD012D39D030D2BE
:1090B0001EF8016026EA07070EF801709342F3D309
:1090C000B0F906100C449A1AD2B2072A10D9022D10
:1090D00036D0002D14BFFF26002613462670083B0D
:1090E000B0F90610DBB2072B0C44F7D802F00702E8
:1090F000002AD9D01D4B012D9B5C1DD017D3022D0A
:10910000D2D1227853402370F0BD13441BB2002209
:10911000A1E7022D25D11EF8016077400EF80170FD
:10912000CCE71EF8016037430EF80170C6E72278DD
:1091300022EA03032370F0BD227813432370F0BDAD
:1091400011462378DB4323700839B0F90630C9B2E1
:1091500007291C44F5D812F00702A5D0034B9B5CED
:10916000CFE73444AFE700BF00020100F001010087
:1091700070B4C47DBDF80C50022C18D0032C1FD045
:10918000012C0BD0002A03DBB0F90840944201DC2B
:1091900070BC7047039570BCFFF7B0BAC4880395E4
:1091A000013CA41A0A4621B270BCFFF749BF0689E8
:1091B000C488013E641AB21AE41A12B221B2E1E77D
:1091C00004890395E41A641A114622B270BCFFF7B1
:1091D00037BF00BF70B4C57DBDF80C60022D1AD03A
:1091E000032D12D0012D03D0039670BCFFF728BFCA
:1091F000C488E41AA41A0A4621B2002A03DBB0F993
:109200000840944213DC70BC70470489013C641A26
:10921000114622B2F1E7C48805890396013CAD1AD4
:10922000ED1A621A11B22AB270BCFFF709BF039699
:1092300070BCFFF763BA00BF2DE9F8430446406AEB
:10924000002863D0A16DFEF7F3FD05227449204686
:10925000FFF714FCA1790139C9B22046FFF746FB9C
:10926000B4F90820E588A66AD31D48BF02F10E03B1
:10927000DB10626A15FB03F51FFA85F8002A7BD024
:1092800094F82C300125AB4082F83B3082F85E50D8
:1092900082F85D50606A036840211B6808F1FF375F
:1092A0009847BFB2B8F1000F23D03744A846013E1B
:1092B000606A16F8011F03681B6898470135B742BA
:1092C000EDB216D0202DF3D10121606AFEF712FF16
:1092D00094F82C20636A520083F83B2083F85E8068
:1092E00083F85D80606A036840211B689847012508
:1092F000DEE70121606AFEF7FDFE606A002800F0EB
:109300008D80E16DBDE8F843FEF792BD236A002B26
:109310002BD0D97A626DE1B172B6D97ACE0706D573
:109320004048D9680568294099610160D97A8D075C
:1093300006D53D48196905682940D9610160D97A87
:10934000480705D5394859690568294019620160FF
:1093500062B61B68D968914207D035481860354914
:10936000DA6042F0804018611960226C216D136848
:1093700023EA0103136068E7E26BE36C1168276A74
:109380000B4306EB080913604FF0004E4E450DD01D
:1093900016F801CB2FB33A68C2F82CE0C2F834C0FB
:1093A000D36A002BFCDA4E45936BF1D1226C236D0E
:1093B00011680B43136097B1FB7A83B1D90703D5CA
:1093C0001D4BBA691A60FB7A9A0703D51B4BFA69E1
:1093D0001A60FB7A5B0702D5194B3A6A1A60BDE83E
:1093E000F883A36BD4F8348008208021D8F80020BB
:1093F000656C1CEA010F14BF2A43AA43C8F8002079
:109400001A68A56C2A431A601A68A56C013822EA0A
:1094100005024FEA51011A60E8D1B7E7276AC5E7AC
:10942000F801010080E100E084E100E088E100E073
:1094300001403F0000003F8000E100E004E100E067
:1094400008E100E02DE9F04F85B09946BDF938708C
:10945000BDF83CA0BB1AC1EB090B002BB8BF5B42A7
:10946000BBF1000FB8BFCBF1000B5B450D461646B4
:109470000093804648DC4D453A4633464CDC19465D
:1094800013460A46C5EB09019B1A89B2002B0CB2A0
:10949000B8BF5B4204EBD474BE42ACBF4FF0FF32A6
:1094A00001224D45039102924FEA640429DC9BB2EC
:1094B00001930DE0D8F80070BF69B847019BE41A2A
:1094C000A3B21CB20135002C2DB211DBA94518DB6B
:1094D000009B5B452A46534631464046EADCD8F8B5
:1094E000002053469769294632464046B847E5E78B
:1094F000029A1644039AA94502EB030436B224B239
:10950000E6DA05B0BDE8F08F4A462B46B946354647
:109510004D4517461E46B2DD304629463E464D466D
:1095200007468946AEE700BF10B404682469A44624
:1095300010BC604730B40468BDF808500295A46BB5
:10954000A44630BC604700BF30B40468BDF8085082
:109550000295E46BA44630BC604700BF70B4046859
:10956000BDF90C60BDF8105003960495246CA44618
:1095700070BC6047704700BF10B582B0B0F90C20D6
:1095800001910168009200220C6CB0F90A3011467A
:10959000A04702B010BD00BF704700BF01F003013B
:1095A0000129C17506D0032904D0C28803894281EC
:1095B000838170470289C38842818381704700BFDD
:1095C0002DE9F0410568134E6F6986B0B742044635
:1095D000BDF8308010D1013B13441BB20093CDF88D
:1095E00004800B46AD6A2046A8472368DB6AB34275
:1095F0000AD106B0BDE8F081059304920391B84703
:1096000003A925680EC9E6E7204606B0BDE8F0418B
:10961000184700BF759500002DE9F0410568124E0E
:109620006F6986B0B7420446BDF830800FD1013B68
:10963000CDF804800B4400921BB2AD6A2046A847C7
:109640002368DB6AB3420AD106B0BDE8F081059316
:1096500004920391B84703A925680EC9E7E720469D
:1096600006B0BDE8F0411847759500002DE9F04FB0
:109670000568DFF858B06F6985B05F450646BDF9EB
:109680003890BDF83CA00C46904615D11F19BC423D
:109690000CDACDF800A0214601342D6A4B46424633
:1096A000304624B2A847BC423568F2DBEB6A5B4522
:1096B00007D105B0BDE8F08F0393B8473568039B29
:1096C000E4E7304605B0BDE8F04F18477595000057
:1096D0002DE9F04387B099420546BDF93840BDF801
:1096E0003C6025D0A24212D00768DFF88080D7F80E
:1096F0001490C14532D18DE850002846BC6AA0477D
:109700002B68DB6A434524D107B0BDE8F08399425A
:1097100002DD08461946034628680E96C46B0133DD
:109720005B1A1BB22846A44607B0BDE8F043604769
:10973000A24202DD134622461C4628680E96631C90
:10974000846B9B1A1BB22846A44607B0BDE8F043C1
:109750006047284607B0BDE8F043184705930492D8
:109760000391C84703A92F680EC9C4E77595000087
:109770002DE9F04FD0F800E0DFF89090DEF814B05B
:1097800083B0CB450446BDF93080BDF834A00D460A
:1097900017461E4631D1CDF800A0DEF824B0294688
:1097A00033463A462046D8472368CDF800A008F152
:1097B000FF323A44D3F824B0294612B23346204649
:1097C000D8472368CDF800A02946D3F820B03A4600
:1097D00043462046D8472068CDF800A0711E294492
:1097E0004346056A09B23A462046A8472368DB6A21
:1097F0004B4506D103B0BDE8F08FD847D4F800E060
:10980000C9E7204603B0BDE8F04F18477595000042
:10981000F0B4002401264FF6FF75094F076004716C
:10982000C475C48104824476C461867506768582D7
:109830004582C180028141818281F0BC704700BFB6
:10984000280701002DE9F04F85B00668BDF84450A7
:10985000BDF93880CDF8008004460195D6F848B0AF
:109860000392BDF93C60BDF9407089469A46D847DD
:1098700023680195009742465146D3F84880204618
:109880003346C0472068039B0E930F95856C4B466B
:109890003A4631462046AC4605B0BDE8F04F604739
:1098A0002DE9F04F87B01746BDF94040009125469D
:1098B000E91D059344BF2B4603F10E010268BDF874
:1098C000486053690294C91003912B49BDF9444083
:1098D00001968B42824645D1002C3CDD029B3C44E4
:1098E0005E1EB6B24FF0000923B2049301364D4616
:1098F000029B002B28DD059B002403EB090806E0F2
:10990000EDB22B0604F1010411D4A6421CD0A1B281
:1099100011F0070F23B24FEA4505F1D1002BB8BF74
:109920000733DB10013418F803502B06EDD5009BEC
:10993000D2F818B019443A4609B2019B5046D847AC
:10994000A642DAF80020E2D1039B01379944049B38
:109950003FB2BB42CCD1D36A074A934206D107B08B
:10996000BDE8F08F9847DAF80020B5E7504607B019
:10997000BDE8F04F184700BF7595000070B4BDF901
:109980000C60BDF91050BDF8144003960495059481
:1099900070BCFFF785BF00BF2DE9F04F93B0904634
:1099A0000591C1691090BDF870000790BDF87490E2
:1099B0009DF878A00493002900F0CD800A7A0AC9A6
:1099C000894604998A1AD2B203EBC203BAF1010F95
:1099D000DA780B9293F905201E8893F802B00F9263
:1099E00093F9064079D913B2099323B20C93109BD3
:1099F0001A68A94B1193194653698B4240F0A6800F
:109A00000B9B002B55D01FFA88F300210D93C846FD
:109A10002344DDF8409006910E930F460C46BBF1AF
:109A2000000F3FD0BDF818100C9B03971FFA8AF067
:109A3000CB1813FB00F304900E9801440D980344D7
:109A400009B21BB20A910893002505E00135EBB27B
:109A500064009B45E4B222D9039B2B44590703D1F0
:109A6000731C18F806409EB22306EFD5099BBDF87B
:109A70001000E91811FB00F10598BAF1010F0FFA77
:109A80008AF301441CD0079801900093D26909B26F
:109A900017464846089AB847D9F80020D6E7039FEA
:109AA0005F44FFB2069B0B9901330693DBB29942E8
:109AB000B5D8D36A119A934243D113B0BDE8F08F61
:109AC0000F9B191893690A9A29441F4609B2079BEC
:109AD0004846B847D9F80020B8E700230C9309930B
:109AE00085E70A9A0D9B0132013B52B213F0FF0346
:109AF0000A920D936FD1DDF81890079BDDF83C803A
:109B0000DDF820A04B4517D0BAF1010F00F0C88056
:109B10000B9A109DCDF804900BEB8B014FEACB0311
:109B20000A4400931146DEF81C405346424609B2EF
:109B30002846A047D5F800E0DEF82C30119A934271
:109B4000BBD0109813B0BDE8F04F1847109D2846C1
:109B500098472A6854E7109A0598B2F90A30834268
:109B6000ABDDB2F90C304345A7DD062313FB0A0336
:109B7000002BA2DD08EBCA03002B9EDD537E2BB920
:109B8000049BAF2B02D90133DBB20493109BD3F8B3
:109B900000E0414B11931A46DEF81430934240F036
:109BA0008E801FFA88F30E9308339BB2BDF8142001
:109BB000059305230D9300230A93CDF83C800FFAFB
:109BC0008AF3DDF84080CDF818900B921FFA8AFBDB
:109BD000CDF820A099460A9ABDF810000B9C0E9D66
:109BE0000523194611FB00232C481146C75C039737
:109BF00002FB0B4214FA81F312B21BB209920C93CE
:109C00002C462E461CE0089B0999012B2AB24B4694
:109C100040462DD0079F0197CDF80090DEF81CA09C
:109C2000D047D8F800E0039B5B0801340393059B01
:109C3000A4B25D445E44A342ADB2B6B23FF451AFAC
:109C4000039BD807DFD4079B069A9342EBD0089B6F
:109C5000012B16D0069B0193CDF80090DEF81CA0D6
:109C600009994B4632B24046D047D8F800E0DAE7CF
:109C7000DEF818A0079B0C9922B2D047D8F800E074
:109C8000D1E7DEF818A00C991346404622B2D0471F
:109C9000D8F800E0C7E700BF75950000780701001D
:109CA0000B99109DCDF800900531DEF8204009B2E7
:109CB000424608232846A047D5F800E03CE7109C20
:109CC00020469847D4F800E06BE700BFF0B5C369C1
:109CD00085B004462BB30A2968D00D294AD01A7AD8
:109CE000914247D3587A884244D35D688A1A05EB7B
:109CF000C205AA78002A50D0E87800284DD0207EEE
:109D000000283AD095F905E0B4F90E00A67DB4F923
:109D10000A70724406FB0202BA4262DCB4F91020F7
:109D200030E00A2956D00D2924D0027E002A4BD0DB
:109D3000B0F90E00A57DB4F90A60062212FB0502F7
:109D4000B2423EDD228AE38102EBC50212B218461E
:109D50002282A78A668A02950B468DE8C0000146DA
:109D60002046FFF719FEA37DE28903EB430302EBD4
:109D70004303E381012005B0F0BDA67DB4F90E00D8
:109D8000B4F91020B4F814E0678A02960B468DE807
:109D9000804001462046FFF7FFFD2979E389A27D37
:109DA000012001FB0233E38105B0F0BD0022C28136
:109DB0009A7A817D038A01FB02330382012005B078
:109DC000F0BDB4F91020C4E7857DB4F91020B0F9D6
:109DD0000E00BEE7028A817DC38102EBC1030382CC
:109DE000C8E70020E0819B7A228A03FB062212B298
:109DF0002282C7E7C1810282704700BF002908BFE5
:109E000001218175704700BF81824182704700BF88
:109E1000C07D7047B0F90A00704700BFB0F90C0070
:109E2000704700BF10B4EFF3108272B6437F33B9AE
:109E3000017F012907D003290FD00123437702B9FD
:109E400062B610BC7047124C2168A1B11149436140
:109E50000B68836108605861EFE70F4C216881B19E
:109E60000E4943610B688361086058610C4B4FF0E9
:109E700080511960E1E7074B416181612060186002
:109E8000DBE7064B4161816120601860EEE700BFAF
:109E90009C9EFF1F989EFF1F8C9EFF1F909EFF1F82
:109EA00004ED00E070B5EFF3108272B60C4C206840
:109EB00080B10C4E00254369236073B19D6102B9E6
:109EC00062B6457783689847EFF3108272B62068D0
:109ED0000028F0D102B962B670BD3360EFE700BF71
:109EE0008C9EFF1F909EFF1FFFF7DCBF184A30B407
:109EF0001468002C27D0036821688B420ED2CB1A3D
:109F000000218460C1602360E0601060022303755B
:109F100030BC704711688B42144608D3A2685B1AA4
:109F20000360002AF6D18260C460A060EEE7D268C8
:109F3000C2608460E060C568CB1A0222A86023601A
:109F4000027530BC70478460C4601060DEE700BFFB
:109F5000949EFF1FF8B5224E34682CB32368002B63
:109F60003AD1204F1D4604E03468ECB12368002B41
:109F700032D1A36803B1DD602069336003682575C1
:109F80001B68BB4221D1037F4560022BC46020D0F7
:109F9000FFF748FF6368002BE6D023602046FFF7F9
:109FA000A5FF3468002CE1D1EFF3108372B60E4A9E
:109FB00000211068116003B962B628B18468FFF708
:109FC00095FF20460028F9D1F8BD22460021984788
:109FD000E0E783689847DDE7013B2360E4E700BFE3
:109FE000949EFF1F65860000A49EFF1F024A13680F
:109FF00001331360FFF7AEBFB09EFF1F704700BF75
:10A000000368F0B4FBB1002501249D60DC601B4CAB
:10A010001A601C44241104F144056A1103269200BD
:10A020009E60174F0679174B47F8241002F16042E3
:10A0300002F5614205F01F05012000FA05F5E6541E
:10A040001560F0BC7047104C236843F40003236094
:10A0500000BF0E4B0E4DA4F58734A4F59E74012667
:10A060001E60234604609C68002CD0D01033AB42A5
:10A070000360F8D1002303601846E2E7008FFCBFBD
:10A08000FC90FF1F44E400E03C800440007003406B
:10A09000407103400168A9B10B4BF0B40B441B1194
:10A0A0000A4E0B4F0B4D46F8237003F1440202F0A9
:10A0B0001F0401235211A340002445F822308C6074
:10A0C0000460F0BC704700BF008FFCBFFC90FF1F16
:10A0D000FD9F000080E100E0024A034B0121116076
:10A0E0001B6818470C710340FC90FF1F024A034B8A
:10A0F000012111605B6818471C710340FC90FF1F31
:10A10000024A034B012111609B6818472C710340E0
:10A11000FC90FF1F024A034B01211160DB681847C6
:10A120003C710340FC90FF1FF8B50E4671B17AB147
:10A130000746144600253B6816F8011B1B68384685
:10A140009847013C0544F6D12846F8BD0846F8BDBD
:10A150001046F8BD00B5064A036812885B6883B0F4
:10A1600001A9ADF804200222984703B05DF804FB72
:10A17000780C0100F0B507468BB0002A33D0012AD5
:10A1800008BF0A2251B3212400E0F4B2B1FBF2F57A
:10A1900002FB1511C8B2092900F1300198BFC8B2FD
:10A1A0000AA988BF3730214488BFC0B201F8240C07
:10A1B000661E2946002DE8D133B1013CE4B20AAB5A
:10A1C00023442D2203F8242C3B6801AA11195B6853
:10A1D0003846C4F1220298470BB0F0BD30228DF80A
:10A1E00025202124E8E70368C9B21B6898470BB013
:10A1F000F0BD00BF0029BABF49422D2300230A2227
:10A20000FFF7B8BF374A384913681B06FCD40B6800
:10A2100013F08003F8D172B634490A78002A5FD06F
:10A22000334A3448F0B4344C176806682568D4685B
:10A230000C303E44143200681268304F35442C44D0
:10A2400020440244C2F34E022D4E2E482E4D2F4C78
:10A2500042F400423A60376806682D682C4A246848
:10A260000C303E44006812682A4F35442C44204488
:10A270000244C2F34E02284E2848294D294C42F48C
:10A2800000423A60376806682D68274A24680C3017
:10A290003E4400681268254F35442C442044024453
:10A2A000C2F34E02224E2348234D244C42F4004276
:10A2B0003A60376806682D68214A24680C303E44AD
:10A2C0000068126835442C4420440244C2F34E0214
:10A2D0001C4842F4004202600B7062B6F0BC70474A
:10A2E00062B6704724B0034024B00B40A99EFF1F04
:10A2F00038B003403CB0034040B003402CB00340B2
:10A3000058B003405CB0034060B0034064B0034009
:10A310006CB0034030B0034038B00B403CB00B4051
:10A3200040B00B4044B00B404CB00B402CB00B4045
:10A3300058B00B405CB00B4060B00B4064B00B40B9
:10A340006CB00B4030B00B4030B42948294A2A4B3E
:10A350002A4D6024E121047011701B78284C082BD1
:10A3600030D00A2B2748284937D00C2B0CBF352278
:10A370003D2212232A60236002600B60234B244994
:10A380001B78244ABBB101230B601360224B234985
:10A390001B78234A012B26D9042B0FD9082B1ED951
:10A3A000102B94BF862387230B6013601D4B012263
:10A3B0001A7030BC70470B601360E7E784230B60B2
:10A3C0001360F3E700F58E200F49083001221323B4
:10A3D0002A60236002600B60D0E73922F7E785230B
:10A3E0000B601360E2E780230B601360DEE700BFC1
:10A3F00000400740014007400C91FF1F08B0034098
:10A400000CB0034008B00B400CB00B40AC9EFF1FDB
:10A4100020B0034020B00B400D91FF1F24B003403B
:10A4200024B00B40A99EFF1F0C2830B417D910236D
:10A43000984228BF18461C46104A114D1178181A28
:10A440008C42287018D00F4913700B7823B10E4935
:10A450000E4A00230B60136030BCFFF775BF0A285B
:10A4600002D90C231C46E7E7082802D90A231C4618
:10A47000E2E708231C46DFE730BC70470C91FF1F62
:10A48000A89EFF1FA99EFF1F24B0034024B00B40CD
:10A4900028282FD8334B2DE9F0411E5CFF2E2BD0FE
:10A4A000314B1B78002B2AD132062CD472B62F4D9B
:10A4B0002F4C2F46012326602B7062B672B623689C
:10A4C0001B060CD43B781BB9F4E72B78002BF1D09A
:10A4D00062B602F09BF972B623681806F5D5254BD3
:10A4E0001B6800222A7062B6234A107843FA00F0F3
:10A4F000BDE8F081002070470020BDE8F081FFF743
:10A5000081FE3206D2D572B61C4DDFF87C801C4C21
:10A5100006F04007FFB206F03F06D8F80030DFB182
:10A5200023F01003C8F8003001232660134A2B7073
:10A5300062B672B6236819060CD413781BB9ECE71F
:10A540002B78002BE9D062B602F060F972B623686E
:10A550001B06F5D50B4BC3E743F01003C8F80030DA
:10A56000E2E700BF7C0C0100A99EFF1FAB9EFF1F0E
:10A5700000B0034010B00340A89EFF1FAA9EFF1F1B
:10A5800000B00B4010B00B400CB00B400A4A0B4916
:10A59000136843F4805313600B7843B9084BC0220F
:10A5A0001A70084B80F30C0000B218807047044BFF
:10A5B00080221A70F5E700BF2C800440AC9EFF1F7C
:10A5C00021C00C4000C00C40F0B51B4B1B4E59681D
:10A5D00018689A68DB6885B06C460FC433789907B1
:10A5E0001DD5174A174C1378174913F0700318BF7D
:10A5F0001370164A164B802717700026332003224B
:10A6000026706D4608701A7072B6043C45F001055C
:10A610002046A84762B6237813F0700309D10D4B8A
:10A62000064901E0013B02D00A78D207FAD505B00D
:10A63000F0BD237005B0F0BDA80C01000100024080
:10A6400000000240040002400B00024007000240EC
:10A650000A000240410D0300B0F5006F0AD210B5A8
:10A66000094B1B78DB07044606D504F1A05000789F
:10A67000C0B210BD00207047FFF7A6FF04F1A05044
:10A680000078C0B210BD00BF01000240B0F5006FFD
:10A6900017D238B50F4B1B78DA070D46044611D593
:10A6A00004F1A0500378AB420AD00B4A137813F0A0
:10A6B000700318BF1370074A05701378DB07FCD5C9
:10A6C00038BD7047FFF780FF04F1A0500378AB421C
:10A6D000EBD1F5E7010002400000024008B5F5F7B4
:10A6E000E3FFF7F7CBFD02F091F8FAE7844641EA81
:10A6F000000313F003036DD1403A41D351F8043BFA
:10A7000040F8043B51F8043B40F8043B51F8043B4B
:10A7100040F8043B51F8043B40F8043B51F8043B3B
:10A7200040F8043B51F8043B40F8043B51F8043B2B
:10A7300040F8043B51F8043B40F8043B51F8043B1B
:10A7400040F8043B51F8043B40F8043B51F8043B0B
:10A7500040F8043B51F8043B40F8043B51F8043BFB
:10A7600040F8043B51F8043B40F8043B51F8043BEB
:10A7700040F8043B51F8043B40F8043B403ABDD25A
:10A78000303211D351F8043B40F8043B51F8043BFC
:10A7900040F8043B51F8043B40F8043B51F8043BBB
:10A7A00040F8043B103AEDD20C3205D351F8043B8B
:10A7B00040F8043B043AF9D2043208D0D2071CBF57
:10A7C00011F8013B00F8013B01D30B880380604680
:10A7D000704700BF082A13D38B078DD010F00303F6
:10A7E0008AD0C3F10403D21ADB071CBF11F8013B66
:10A7F00000F8013B80D331F8023B20F8023B7BE7B5
:10A80000043AD9D3013A11F8013B00F8013BF9D2DF
:10A810000B7803704B7843708B7883706046704779
:10A8200008B5104C08E0236859050DD423681A05B3
:10A830000FD42368DB0411D423685803F3D500F048
:10A840008DFE23685905F1D502F044F823681A05F6
:10A85000EFD502F0D5F82368DB04EDD500F0F0FC6D
:10A86000EAE700BF3480044008B5FFF7D9FF00BF16
:10A87000014B10221A80704700200540704700BF2E
:10A88000094908B50B6830B16A461844A2F58052F0
:10A89000904202D20860184608BD03F063FB0C2307
:10A8A00003604FF0FF3008BD1091FF1FFEE700BFAF
:10A8B000EFF3138070B9EFF310836BB9EFF30582F8
:10A8C0005AB94FF48070EFF311832BB1984228BF2F
:10A8D000184670474FF0FF3070470F2A01D81846CE
:10A8E000F1E7014BD05CEEE7F0E300E0F0B44D1E81
:10A8F0002E46002400E00134B0FBF2F302FB13000B
:10A90000092800F130078ABF3730F8B2C0B206F824
:10A91000010F1846002BEED10A1953704CB1107874
:10A9200015F8016F28700133E01A834202F80169BB
:10A93000F5DB0846F0BC7047704700BF10B40F4B02
:10A9400053F8302092F880422CB1012369B182F88B
:10A95000803010BC704703EBC0035B681A6841B9D4
:10A9600022F002021A6010BC704782F8003110BC5D
:10A97000704742F003021A6010BC7047B80C010027
:10A980001C4A02EBC00301295B6811D004291BD0CB
:10A9900052F83000002280F8802229B1022920D00C
:10A9A000032922D01A6070474FF480721A607047F2
:10A9B00052F830004FF4A27280F880121A601A68C0
:10A9C00022F020021A60704752F830104FF4A27241
:10A9D000012081F880021A601A6842F020021A6091
:10A9E000704740F203121A6070474FF481721A6088
:10A9F000704700BFB80C0100212848D8F8B5042AD8
:10AA000044D8DFE802F0484B4E0345004FF41026CF
:10AA10002B4B03EBC0030D465C68216811F4E06129
:10AA200048D0284B284A2949C3F89C2104F14042C8
:10AA30002748C3F8A411A2F59221264FC3F8A0011C
:10AA40007C292548C3F8A871C3F8AC012CD9A2F51C
:10AA500094237C2B2AD9A2F596237C2B28D9A2F506
:10AA600098237C2B29D9A2F59A227C2A27D81B4827
:10AA700072B6236823F4702343F08072C4F3840118
:10AA80001643236040F82150266062B6F8BD704737
:10AA90004FF43026BCE74FF40026B9E74FF44026C8
:10AAA000B6E74FF42026B3E70D48E1E70D48DFE7AE
:10AAB0000D48DDE7FFF764FFB3E70C48D8E7F8BDC2
:10AAC000B80C01000082FF1FF188FF1F9988FF1F4B
:10AAD000C588FF1F6D88FF1F4188FF1FEC91FF1F76
:10AAE0001491FF1F4C91FF1F9C91FF1FCC91FF1FE2
:10AAF0001A4B03EBC00010B4426802F14043A3F5C7
:10AB000092217C2923D9A3F594217C290DD9A3F581
:10AB100096217C291FD9A3F598217C2919D9A3F561
:10AB20009A237C2B11D80E4C00E00E4C72B61368A1
:10AB30000D4823F08773C2F3840123F4803343F07C
:10AB40008073136044F8210062B610BC7047074C54
:10AB5000ECE7074CEAE7074CE8E700BFB80C010058
:10AB6000EC91FF1F4C91FF1F39A900001491FF1FAA
:10AB7000CC91FF1F9C91FF1F30B4054B054D064C37
:10AB8000002210211A602A602060196030BC7047D2
:10AB900014D0034004D0034000D00340282838B527
:10ABA0002ED0002904464FDD5F4B1B78012505FAA6
:10ABB00003F28A4202D8212837D938BD0338C2B2FD
:10ABC000012A3AD9202C4AD0192C48D0574A126869
:10ABD00002FB011222FA03F31D2800F29B80DFE83A
:10ABE00000F0928B847D9999766F999999999999AA
:10ABF00099999968615A53994C9999999999994554
:10AC0000494B1B780B2B08D90C2B1CBF0C3B194153
:10AC10000846BDE83840FFF7B9BCC3F10C039940C2
:10AC20000846BDE83840FFF7B1BC2946FFF786FE6D
:10AC30002946BDE83840FFF7A3BE3D4A126802FB33
:10AC4000011222FA03F3C7E72128B6D80021FFF743
:10AC500075FE20460121BDE83840FFF791BE354A18
:10AC6000126802FB011222FA03F3B5E73249334AB4
:10AC70000B604FF45173136038BD3149314A0B609A
:10AC80004FF45173136038BD2F49304A0B6040F2C6
:10AC90004443136038BD2E492E4A0B6040F24443B2
:10ACA000136038BD2C492D4A0B6040F244431360B9
:10ACB00038BD2B492B4A0B6040F24443136038BD2A
:10ACC00029492A4A0B6040F24443136038BD2849A1
:10ACD000284A0B6040F24443136038BD2649274A96
:10ACE0000B6040F24443136038BD2549254A0B6090
:10ACF00040F24443136038BD2349244A0B604FF4AB
:10AD00005173136038BD2249224A0B604FF45173CE
:10AD1000136038BD212C3FF650AF7F29D4BF0021EE
:10AD20000121204693E700BFF491FF1F08800340F4
:10AD30000890034008800B4010800B4048A004405E
:10AD400018800B404CA004401880034008B0044019
:10AD50001080034004B004404080034018C0044009
:10AD60003880034014C004402880034010B00440E1
:10AD7000208003400CB004403080034010C00440E9
:10AD8000488003401CC004401890034034900440A5
:10AD9000109003403090044038B1102828BF102094
:10ADA000044AC3B2107813707047024A0123107826
:10ADB00013707047F491FF1F2DE9F8430E4680464B
:10ADC0003249334D304603F053F847F6122300283A
:10ADD0001ABF1D464FF002094FF00109002425FA61
:10ADE00004F002F04FFE4FF05E51074602F0A2FE63
:10ADF0000146304603F050F830B90134072CEED14B
:10AE0000E80902F03FFE07463146384602F046FFA9
:10AE10004FF07C5102F084FD03F078F84FF6FF729A
:10AE20009042A8F1030328BF1046012B29D9B8F19D
:10AE3000170F17D8174B23FA08F303F0010383F019
:10AE4000010223B9B8F1190F0FD0BDE8F883124BF6
:10AE5000124D13491A6044EAC9042A6008601C6054
:10AE6000BDE8F883B8F1200FECD10E4B0E4D0F4921
:10AE7000002244EAC9041A602A6008601C60BDE828
:10AE8000F8830B4B0B4D0C49F2E700BF001BB7409A
:10AE9000006CDC026006F000008003400480034088
:10AEA0000880034000800B4004800B4008800B406A
:10AEB000009003400490034008900340212801D8EB
:10AEC000FFF73CBD704700BF212806D8044B53F85C
:10AED000303093F80002C0B270470020704700BFC6
:10AEE000B80C0100212801D8FFF74ABD704700BF08
:10AEF00072B60C490C4B0D4A1B680868126862B6A2
:10AF0000520102D5322B88BF01300949C3F5BB334A
:10AF10004FF47A72FF33A1FB031302FB00F000EB46
:10AF200093107047B09EFF1F18E000E004ED00E0B2
:10AF3000ABAAAAAA2DE9F843054672B6204F214BC9
:10AF4000214A1B683C68126862B6520102D5322B56
:10AF500088BF013495B3C3F5BB331C4EDFF8649052
:10AF6000DFF86480FF334FF47A72A6FB031302FB11
:10AF700004F404EB931472B6D9F800103A68D8F8C8
:10AF800000E062B6C1F5BB33FF33A6FB03031EF03E
:10AF9000806FC4EB93134FF47A7002D0322988BFCC
:10AFA000013200FB0233B3F57A7F04D3013D05D0B3
:10AFB00004F57A74DFE701F029FCDCE7BDE8F883EB
:10AFC000B09EFF1F18E000E004ED00E0ABAAAAAAC3
:10AFD000F8B52D4B2D49DFF8D0E0DFF8D0C02C4E6E
:10AFE0002C4D2D4C2D4A2E4F4FF4000018604FF081
:10AFF000807018604FF0007018604FF0806018602B
:10B000004FF0006018600020086028234BF6FF71A5
:10B01000CCF80010CEF80030336013602B60236052
:10B020003B60B3629362092245F8242CC4F8D80F20
:10B0300005F57F65C7F8D41F07F5FF2707F5FA6701
:10B04000C6F8F83F2B6006F5FF26C4F8D42F05F5A7
:10B05000FD2504F5FF24386006F2F47611483160CE
:10B0600005F5FF6504F5FD642B6023600260FFF7C2
:10B070006BF91920FFF75EFF00F0B6FF40F21310E6
:10B08000BDE8F840FFF756BF08E100E00480034048
:10B0900014800340248003402C8003401C80034024
:10B0A0003480034000800B400C8003400880034044
:10B0B0002DE9F84F214B1B6807460BB101221A708E
:10B0C000DFF888901E4D99F80040DFF884801D4E0F
:10B0D0000134272C8ABF4FF0000A5FFA84FA5446E5
:10B0E000AB462B78A34216D1FFF7E2FB40281FDCCA
:10B0F00033791B06F5D59BF800300133272B86BF2B
:10B1000000221346DAB218F80330DBB2F3712A706A
:10B110002B78A342E8D00C490A4BFFB208F8047020
:10B120000120AC22087089F800A0DA70BDE8F88F21
:10B13000FF28D6DD01F06AFBD3E700BF289FFF1F81
:10B14000259FFF1F00C00640249FFF1F2C9FFF1F4D
:10B15000BC9EFF1F1C4BDFF894C01A681B49F0B55A
:10B1600042F480521A4D1A60DFF884E0194F1A4EEB
:10B170001A4C00238CF800304FF451722B701F28AA
:10B1800040F213358EF800303B70337025600A6052
:10B1900012D819460124124A124D117012485470E7
:10B1A00000212C27402693724FF4003491701174C3
:10B1B000D7702E700460F0BDC0F34431C0F3471463
:10B1C00000F01F03E7E700BF348004400CC00440D8
:10B1D000B99EFF1F259FFF1F249FFF1F08C004402B
:10B1E00000C0064031E400E004E100E0B89EFF1F2B
:10B1F0002C9FFF1F034B1B68DB0401D5FFF758BFD3
:10B20000704700BF3480044010B5044C237823B14C
:10B2100001F0FCFA2378002BFAD110BD249FFF1F08
:10B22000054A064B10781B78C0B2DBB2984238BF93
:10B230004030C01A704700BFB89EFF1FB99EFF1F65
:10B2400030B42B4B1A7994061FD52A48DA79037843
:10B25000294901333F2B0978C8BF00238B42D2B262
:10B2600003D0264CD9B2E2540170254A116861B16D
:10B27000244A1278D2B2934236BFC2F140029B1ADE
:10B280009B18272BC4BF01230B70194AD378DBB25C
:10B29000180611D45A060DD5154B1B795B0609D536
:10B2A000194B1A491B6800220A7003B11A70104B1F
:10B2B0002C22DA7030BC704711790906EAD514499E
:10B2C00010480C780178C9B28C420DD04A1C272A4C
:10B2D00084BF00210A460F4D054C98BFD1B2AA5C2D
:10B2E000D2B2E2710170D5E76C21D170D2E700BF14
:10B2F00000C00640B89EFF1FB99EFF1FE49EFF1FBF
:10B30000B49EFF1F259FFF1F289FFF1F249FFF1F25
:10B310002C9FFF1FBC9EFF1F21282FD8184B195CA4
:10B32000FF292BD0174B184ADFF870C003EBC00081
:10B33000F0B54368DFF868E0144F154D154E002452
:10B340001C60DEF80030012043F020038840CEF876
:10B35000003014604FF4A07338602E60C2F800C053
:10B36000013BFDD113689B05FCD42023013BFDD19B
:10B37000094B09B233F8110080B2F0BD00207047CC
:10B38000C80D0100B80C01000050044008500440F2
:10B3900004500440000002030051044080014A00B0
:10B3A00038800440431E032B14D872B60A4951F862
:10B3B000230068B170B4094C058834F8132046683E
:10B3C00041F82360521B24F8132062B670BC70470A
:10B3D00062B6704700207047889FFF1FCCA1FF1FF7
:10B3E000013803280BD872B6074B53F8203043B10D
:10B3F00000205B680130002BFBD162B67047002053
:10B4000070471846F9E700BFDC9FFF1F30B472B6E3
:10B410002B4A13781D0706D52A4B196A002936D006
:10B42000996A002941D053781C0706D5254B196C21
:10B4300000293ED0996C002939D09378190705D599
:10B44000204B196E002936D0996E89B1D3781B072D
:10B4500007D51C4BD3F880207AB3D3F8882011216C
:10B460003AB162B6184B00221A7030BC00F04ABEE6
:10B470000D21154C154D227843F8315003EBC103D3
:10B480000830013A5860227062B630BC704704221E
:10B490000D4C0F4D217843F8325003EBC2030830B6
:10B4A0004A1E5860227062B6EFE70521E1E70921E4
:10B4B000DFE70822ECE70C22EAE71022E8E700BF0A
:10B4C000EC0D01000080FF1F05A0FF1FC800400019
:10B4D00088004000431E032B1DD81B4A400140F04A
:10B4E000100030B4104472B6184CE25C032A1BD82A
:10B4F000DFE802F00212151703220D88E25410F063
:10B50000080F14BFC823882343EA054308310360AA
:10B51000416062B630BC704708300222EDE7052278
:10B52000EBE708300422E8E7094A52F8230038B173
:10B53000084A52F82300416042F8231062B6E9E756
:10B5400042F82310034AF7E70080FF1F14A0FF1FF3
:10B55000DC9FFF1FEC9FFF1F00BE70472DE9F04FDF
:10B56000DFF818B3DFF818A387B044E0AD4F4FEA17
:10B57000930807EBC809013ED9F8042003F008033B
:10B58000F6B2A2F1080003F0FF04002B40F00181A5
:10B5900057F838301B0C99B222F8081C002B00F029
:10B5A000EF80A14B22F8064C42F8044C53F82620B9
:10B5B000002A00F0CF819D4D55F8263058609C4CF4
:10B5C00045F8260034F81630194424F8161000F017
:10B5D00079FD002800F0C281964A974B19F0080FB8
:10B5E00000F1080018BF1346C9F8040047F83830C6
:10B5F00008238BF800309BF80040E4B265071CD5A7
:10B600008E4B1B78B3B18E490A7802F0FF0322B14A
:10B61000013BDBB20B7003B900BE8A490A7802F025
:10B62000FF032AB1013BDBB20B70002B00F06881F5
:10B6300000F066FE04238BF8003004F0080303F0EA
:10B64000FF02002B00F0C9809AF80030DBB21E091F
:10B650008CD19A08DFF8CC9159F8321009EBC2006E
:10B66000C1F38301013940680C2900F28580DFE8CD
:10B6700001F07A7A838383838383468383830700FD
:10B680000168714D4068714F714E6860296088B2E1
:10B6900040F281610024674B49F832304FF0010ECF
:10B6A00088423C60C9F81040C9F8184086F800E0AC
:10B6B0005C4A00F2E780B0F5D06F80F01B82B0F5F5
:10B6C000817F00F0D98100F26981802800F02A8210
:10B6D000822840F0D781A98801F07F01042900F277
:10B6E000D1815C485C4A8900084414705470017828
:10B6F0008C0740F1608382F800E0022173E1534F30
:10B700003A682AB3554B524E554819883478057813
:10B7100040298E4645F0020828BF4FF0400E002C0D
:10B7200084F001043470CEEB01010CBF8824C824DE
:10B7300009EBC80689B285F0010544EA0E4472603F
:10B74000198049F8384072440570002965D03A6084
:10B750003D4B1A88B2F5A06F0ED100219A7859702E
:10B76000404B1A7008E038493F4C0D68A54200F084
:10B770009880304949F832103C4A0123137037E76A
:10B780002C4A2D4B19F0080F18BF134647F83830D4
:10B790002EE700F0B7FC364A364952F82630002B27
:10B7A00000F0E38058688C5D42F8260003F108023F
:10B7B000C9F80420032C05D8DFE804F02C02292660
:10B7C00002228A551A8819F0080F0CBF8823C82353
:10B7D00043EA024347F838300AE7E00700F1938074
:10B7E000210600F1D180A20706D5234A2349137808
:10B7F0000220DBB213700870E30602D51F4B102243
:10B800001A7007B0BDE8F08F04228A55DAE70522E6
:10B810008A55D7E703228A55D4E7BEF1400F18BFF7
:10B82000002294E70080FF1F889FFF1F349FFF1FA7
:10B83000CCA1FF1FC80040008800400010A0FF1FDF
:10B84000999FFF1F84A0FF1FFC9FFF1F309FFF1FBA
:10B85000989FFF1FC020074008A0FF1F449FFF1FA5
:10B8600004A0FF1F982007402109000394200740EF
:10B87000DC9FFF1F14A0FF1F882007408020074087
:10B8800090200740B0F5106F00F07C8140F2A3805B
:10B8900040F62112904240F07B82A54A01231370AA
:10B8A0006AE74C68A3498C427FF463AF0178A92909
:10B8B0007FF45FAF417845297FF45BAF8178C2297F
:10B8C0007FF457AFC1786B297FF453AF9A489B4EF2
:10B8D0000178347881F00105002C41F002010570F7
:10B8E0000CBF8820C82084F0010449F8310009EB1E
:10B8F000C10193483470002505244D60047038E779
:10B9000000F064FF94E68F4B89488B491A614FF031
:10B91000020E80F800E08C4F0A708C491960996023
:10B920008B4E8C4D8C4C9A610D213970FF213170FA
:10B93000DFF84CE229702270884D894A8EF8001099
:10B940009F27012406F8047C5D600470DA6007B06C
:10B95000BDE8F08F43F82600824D30E6824A47F872
:10B96000380013780133137042E68B5D032B00F22D
:10B97000BA8001A252F823F0F1B50000F1B5000041
:10B98000D1B90000CBB900006F49724B80220D2065
:10B9900008701A70A2077FF52FAF26E740F2023237
:10B9A000904240F0ED81AA8802F07F02042A69D813
:10B9B0006D88002D66D16449CDF804E092001144F1
:10B9C0000A7842F002020A70C1E101238B550FE6AA
:10B9D00000238B550CE6B0F5086F53D16349644AD8
:10B9E000097811707146ED888D4280F0E8825248E6
:10B9F0000478402DAE4644F0020C28BF4FF0400EB4
:10BA000002EB0E0309EBCC01029301234A604FEADB
:10BA10000E48CEEB050101930025C82242EA080337
:10BA200084F0010249F83C3035700270DFF814C12F
:10BA3000424BDFF8048149BBBEF1400F7FF42DAFCC
:10BA400042F0020C09EBCC03029ADFF8F8E05A60EE
:10BA50008DBB0D0445F088059DF804304EF83C5030
:10BA60000A4433700470134640297FF416AF002156
:10BA7000404A3B60118010E7AA8802F07F02042A46
:10BA800040F28B81304A0F23137006E74029D7D943
:10BA900042F002020CEBC200029E4660BDB19DF86E
:10BAA000045035481D703346403988F80040403313
:10BAB0004CF83200DCE79DF8043033700D04029B33
:10BAC000047045F0C8050B444EF83C50CCE79DF897
:10BAD00004501D70029B1D4888F8004040394033D7
:10BAE0004CF83200C4E719F0080F0CBF02230323FF
:10BAF0008B557DE521494A68002AC3D06C88B5F88A
:10BB000004E003E00C314A68002ABBD00B88A34252
:10BB1000F8D14B887345F5D1240A032C0CBF11785A
:10BB2000098960E7124A0221147054705BE700BF74
:10BB3000942007400100040004A0FF1F989FFF1FEE
:10BB4000999FFF1F0080FF1FC02007408800400012
:10BB5000882007408020074098200740489FFF1F0B
:10BB60009C9FFF1F349FFF1F05A0FF1F10A0FF1FFA
:10BB700008A0FF1F449FFF1FC8004000F00D0100F8
:10BB80008C200740B248116AAC7804700C0600F1B2
:10BB90009881D9F82820AF49100600F1DB81D9F847
:10BBA0003020AC49120600F1D081D9F83820A949DB
:10BBB000130600F1C581D9F84020A649150600F109
:10BBC000BA81D9F84820A349140600F1AF81D9F809
:10BBD0005020A049100600F1A481D9F858209D49B1
:10BBE000120600F19981D9F860209A49130600F1F4
:10BBF0008E81D9F868209749150600F18381D9F81C
:10BC000070209449140600F17881D9F87820914980
:10BC1000100600F16D81D9F880208E49120600F1DE
:10BC20006181D9F888208B49130600F15581D9F834
:10BC300090208849150600F14981D9F89820854956
:10BC4000140600F1FF808448844A854901908548A4
:10BC5000854D864C049700230596029580460F4635
:10BC600016461D460394306828B1446800F04AFA2D
:10BC70002046002CF9D100233360029B38681A4615
:10BC8000002342F8253028B1446800F03BFA2046F2
:10BC9000002CF9D100223A60019A98F80030114640
:10BCA000002241F8042B039A0191023B4FF000015E
:10BCB00022F81510032B07D8DFE803F05D025D02C0
:10BCC0004FF0010388F800300135042D06F1040619
:10BCD00007F1040708F10108C5D1654C654D2278CC
:10BCE000654B049F059E0021100729701A7000F112
:10BCF0009280624962780A700021C9F83010C9F850
:10BD000038101107DFF84C816ED4A2785C49DFF857
:10BD100044810A7000211207C9F85010C9F8581060
:10BD20004BD4E27857494B4C0A7013074FF000018F
:10BD3000C9F87010C9F8781000F1AE80337801931B
:10BD4000002283F00105C9F89020C9F8982000214D
:10BD5000029188468E460A464B48047844F0020C0D
:10BD600009EBCC030393019B002B039B5A600CBF90
:10BD70008822C82252E64FF0000388F80030A3E77B
:10BD8000B0F5A06F7FF47EAE012300250193DEE7BE
:10BD900040F621229042F7D074E66D88002D7FF4A2
:10BDA00071AE3A49CDF804E0920011440A7822F0CD
:10BDB00002020A70CBE7022115E600F083F90028A1
:10BDC00000F0EB800830324AC8F86400C8F8602000
:10BDD00000F078F9002800F0DA8008302D4AC9F820
:10BDE0006C00C9F868209CE700F06CF9002800F0AE
:10BDF000E0800830264AC8F84400C8F8402000F027
:10BE000061F9002800F0CF800830224AC9F84C00C0
:10BE1000C9F8482079E700F055F9002800F0A5801E
:10BE200008301B4AC9F82400C9F8202000F04AF95C
:10BE3000002800F094800830164AC9F82C00C9F890
:10BE4000282056E7D1F89C00083800F05BF9FAE6A4
:10BE500010A0FF1F0080FF1FEC9FFF1F889FFF1F88
:10BE6000DC9FFF1F14A0FF1F349FFF1FCCA1FF1FEB
:10BE7000EC0D010005A0FF1FC4200740C8200740AB
:10BE8000CC200740D020074004A0FF1FC02007405F
:10BE900088004000C800400000F014F9002870D06D
:10BEA00008304F4AC4F88400C4F8802000F00AF932
:10BEB000002860D008304B4AC9F88C00C9F88820A7
:10BEC0003CE7506A083800F01DF962E6D1F89400AA
:10BED000083800F017F9B0E6D1F88C00083800F007
:10BEE00011F9A4E6D1F88400083800F00BF998E6BF
:10BEF000C86F083800F006F98DE6486F083800F082
:10BF000001F982E6C86E083800F0FCF877E6486E62
:10BF1000083800F0F7F86CE6C86D083800F0F2F861
:10BF200061E6486D083800F0EDF856E6C86C083850
:10BF300000F0E8F84BE6486C083800F0E3F840E61B
:10BF4000C86B083800F0DEF835E6486B083800F0BA
:10BF5000D9F82AE6C86A083800F0D4F81FE62A782B
:10BF6000C9F8280001322A70C3E62A78C9F82000EF
:10BF700001322A705AE72A78C9F8880001322A70FB
:10BF8000DCE62A78C4F8800001322A708EE72A782D
:10BF9000C9F8680001322A70C3E62A78C8F8600040
:10BFA00001322A7014E72A78C9F8480001322A7051
:10BFB000ABE62A78C8F8400001322A701FE7402912
:10BFC0008E4628BF4FF0400E02EB0E030293012372
:10BFD000CEEB01014FEA0E4800250193BCE600BFFD
:10BFE00088004000C8004000F8B500F08FFD294BE4
:10BFF00029482A4C2A4F2B4DDFF8BCC0DFF8BCE0A3
:10C00000294E00221A605A609A60DA601A615A61F9
:10C010009A61DA611A625A629A62DA621A635A6340
:10C020009A63DA631A645A649A64DA641A655A6520
:10C030009A65DA651A665A669A66DA661A675A6700
:10C040009A67DA67C3F880200168C3F8842041F456
:10C0500080210160C3F307212170C3F30740134916
:10C0600038701B0E2B70FF238CF80030104D8EF8AB
:10C07000003010480B700123337084F86420702660
:10C080004FF40074102207F82C3C2E70046081F8E5
:10C09000F820F8BD0080FF1F348004409C2007403A
:10C0A000B0200740B42007409420074010200740EC
:10C0B00049E400E008E100E08020074088200740D4
:10C0C000704700BF72B60D480268B2FA82F30F2BB8
:10C0D00010DC4FF00041D94022EA0102026062B652
:10C0E000074803EBC303DB00C2180021C150104610
:10C0F0005160704762B60020704700BFF891FF1F83
:10C10000BC83FF1F0D4B0E4AC31AA2FB03231B095E
:10C110000F2B0CD80B4A127852B972B60A484FF05E
:10C120000041026821FA03F31A43026062B67047C5
:10C13000064A1278002AF0D0FFF768B9BC83FF1FC7
:10C14000398EE33805A0FF1FF891FF1F10A0FF1FD5
:10C1500038B50E4B0E4C1B68218805468BB1B1F5E6
:10C16000917F05D20B4A4B1C55549BB2238038BD9E
:10C170000022084898470021064A5554012323808D
:10C1800038BDB1F5917FEDD338BD00BF3CA0FF1F96
:10C19000D6A1FF1FDCA1FF1F2DE9F843214E224F3E
:10C1A0003168012380463B70B1B1204D4B8801EBD3
:10C1B0008302013300240F2BC2F808802C7004D8AE
:10C1C0004B8000233B70BDE8F88340230B800320A5
:10C1D000FFF780F93460F4E7DFF8549099F8003005
:10C1E000002BF0D0114D45F6215408E0013C12D04F
:10C1F0002B7883B900F00AFB99F800307BB103205B
:10C20000FFF7EEF80528F1D8FFF75CFF0146306034
:10C210000028EBD0CAE701232B70BDE8F883BDE806
:10C22000F88300BF58A0FF1F2CA0FF1F5CA0FF1FBA
:10C2300010A0FF1F1201F8B5D5B2A1B3012943D058
:10C240004378044600781B0643EA004040F47040FF
:10C2500045F004068F1E3043FFF79EFF022F04F1C6
:10C26000020314D9053414F8023C14F8032C14F812
:10C27000010C1B0443EA0223334343EA0060033FFB
:10C28000FFF78AFF022F234604F10304EBD8022FA5
:10C2900023D0012F0DD045F4774040F00500BDE8D4
:10C2A000F840FFF779BF14482843BDE8F840FFF78E
:10C2B00073BF187845F4770545F0060545EA002078
:10C2C000BDE8F840FFF768BF03780C4845EA03452E
:10C2D0002843BDE8F840FFF75FBF1A78587845F06B
:10C2E000774545F0070545EA022545EA0040BDE8E7
:10C2F000F840FFF751BF00BF06F0F70007F000F766
:10C3000038B5084B1C7824B9074D296809B14B880A
:10C3100003B938BD9B000B800320FFF7DBF82C60CE
:10C3200038BD00BF2CA0FF1F58A0FF1F2DE9F04112
:10C33000AD4E33680746002B00F092801D885A8866
:10C34000910803EB81010432AA428C6842D25A80E0
:10C3500004F00F064FEA1428A449A6F1080208F0D9
:10C360000F00C4F30313062A00F101050B701AD95C
:10C37000B31E012B5FFA88F04ED9052E48D0042E4B
:10C3800000F0A481731F022B7FD90F2E0ED1F72846
:10C3900042D8F02802D0964B1B883BB1FFF7D8FE5D
:10C3A0000020BDE8F08127B1BD4202D00020BDE8E9
:10C3B000F081082EC4F3033300F08780092E11D0DA
:10C3C0000A2E40F094800A2BF0D18A4B8A4A1B68CF
:10C3D000A02181E01846FFF795FE0420FEF7E2FF5A
:10C3E0003060B5E7092BE1D1270E00F07B81834B4C
:10C3F000814A1B689021C4F307461170EDB2FCB26C
:10C40000002B00F09D80224631462846984797E051
:10C41000F02843D9F72841D0F1380E28C6D801A317
:10C4200053F820F0DBC50000BFC50000ADC500001B
:10C43000ADC30000ADC300009FC50000ADC3000048
:10C440007FC60000ADC3000049C6000063C60000FF
:10C4500087C50000ADC300006FC5000053C50000D4
:10C46000674B1B78002BA1D00420FEF79BFF0346EF
:10C47000306000289AD00588002D7FF460AFFFF768
:10C4800041FE35602846BDE8F081FFF761FEC4F348
:10C490000740FFF75DFE072E02D1200EFFF758FE82
:10C4A000534B584A198858481468584D524A0170DD
:10C4B00000270E0AF0201F802E7010700CB301228E
:10C4C0005348A0470120BDE8F081082B7FF46EAFF0
:10C4D000504B494A1B688021C4F307461170EDB2E6
:10C4E000240E6BB3284622463146984728E00B2E8F
:10C4F00011D10B2B7FF45AAF474B3F4A1B68B02139
:10C50000EAE7464B1B68002B00F0FB804048984749
:10C510000120BDE8F0810C2E40F000810C2B7FF44F
:10C5200045AF3F4B344A1B68C0211170EDB2C4F3D4
:10C530000746002B00F0C88028463146240E984755
:10C540003849314A314B0D7016701C700120BDE81E
:10C55000F081354B1B68002B00F0D6809847C4F360
:10C560000746254BEDB2240E83F80080E8E72F4BF9
:10C570001B68002BF2D12E4B1B68A3B1FE209847FD
:10C58000C4F30746EDE72B4B1B68002BE6D1284B85
:10C590001B6843B1FC209847C4F30746E1E7264BEC
:10C5A0001B68002BDAD1C4F30746DAE7234B1B687C
:10C5B000C4F30746002BD4D030469847D1E7204B30
:10C5C0001A68002AEFD0260C630C06F07F0003F4F3
:10C5D0007E531843F6B29047C3E71A4B1B68C4F367
:10C5E0000746002BE8D1BCE764A0FF1FDAA1FF1FBC
:10C5F000D6A1FF1F40A0FF1FD4A1FF1F74A0FF1FE3
:10C6000010A0FF1F3CA0FF1FD8A1FF1FD9A1FF1F33
:10C61000DCA1FF1F6CA0FF1F70A0FF1F54A0FF1F15
:10C6200030A0FF1FDBA1FF1F1CA0FF1F20A0FF1FCA
:10C6300024A0FF1F60A0FF1F50A0FF1F68A0FF1FC6
:10C6400038A0FF1F4CA0FF1F3F4B1B68002B85D15C
:10C650003E4B1B68002BA6D0FA209847C4F3074630
:10C660007FE73B4B1B68002B7FF478AF374B1B6891
:10C67000002B98D0FB209847C4F3074671E7354B51
:10C680001B68002B7FF46AAF304B1B68002B8AD0ED
:10C69000F8209847C4F3074663E70E2B7FF486AE75
:10C6A0002D4A2E4B1268E0211970002A47D0260C23
:10C6B000610C06F07F0301F47E511943EDB2A1F540
:10C6C000005128469047F6B2240E39E7FFF740FDA7
:10C6D000C4F30740FFF73CFD200EFFF739FD0020B3
:10C6E000BDE8F0811E4B1D4A1B6880211170EDB220
:10C6F000C4F3074683B1314628463A4698473C463C
:10C700001EE70120BDE8F081104B1B68002B3FF4B1
:10C710004AAFFF20984746E71C4611E70D2EBCD1D3
:10C720000D2B7FF443AE0F4B0C4A1B68D0211170C8
:10C73000EDB2C4F30746002B7FF4FEAEC4E7C4F3AA
:10C740000746EDB2240EFBE648A0FF1F24A0FF1F02
:10C7500028A0FF1F18A0FF1F34A0FF1FD4A1FF1F98
:10C760006CA0FF1F44A0FF1F38B5164D2868E0B12C
:10C7700001884488A14213DD03191B7A83B104F1B7
:10C780000803C2180C1B002302E012F8011F21B19C
:10C790000133A342F9D1204638BD1C46204638BD9E
:10C7A000FFF7B0FC0020286038BD074B1B780BB9A1
:10C7B000002038BD0220FEF7F5FD28600028D7D103
:10C7C000F6E700BF80A0FF1F10A0FF1F0D4B1B78D6
:10C7D000BBB910B50C4C216803F0FF024B883F2B0E
:10C7E00007DC07330B4401F1470003F8012F8342B4
:10C7F000FBD140230B800120FEF76CFE0023236059
:10C8000010BD704778A0FF1F7CA0FF1F38B5224CD9
:10C81000237803B138BD01232370FFF7A5FF70BB58
:10C8200000F048F840BB00F0DBF810BBFEF7F8FC66
:10C83000E0B900232370EFF30583002BEAD1EFF377
:10C84000108172B6154B1868E0B1154C2278CAB940
:10C8500045691D6001232370C5B1AA6101B962B6A3
:10C8600000254577836898472570D3E700F020F8C6
:10C87000DFE700F01BF8D9E700F016F8D3E7FFF781
:10C880001FFCCDE70029C5D162B638BD054B1D6040
:10C890000029E5D1E3E700BF85A0FF1F9C9EFF1F95
:10C8A000A09EFF1F989EFF1F704700BF704700BFEC
:10C8B000704700BF054A064B10781B78C0B2DBB248
:10C8C000984238BF4030C01A704700BF8CA0FF1F8D
:10C8D0008DA0FF1FF0B4384B1A7912F0300F2CD016
:10C8E00072B6997D01F0FF0200293DD062B6334F48
:10C8F000334938780D78334E1C46C0B2EDB2431C34
:10C90000402BE17928BF0023AB4202F1FF32C9B2CC
:10C910001CBFF154184612F0FF02F0D12A4B1B68DD
:10C92000C2B23A704BB1A84236BFC5F14005401BB8
:10C9300040192728C4BF01221A701F49CA78D2B2F1
:10C94000150616D452060DD51B4B1B795B0609D56F
:10C950001E4B1F491B6800220A7003B11A70164B48
:10C960003C22DA70F0BC70474022D9795A7462B622
:10C97000E3E70B791C06E5D5164B174E1C78337888
:10C98000E4B2DBB29C420ED0144D01E0A3420AD0C7
:10C990000133402B28BF00230879E85CC0B2C8717E
:10C9A000087D0728F2D9DBB2034933700B791806EA
:10C9B00044BF7C23CB70C5E700A006408CA0FF1FBE
:10C9C0008DA0FF1FD0A0FF1F88A0FF1F14A1FF1F75
:10C9D00010A1FF1F18A1FF1F11A1FF1F90A0FF1F93
:10C9E000054A064B10781B78C0B2DBB2984238BFBC
:10C9F0004030C01A704700BF8CA1FF1F21A1FF1F4C
:10CA0000F0B4384B1A7912F0300F2CD072B6997DF1
:10CA100001F0FF0200293DD062B6334F3349387828
:10CA20000D78334E1C46C0B2EDB2431C402BE17969
:10CA300028BF0023AB4202F1FF32C9B21CBFF15440
:10CA4000184612F0FF02F0D12A4B1B68C2B23A70AE
:10CA50004BB1A84236BFC5F14005401B40192728FD
:10CA6000C4BF01221A701F49CA78D2B2150616D463
:10CA700052060DD51B4B1B795B0609D51E4B1F4972
:10CA80001B6800220A7003B11A70164B3C22DA7040
:10CA9000F0BC70474022D9795A7462B6E3E70B794B
:10CAA0001C06E5D5164B174E1C783378E4B2DBB282
:10CAB0009C420ED0144D01E0A3420AD00133282B32
:10CAC00028BF00230879E85CC0B2C871087D072838
:10CAD000F2D9DBB2034933700B79180644BF7C23CB
:10CAE000CB70C5E700B006408CA1FF1F21A1FF1F3E
:10CAF0004CA1FF1F1CA1FF1F90A1FF1F20A1FF1F22
:10CB000094A1FF1F8DA1FF1F24A1FF1F70B584B04A
:10CB100072B6194B194D1A48702241260F248021F4
:10CB20001A702E701A460470197013781B06FCD503
:10CB3000144B186862B6144B144C984298BF00EB23
:10CB4000800001A998BF40000A22FDF7CFFE01A98D
:10CB50002046002311F8012B01333AB10A2B20F8AB
:10CB6000022FF7D11623237004B070BD5B00DBB237
:10CB7000237004B070BD00BF0000024007000240F7
:10CB800006000240080002407F969800C492FF1FF2
:10CB90002DE9F043DFF8EC808BB006460F4600F03D
:10CBA00073F898F90030013304460D4637D030460B
:10CBB000394600F0DFF9002831D02BA3D3E9002358
:10CBC0003046394600F026FE814668BB28A3D3E9EB
:10CBD00000233046394600F0FFFD00B398F90030DD
:10CBE000254ACDF82090042400200021022BCDE915
:10CBF0000467CDE9026700940192CDE906012CD0CB
:10CC0000684600F0BDF940B3089B1BB101F0AAF9DA
:10CC1000089B0360DDE906010BB0BDE8F083204608
:10CC200029460BB0BDE8F083134A98F90030019211
:10CC300003210022CDE90467CDE902670091089243
:10CC40002BB90E4B4FF06042CDE90623D8E70C49D3
:10CC50000020022BCDE90601D2D101F083F9222375
:10CC60000360D1E7AFF30080EF39FAFE422E864031
:10CC700051302DD5104987C05C0E0100FFFFEF47F2
:10CC80000000F07FDA92FF1F2DE9F04FB04F21F046
:10CC90000042BA4283B00C464FEAD17605460DD920
:10CCA000AC4FBA4225D9C1F31303034340F0EF80E0
:10CCB0000EB10020014603B0BDE8F08FA64B9A42AA
:10CCC00000F2CC80A54B9A4200F2DE808AA3D3E921
:10CCD000002300F05DF90022A14B00F09BFD00282D
:10CCE00000F005812846214600229D4B00F050F9B6
:10CCF000E1E783A3D3E9002300F08CFD002840F096
:10CD0000CB802846214680A3D3E9002300F064FDB0
:10CD10000028CED1934B284603EBC60821467CA3BE
:10CD2000D3E9002300F0E6FAD8E9002300F030F957
:10CD300000F07AFD804600F077FA77A3D3E900236C
:10CD400006460F4600F0D6FA02460B462846214614
:10CD500000F01CF972A3D3E90023CDE900013046AD
:10CD6000394600F0C7FA82468B4652465B46DDE9FB
:10CD7000000100F00BF905460C462A4623462846DA
:10CD8000214600F0B7FA68A3D3E9002306460F4610
:10CD900000F0B0FA66A3D3E9002300F0F7F83246BA
:10CDA0003B4600F0A7FA64A3D3E9002300F0F0F8B3
:10CDB00032463B4600F09EFA61A3D3E9002300F01F
:10CDC000E5F832463B4600F095FA5FA3D3E900232D
:10CDD00000F0DEF832463B4600F08CFA02460B4685
:10CDE0002846214600F0D2F806460F46284621463E
:10CDF00032463B46B8F1000F56D000F07BFA32467F
:10CE000004460D463B4600204FF0804100F0BEF83E
:10CE100002460B462046294600F096FB02460B468A
:10CE20005046594600F0B2F8DDE9002300F0AEF8B4
:10CE30000B4602464A49002000F0A8F86FF47F73C1
:10CE400098454FDA08F57A7801EB085100224FF047
:10CE5000B87300F04FFA03B0BDE8F08F424B9A422E
:10CE60003FF658AF414BF4002344D3E9002300F0D0
:10CE70008DF83F4BC6F101081C44CDE90001D4E90F
:10CE800000ABC6EB080870E74FF0000875E70246F4
:10CE90000B4600F07DF80EE717A3D3E900231046F8
:10CEA000194600F027FA06E700F024FA002280462F
:10CEB00089464FF080433046394600F067F8024615
:10CEC0000B464046494600F03FFB2A46234600F009
:10CED0005DF802460B460020214900F057F803B0E8
:10CEE000BDE8F08F01EB085103B0BDE8F08F80463C
:10CEF00043E700BFAFF300809C7500883CE4377EB9
:10CF0000EF39FAFE422E864051302DD5104987C0A8
:10CF1000FE822B654715F73F0000E0FE422EE63FFC
:10CF2000763C7935EF39EA3DD0A4BE726937663E6A
:10CF3000F16BD2C541BDBB3E2CDE25AF6A56113F19
:10CF400093BDBE166CC1663F3E5555555555C53F00
:10CF5000412E8640FFFFEF7F422ED63FFFFF2F3E40
:10CF60000000F03F600E0100B1A2F03F800E010012
:10CF7000700E010041F0004101F58010C00F7047B4
:10CF80000020704781F0004102E000BF83F00043C1
:10CF900030B54FEA41044FEA430594EA050F08BF54
:10CFA00090EA020F1FBF54EA000C55EA020C7FEA18
:10CFB000645C7FEA655C00F0E2804FEA5454D4EB95
:10CFC0005555B8BF6D420CDD2C4480EA020281EA5F
:10CFD000030382EA000083EA010180EA020281EA97
:10CFE0000303362D88BF30BD11F0004F4FEA0131E9
:10CFF0004FF4801C4CEA113102D0404261EB4101F8
:10D0000013F0004F4FEA03334CEA133302D052427D
:10D0100063EB430394EA050F00F0A780A4F1010439
:10D02000D5F1200E0DDB02FA0EFC22FA05F2801873
:10D0300041F1000103FA0EF2801843FA05F3594159
:10D040000EE0A5F120050EF1200E012A03FA0EFCD8
:10D0500028BF4CF0020C43FA05F3C01851EBE37102
:10D0600001F0004507D54FF0000EDCF1000C7EEB1F
:10D0700000006EEB0101B1F5801F1BD3B1F5001F5D
:10D080000CD349085FEA30004FEA3C0C04F101047C
:10D090004FEA445212F5800F80F09A80BCF1004FA5
:10D0A00008BF5FEA500C50F1000041EB045141EA27
:10D0B000050130BD5FEA4C0C404141EB010111F428
:10D0C000801FA4F10104E9D191F0000F04BF0146D3
:10D0D0000020B1FA81F308BF2033A3F10B03B3F1B1
:10D0E00020020CDA0C3208DD02F1140CC2F10C0241
:10D0F00001FA0CF021FA02F10CE002F11402D8BF9F
:10D10000C2F1200C01FA02F120FA0CFCDCBF41EA6A
:10D110000C019040E41AA2BF01EB0451294330BD39
:10D120006FEA04041F3C1CDA0C340EDC04F1140416
:10D13000C4F1200220FA04F001FA02F340EA0300ED
:10D1400021FA04F345EA030130BDC4F10C04C4F133
:10D15000200220FA02F001FA04F340EA0300294613
:10D1600030BD21FA04F0294630BD94F0000F83F45D
:10D17000801306BF81F480110134013D4EE77FEA40
:10D18000645C18BF7FEA655C29D094EA050F08BF8C
:10D1900090EA020F05D054EA000C04BF194610466D
:10D1A00030BD91EA030F1EBF0021002030BD5FEAB1
:10D1B000545C05D14000494128BF41F0004130BDD9
:10D1C00014F580043CBF01F5801130BD01F000452D
:10D1D00045F0FE4141F470014FF0000030BD7FEAA0
:10D1E000645C1ABF194610467FEA655C1CBF0B469B
:10D1F000024650EA013406BF52EA033591EA030FB2
:10D2000041F4002130BD00BF90F0000F04BF0021A9
:10D21000704730B54FF4806404F132044FF00005DC
:10D220004FF0000150E700BF90F0000F04BF002155
:10D23000704730B54FF4806404F1320410F00045BB
:10D2400048BF40424FF000013EE700BF42004FEAB6
:10D25000E2014FEA31014FEA02701FBF12F07F4333
:10D2600093F07F4F81F06051704792F0000F14BF30
:10D2700093F07F4F704730B54FF4607401F0004574
:10D2800021F0004120E700BF50EA010208BF7047CB
:10D2900030B54FF000050AE050EA010208BF7047C0
:10D2A00030B511F0004502D5404261EB41014FF429
:10D2B000806404F132045FEA915C3FF4DCAE4FF02D
:10D2C00003025FEADC0C18BF03325FEADC0C18BF14
:10D2D000033202EBDC02C2F1200300FA03FC20FA65
:10D2E00002F001FA03FE40EA0E0021FA02F11444B2
:10D2F000C1E600BF70B54FF0FF0C4CF4E06C1CEAC7
:10D3000011541DBF1CEA135594EA0C0F95EA0C0F3B
:10D3100000F0DEF82C4481EA030621EA4C5123EAAE
:10D320004C5350EA013518BF52EA033541F48011DD
:10D3300043F4801338D0A0FB02CE4FF00005E1FB90
:10D3400002E506F00042E0FB03E54FF00006E1FBDA
:10D3500003569CF0000F18BF4EF0010EA4F1FF041D
:10D36000B6F5007F64F5407404D25FEA4E0E6D415D
:10D3700046EB060642EAC62141EA55514FEAC5206E
:10D3800040EA5E504FEACE2EB4F1FD0C88BFBCF5EA
:10D39000E06F1ED8BEF1004F08BF5FEA500E50F19B
:10D3A000000041EB045170BD06F0004646EA010161
:10D3B00040EA020081EA0301B4EB5C04C2BFD4EB93
:10D3C0000C0541EA045170BD41F480114FF0000E8C
:10D3D000013C00F3AB8014F1360FDEBF002001F0FA
:10D3E000004170BDC4F10004203C35DA0C341BDC74
:10D3F00004F11404C4F1200500FA05F320FA04F046
:10D4000001FA05F240EA020001F0004221F0004179
:10D4100010EBD37021FA04F642EB06015EEA430EEC
:10D4200008BF20EAD37070BDC4F10C04C4F120051C
:10D4300000FA04F320FA05F001FA04F240EA0200CF
:10D4400001F0004110EBD37041F100015EEA430EA0
:10D4500008BF20EAD37070BDC4F1200500FA05F2C0
:10D460004EEA020E20FA04F301FA05F243EA02033F
:10D4700021FA04F001F0004121FA04F220EA02004E
:10D4800000EBD3705EEA430E08BF20EAD37070BD94
:10D4900094F0000F0FD101F00046400041EB010174
:10D4A00011F4801F08BF013CF7D041EA060195F056
:10D4B000000F18BF704703F00046520043EB030310
:10D4C00013F4801F08BF013DF7D043EA06037047FD
:10D4D00094EA0C0F0CEA135518BF95EA0C0F0CD008
:10D4E00050EA410618BF52EA4306D1D181EA03014E
:10D4F00001F000414FF0000070BD50EA410606BF48
:10D500001046194652EA430619D094EA0C0F02D18C
:10D5100050EA013613D195EA0C0F05D152EA0336D1
:10D520001CBF104619460AD181EA030101F00041EF
:10D5300041F0FE4141F470014FF0000070BD41F038
:10D54000FE4141F4780170BD70B54FF0FF0C4CF412
:10D55000E06C1CEA11541DBF1CEA135594EA0C0F31
:10D5600095EA0C0F00F0A7F8A4EB050481EA030E7E
:10D5700052EA03354FEA013100F088804FEA033365
:10D580004FF0805545EA131343EA12634FEA022233
:10D5900045EA111545EA10654FEA00260EF00041F4
:10D5A0009D4208BF964244F1FD0404F5407402D246
:10D5B0005B084FEA3202B61A65EB03055B084FEAD7
:10D5C00032024FF480104FF4002CB6EB020E75EBD4
:10D5D000030E22BFB61A754640EA0C005B084FEAFC
:10D5E0003202B6EB020E75EB030E22BFB61A754679
:10D5F00040EA5C005B084FEA3202B6EB020E75EBC4
:10D60000030E22BFB61A754640EA9C005B084FEA3B
:10D610003202B6EB020E75EB030E22BFB61A754648
:10D6200040EADC0055EA060E18D04FEA051545EA37
:10D6300016754FEA06164FEAC30343EA52734FEAE0
:10D64000C2025FEA1C1CC0D111F4801F0BD141EA59
:10D6500000014FF000004FF0004CB6E711F4801FBE
:10D6600004BF01430020B4F1FD0C88BFBCF5E06F9E
:10D670003FF6AFAEB5EB030C04BFB6EB020C5FEAAE
:10D68000500C50F1000041EB045170BD0EF0004E03
:10D690004EEA113114EB5C04C2BFD4EB0C0541EA35
:10D6A000045170BD41F480114FF0000E013C90E632
:10D6B00045EA060E8DE60CEA135594EA0C0F08BFF6
:10D6C00095EA0C0F3FF43BAF94EA0C0F0AD150EAF5
:10D6D00001347FF434AF95EA0C0F7FF425AF104688
:10D6E00019462CE795EA0C0F06D152EA03353FF4B0
:10D6F000FDAE1046194622E750EA410618BF52EA2D
:10D7000043067FF4C5AE50EA41047FF40DAF52EA00
:10D7100043057FF4EBAE12E74FF0FF3C06E000BF9D
:10D720004FF0010C02E000BF4FF0010C4DF804CDAA
:10D730004FEA410C7FEA6C5C4FEA430C18BF7FEA6A
:10D740006C5C1BD001B050EA410C0CBF52EA430C98
:10D7500091EA030F02BF90EA020F0020704710F118
:10D76000000F91EA030F58BF994208BF90422CBFA7
:10D77000D8176FEAE37040F0010070474FEA410CA0
:10D780007FEA6C5C02D150EA013C07D14FEA430CBE
:10D790007FEA6C5CD6D152EA033CD3D05DF8040B2F
:10D7A000704700BF8446104662468C461946634661
:10D7B00000E000BF01B5FFF7B7FF002848BF10F138
:10D7C000000F01BD4DF808EDFFF7F4FF0CBF01207D
:10D7D00000205DF808FB00BF4DF808EDFFF7EAFFF9
:10D7E00034BF012000205DF808FB00BF4DF808EDB4
:10D7F000FFF7E0FF94BF012000205DF808FB00BFA9
:10D800004DF808EDFFF7CEFF94BF012000205DF832
:10D8100008FB00BF4DF808EDFFF7C4FF34BF01203F
:10D8200000205DF808FB00BF4FEA410212F500122C
:10D8300015D211D56FF47873B3EB625212D94FEA57
:10D84000C12343F0004343EA505311F0004F23FA41
:10D8500002F018BF404270474FF00000704750EA96
:10D86000013005D111F0004008BF6FF00040704753
:10D870004FF00000704700BF4FEA4102B2F1E043B1
:10D8800024BFB3F5001CDCF1FE5C0DD901F0004CA7
:10D890004FEAC0024CEA5070B2F1004F40EB8300F7
:10D8A00008BF20F00100704711F0804F21D113F123
:10D8B0003872BCBF01F00040704741F480114FEA5C
:10D8C0005252C2F11802C2F1200C10FA0CF320FAE5
:10D8D00002F018BF40F001004FEAC1234FEAD32302
:10D8E00003FA0CFC40EA0C0023FA02F34FEA43036C
:10D8F000CCE77FEA625307D150EA01331EBF4FF0F5
:10D90000FE4040F44000704701F0004040F0FE400F
:10D9100040F40000704700BF80F0004002E000BF0C
:10D9200081F0004142001FBF5FEA410392EA030F0A
:10D930007FEA226C7FEA236C6AD04FEA1262D2EB54
:10D940001363C1BFD218414048404140B8BF5B4259
:10D95000192B88BF704710F0004F40F4000020F0F2
:10D960007F4018BF404211F0004F41F4000121F008
:10D970007F4118BF494292EA030F3FD0A2F1010252
:10D9800041FA03FC10EB0C00C3F1200301FA03F190
:10D9900000F0004302D5494260EB4000B0F5000FB3
:10D9A00013D3B0F1807F06D340084FEA310102F172
:10D9B0000102FE2A51D2B1F1004F40EBC25008BF24
:10D9C00020F0010040EA03007047490040EB0000EE
:10D9D00010F4000FA2F10102EDD1B0FA80FCACF11D
:10D9E000080CB2EB0C0200FA0CF0AABF00EBC2501C
:10D9F00052421843BCBFD0401843704792F0000F0A
:10DA000081F4000106BF80F400000132013BB5E75C
:10DA10004FEA41037FEA226C18BF7FEA236C21D0D2
:10DA200092EA030F04D092F0000F08BF0846704737
:10DA300090EA010F1CBF0020704712F07F4F04D105
:10DA4000400028BF40F00040704712F100723CBF18
:10DA500000F50000704700F0004343F0FE4040F442
:10DA6000000070477FEA226216BF08467FEA236300
:10DA70000146420206BF5FEA412390EA010F40F4EB
:10DA8000800070474FF0000304E000BF10F0004337
:10DA900048BF40425FEA000C08BF704743F096431E
:10DAA00001464FF000001CE050EA010208BF704739
:10DAB0004FF000030AE000BF50EA010208BF7047C0
:10DAC00011F0004302D5404261EB41015FEA010CD5
:10DAD00002BF84460146002043F0B64308BFA3F1CD
:10DAE0008053A3F50003BCFA8CF2083AA3EBC253AF
:10DAF00010DB01FA02FC634400FA02FCC2F12002CE
:10DB0000BCF1004F20FA02F243EB020008BF20F004
:10DB10000100704702F1200201FA02FCC2F120026A
:10DB200050EA4C0021FA02F243EB020008BF20EA5F
:10DB3000DC7070474FF0FF0C1CEAD0521EBF1CEA8D
:10DB4000D15392EA0C0F93EA0C0F6FD01A4480EA7B
:10DB5000010C400218BF5FEA41211ED04FF0006364
:10DB600043EA501043EA5111A0FB01310CF0004090
:10DB7000B1F5000F3EBF490041EAD3715B0040EAB6
:10DB8000010062F17F02FD2A1DD8B3F1004F40EB86
:10DB9000C25008BF20F00100704790F0000F0CF059
:10DBA000004C08BF49024CEA502040EA51207F3A1D
:10DBB000C2BFD2F1FF0340EAC250704740F40000F8
:10DBC0004FF00003013A5DDC12F1190FDCBF00F0E9
:10DBD00000407047C2F10002410021FA02F1C2F197
:10DBE000200200FA02FC5FEA310040F1000053EA33
:10DBF0004C0308BF20EADC70704792F0000F00F081
:10DC0000004C02BF400010F4000F013AF9D040EA86
:10DC10000C0093F0000F01F0004C02BF490011F41A
:10DC2000000F013BF9D041EA0C018FE70CEAD15318
:10DC300092EA0C0F18BF93EA0C0F0AD030F0004C98
:10DC400018BF31F0004CD8D180EA010000F000404C
:10DC5000704790F0000F17BF90F0004F084691F00A
:10DC6000000F91F0004F14D092EA0C0F01D1420244
:10DC70000FD193EA0C0F03D14B0218BF084608D10D
:10DC800080EA010000F0004040F0FE4040F4000057
:10DC9000704740F0FE4040F4400070474FF0FF0CEA
:10DCA0001CEAD0521EBF1CEAD15392EA0C0F93EA31
:10DCB0000C0F69D0A2EB030280EA010C49024FEA83
:10DCC000402037D04FF0805343EA111143EA10133C
:10DCD0000CF000408B4238BF5B0042F17D024FF4F4
:10DCE000000C8B4224BF5B1A40EA0C00B3EB510FCF
:10DCF00024BFA3EB510340EA5C00B3EB910F24BFB8
:10DD0000A3EB910340EA9C00B3EBD10F24BFA3EB3C
:10DD1000D10340EADC001B0118BF5FEA1C1CE0D104
:10DD2000FD2A3FF650AF8B4240EBC25008BF20F0B7
:10DD3000010070470CF0004C4CEA50207F32C2BF0B
:10DD4000D2F1FF0340EAC250704740F400004FF0A8
:10DD50000003013A37E792F0000F00F0004C02BFD9
:10DD6000400010F4000F013AF9D040EA0C0093F0A3
:10DD7000000F01F0004C02BF490011F4000F013BFD
:10DD8000F9D041EA0C0195E70CEAD15392EA0C0F65
:10DD900008D142027FF47DAF93EA0C0F7FF470AF9D
:10DDA000084676E793EA0C0F04D14B023FF44CAFE0
:10DDB00008466EE730F0004C18BF31F0004CCAD175
:10DDC00030F000427FF45CAF31F000437FF43CAFB1
:10DDD0005FE700BF4FF0FF3C06E000BF4FF0010CD3
:10DDE00002E000BF4FF0010C4DF804CD4FEA4002B5
:10DDF0004FEA41037FEA226C18BF7FEA236C11D0FF
:10DE000001B052EA530C18BF90EA010F58BFB2EBB1
:10DE1000030088BFC81738BF6FEAE17018BF40F031
:10DE2000010070477FEA226C02D15FEA402C05D1E5
:10DE30007FEA236CE4D15FEA412CE1D05DF8040B6A
:10DE4000704700BF844608466146FFE70FB5FFF7FD
:10DE5000C9FF002848BF10F1000F0FBD4DF808EDB5
:10DE6000FFF7F4FF0CBF012000205DF808FB00BFA6
:10DE70004DF808EDFFF7EAFF34BF012000205DF800
:10DE800008FB00BF4DF808EDFFF7E0FF94BF01204D
:10DE900000205DF808FB00BF4DF808EDFFF7D2FF4A
:10DEA00094BF012000205DF808FB00BF4DF808ED8D
:10DEB000FFF7C8FF34BF012000205DF808FB00BF5A
:10DEC0004FEA4002B2F1FE4F0FD34FF09E03B3EB87
:10DED00012620DD94FEA002343F0004310F0004FC7
:10DEE00023FA02F018BF404270474FF0000070471D
:10DEF00012F1610F01D1420205D110F0004008BFBC
:10DF00006FF0004070474FF00000704742000ED2A3
:10DF1000B2F1FE4F0BD34FF09E03B3EB126209D464
:10DF20004FEA002343F0004323FA02F070474FF01A
:10DF30000000704712F1610F01D1420202D14FF08F
:10DF4000FF3070474FF00000704700BF0B4601469E
:10DF5000184600F001B800BF13460A4601460220E9
:10DF600000F0C0BE014B1868704700BF0897FF1F44
:10DF700070B50F4E0F4D761BB61018BF002405D09C
:10DF8000013455F8043B9847A642F9D10A4E0B4D8F
:10DF9000761B02F07FFFB61018BF002406D00134B4
:10DFA00055F8043B9847A642F9D170BD70BD00BF3B
:10DFB000A00E0100A00E0100B40E0100A00E010091
:10DFC000024B0146186800F00BB800BF0897FF1F0E
:10DFD000024B0146186800F049BF00BF0897FF1FB9
:10DFE0002DE9F04F01F10B05162D83B0064640F2E6
:10DFF0009F8035F0070500F1BF80A94200F2BC8088
:10E0000000F058FBB5F5FC7FC0F09C826B0A00F075
:10E01000BA80042B00F28381A80900F1390E4FEA7F
:10E020004E033830C44F07EB8303A3F108015C684B
:10E03000A14207D1ACE0002A80F2AC80E468A142A2
:10E0400000F0A680636823F003035A1B0F2AF2DD59
:10E05000B9493C6901F1080E744500F0B381636869
:10E0600023F003035A1B0F2A00F39981002AC1F8F9
:10E0700014E0C1F810E080F29E80B3F5007F80F0DC
:10E080006781DB0803F1010C01229B1002FA03F304
:10E090004A6851F83C80C4F8088001EBCC091A4367
:10E0A000A9F10803E3604A6041F83C40C8F80C401D
:10E0B000831001249C40944200F28A80144206D1CD
:10E0C00020F003006400144200F10400FAD007EBD2
:10E0D000C009CC468046DCF80C108C4507D173E1B2
:10E0E000002A80F28181C9688C4500F06D814B68FF
:10E0F00023F003035A1B0F2AF2DD0C46D1F80CC0A3
:10E1000054F8088F4B1945F001054D6042F00101AC
:10E11000C8F80CC03046CCF808807B613B61C3F87E
:10E120000CE0C3F808E059609A5000F0C5FA1FE00F
:10E13000102921D800F0BEFA1025062302207E4FB8
:10E1400007EB8303A3F108025C68944200F0458169
:10E150006368E168A56823F00303234430465A68E6
:10E16000E96042F001028D605A6000F0A5FA0834BF
:10E17000204603B0BDE8F08F00240C232046336016
:10E1800003B0BDE8F08F80234FF0400E3F2049E7F9
:10E1900070465DE72344E1685A68A56842F00102D1
:10E1A000E96030468D605A6000F086FA08342046F7
:10E1B00003B0BDE8F08F234430465A6842F00102B4
:10E1C0005A6000F079FA0834204603B0BDE8F08FB9
:10E1D000BC68636823F00308A84504D3C5EB0803B3
:10E1E0000F2B00F38C80554BDFF860911A68D9F83B
:10E1F000003001332A4404EB080A00F0608102F584
:10E2000080520F3222F47F6222F00F021146304614
:10E21000019200F04BFCB0F1FF3F8346019A00F001
:10E220005881824500F2FC80454B1968DA4511445B
:10E23000196000F05381D9F80000DFF810E10130D7
:10E240001BBFCAEB0B0A5144CEF800B019601BF09B
:10E25000070100F01781C1F10800C1F58051834426
:10E2600008315A44C2F30B02C2EB01094946304659
:10E27000019300F01BFC431C019B00F03F81CBEBA2
:10E2800000024A4442F001021968C7F808B0494444
:10E29000BC42CBF804201960DFF8A49016D0B8F186
:10E2A0000F0F40F2FD806268A8F10C0323F0070312
:10E2B000E01802F001024FF0050E1A430F2B6260C6
:10E2C000C0F804E0C0F808E000F21C811D4BBC68F7
:10E2D0001A68914288BF19601B4B1A6891426268A4
:10E2E00088BF196022F003029542A2EB050301D812
:10E2F0000F2B04DC304600F0DFF9002438E7621908
:10E3000043F0010345F0010565603046BA60536093
:10E3100000F0D2F90834204603B0BDE8F08F142B8A
:10E3200071D9542B00F2A480280B00F16F0E4FEA34
:10E330004E036E3076E600BF0C97FF1FA0A1FF1FB3
:10E34000A4A1FF1F9CA1FF1F98A1FF1F189BFF1FE7
:10E350005A0A042A5ED9142A00F2B38002F15C0141
:10E3600049005B3207EB810C57F82110DFF8DC81A4
:10E37000ACF1080C8C4500F088804A6822F003025A
:10E38000934202D289688C45F7D1D1F80CC07A68E3
:10E39000C4F80CC0A160CCF80840CC6088E66319D2
:10E3A00042F0010745F00105656030464B610B61A5
:10E3B000C3F80CE0C3F808E05F609A50083400F03E
:10E3C0007BF9D5E64A6873E608F1010818F0030FF7
:10E3D0000CF1080C7FF47FAE30E0DC68A34208BF8C
:10E3E00002303FF435AEB3E60B440C465A68C968B8
:10E3F00054F8085F42F001025A603046E9608D60CF
:10E4000000F05AF9B4E603F15C0E03F15B004FEA49
:10E410004E0307E69A0902F1390149003832A1E7B3
:10E42000BC424A4B3FF400AF9C68626822F0030292
:10E430005AE759F80839994540F0828010F0030FE7
:10E4400000F1FF30F5D17B6823EA04037B606400B0
:10E450009C423FF6BDAE002C3FF4BAAE1C42404693
:10E460007FF435AE64001C4200F10400FAD02EE6C1
:10E47000B3F5AA7F18D8E80B00F1780E4FEA4E03E7
:10E480007730CFE54FF48051EBE60121D8F8043026
:10E49000921001FA02F21A43C8F80420614677E7A5
:10E4A0000123CBF8043025E740F25452934220D8A0
:10E4B000A80C00F17D0E4FEA4E037C30B2E510321D
:10E4C000A4E6542A26D81A0B02F16F0149006E32D5
:10E4D00048E7BC68626822F0030205E7CAF30B0054
:10E4E00000287FF4A8AE4244BB6842F001025A60A3
:10E4F000ECE6FE234FF07F0E7E2093E501224FF0E5
:10E500000009C1E604F10801304600F0AFFCD9F87B
:10E510000010DBE6B2F5AA7F05D8DA0B02F178012C
:10E52000490077321EE740F254518A4205D89A0CCE
:10E5300002F17D0149007C3214E7FE217E2211E7C1
:10E540007B6884E7E808431C5B00F8E50C97FF1F35
:10E550008842F0B50DD98B1898420AD28118002A4A
:10E5600051D09A1A13F8014D01F8014D9342F9D197
:10E57000F0BD0F2A48D941EA00039B0746D100F1BC
:10E58000100401F11003154653F8106C44F8106C98
:10E5900053F80C6C44F80C6C53F8086C44F8086C95
:10E5A000103D53F8046C44F8046C0F2D03F1100374
:10E5B00004F11004E8D8A2F1100323F00F0302F0D5
:10E5C0000F0E1033BEF1030F1944034421D91E1F4F
:10E5D0000D467446043C55F8047B46F8047F032C32
:10E5E000F8D8AEF1040424F0030404342344214495
:10E5F00002F0030262B1013B0A4411F8014B03F837
:10E60000014F8A42F9D1F0BD0346F3E70346F2E732
:10E61000F0BD7246EEE700BF70B4840746D0541ECA
:10E62000002A41D0CDB2034602E0621EE4B3144694
:10E6300003F8015B9A07F8D1032C2ED9CDB245EA35
:10E6400005250F2C45EA054519D903F11002264688
:10E65000103E0F2E42F8105C42F80C5C42F8085C49
:10E6600042F8045C02F11002F2D8A4F1100222F088
:10E670000F0204F00F041032032C13440DD91E4670
:10E680002246043A032A46F8045BFAD8221F22F0F5
:10E6900003020432134404F003042CB1C9B21C4435
:10E6A00003F8011BA342FBD170BC7047144603461C
:10E6B000C2E700BF704700BF704700BF024B0A4669
:10E6C0000146186800F002B80897FF1F2DE9F04FC7
:10E6D000174683B0002900F0C1800E46814607F13D
:10E6E0000B05FFF7E7FF56F804EC162D2EF0030498
:10E6F000A6F1080840D810221546AF4241D89442EE
:10E7000075DAC94B996808EB04008842416800F04B
:10E71000D98021F0010303445B68DB077DD51EF03F
:10E72000010F35D039464846FFF75AFC0746E0B19D
:10E7300056F8043C23F001034344A0F108029A4236
:10E7400000F04481221F242A00F23181132A00F2B2
:10E750000481034632461168196051685960926815
:10E760009A603146484600F081FB4846FFF7A4FF17
:10E77000384603B0BDE8F08F25F00705002D2A4686
:10E78000BBDA0C230020C9F8003003B0BDE8F08FDD
:10E7900056F8083CC3EB080ADAF8043023F0030CFF
:10E7A00004EB0C039342BDDB5746DAF80C1057F824
:10E7B000080F221F242AC160886000F21781132AE3
:10E7C00040F212813168CAF808107168CAF80C105A
:10E7D0001B2A00F22B8108360AF110023168116001
:10E7E00071685160B16891603E461C46D046631B1B
:10E7F0000F2B1DD8D8F8043003F001032343444401
:10E80000C8F80430636843F0010363604846FFF7CB
:10E8100053FF304603B0BDE8F08F21F003012144DF
:10E82000914221DBC36882680C46D3609A60DEE7C0
:10E83000D8F8042008EB050102F00102154343F06B
:10E8400001020B44C8F804504A605A6842F00102C1
:10E8500008315A60484600F009FBD7E7114603B07B
:10E86000BDE8F04FFFF7BCBB1EF0010F7FF45AAFBD
:10E8700056F8083CC3EB080ADAF8043023F0030C1E
:10E8800001EB0C0E96458BDBC36882685746D3605C
:10E890009A6057F8081FDAF80C30CB60221F242A40
:10E8A000996000F29980132A62D93368CAF8083057
:10E8B0007368CAF80C301B2A00F2A08008360AF1EF
:10E8C000100356E021F0030BA34405F1100083452B
:10E8D00059DA1EF0010F7FF425AF56F8081CC1EB82
:10E8E000080ADAF8041021F0030CE34458453FF716
:10E8F00057AF5746DAF80C1057F8080F221F242A92
:10E90000C160886000F2B480132A40F2A5803168AB
:10E91000CAF808107168CAF80C101B2A00F2AF8000
:10E9200008360AF110023168116071685160B168EF
:10E9300091600AEB0501C5EB0B0242F00102996000
:10E940004A60DAF8043003F001031D434846CAF870
:10E950000450FFF7B1FE38465CE733680360736824
:10E9600043601B2A27D800F1080306F10802F2E6EB
:10E970003B4632681A6072685A60B2689A603E46D6
:10E980007446D04633E708EB0501C5EB0B0B4BF0A3
:10E99000010299604A6056F8043C03F001031D43EC
:10E9A000484646F8045CFFF787FE304632E73146BA
:10E9B000FFF7CEFDD5E6B3688360F368C360242A11
:10E9C00028D000F1100306F11002C4E650F8043C10
:10E9D00023F003031C440AE7314638467446D04608
:10E9E000FFF7B6FD3E4602E73A46F7E631463846BF
:10E9F0001C46D046FFF7ACFD3E46F8E6B368CAF8C1
:10EA00001030F368CAF81430242A1BD010360AF1EB
:10EA10001803AEE7336903617369436106F11802B5
:10EA200000F1180397E600BF0C97FF1FB168CAF802
:10EA30001010F168CAF81410242A0FD010360AF109
:10EA40001802CBE63369CAF818307369CAF81C306B
:10EA500018360AF120038CE73A4664E73269CAF8AF
:10EA600018207269CAF81C2018360AF12002B5E68F
:10EA7000314638460193FFF76BFD019B59E7B168BA
:10EA8000CAF81010F168CAF81410242A03D01036FE
:10EA90000AF1180247E73269CAF818207269CAF801
:10EAA0001C2018360AF120023DE700BF38B5074C9C
:10EAB0000023054608462360FBF7E2FE431C00D016
:10EAC00038BD2368002BFBD02B6038BD00A3FF1F8F
:10EAD000FFFFFFFFFFFFFFFFFFFFFFFFFFFFFFFF46
:10EAE000FFFFFFFFFFFFFFFFFFFFFFFFFFFFFFFF36
:10EAF000FFFFFFFFFFFFFFFFFFFFFFFFFFFFFFFF26
:10EB000090F800F06DE9024520F007016FF0000C6D
:10EB100010F0070491F820F040F049804FF0000415
:10EB20006FF00700D1E9002391F840F000F10800F0
:10EB300082FA4CF2A4FA8CF283FA4CF3A2FA8CF328
:10EB40004BBBD1E9022382FA4CF200F10800A4FA8F
:10EB50008CF283FA4CF3A2FA8CF3E3B9D1E90423E3
:10EB600082FA4CF200F10800A4FA8CF283FA4CF31A
:10EB7000A2FA8CF37BB9D1E9062301F1200182FAD4
:10EB80004CF200F10800A4FA8CF283FA4CF3A2FADA
:10EB90008CF3002BC6D0002A04BF04301A4612BAE8
:10EBA000B2FA82F2FDE8024500EBD2007047D1E9EB
:10EBB000002304F00305C4F100004FEAC50514F07A
:10EBC000040F91F840F00CFA05F562EA05021CBF4B
:10EBD00063EA050362464FF00004A9E7002A41D02A
:10EBE00040EA010313F00303F0B425D1032A23D92B
:10EBF00004680D68AC421FD1043A35D0A4F1013548
:10EC000025EA040414F0803F31D1071D0D1D0DE0ED
:10EC100057F8043B0E68A3F10134B34224EA03041D
:10EC20000AD1043A20D014F0803F23D1032A294688
:10EC3000384605F10405EBD803780C789C4202F1C4
:10EC4000FF320CD182B114B916E06AB17BB110F871
:10EC5000013F11F8014FA34202F1FF32F5D0181B1A
:10EC6000F0BC7047104670471046F0BC704718461D
:10EC7000F0BC70470020F3E72046F1E740EA0103CB
:10EC80009B0770B42BD1032A29D90C460346214691
:10EC900054F8046BA6F1013525EA060515F0803F0E
:10ECA00006D1043A032A43F8046B2146EFD8A2B1F7
:10ECB0000C781C70013A013301313CB16AB111F892
:10ECC000014B03F8014B013A002CF7D12AB11A4449
:10ECD000002103F8011B9A42FBD170BC7047034628
:10ECE000E5E700BF2DE9F047254C2568D5F84841F8
:10ECF0000646884692469946C4B360681F2817DCCA
:10ED0000431C76B104EB80050122C5F888A0D4F835
:10ED1000881182401143022EC4F88811C5F8089169
:10ED20001ED00230636044F820800020BDE8F087E8
:10ED3000144B03B34FF4C870FFF742F90446D0B147
:10ED4000D5F84831002780E88800C5F848413846A2
:10ED50000123C4F88871C4F88C71002EE1D0D1E78A
:10ED6000D4F88C110A43C4F88C21DAE705F5A674AF
:10ED7000C5F84841C1E74FF0FF30BDE8F08700BF5C
:10ED8000900E0100C1DF0000024B13B1024800F0F9
:10ED900005B8704700000000A9ED000000230146FF
:10EDA0001A461846FFF79EBF38B5074D074C2C1B77
:10EDB000A41005D0013C55F8043D9847002CF9D12A
:10EDC000BDE8384002F076B8000000000000000006
:10EDD000F8B5234F0C460646FFF76CFCBB685D6830
:10EDE00025F00305291B01F6EF7121F47F6121F065
:10EDF0000F01A1F58054B4F5805F07DB0021304698
:10EE0000FFF754FEBB682B44984204D03046FFF70E
:10EE100053FC0020F8BD61423046FFF747FE013049
:10EE20000DD0104BBA6819682D1B45F0010530460E
:10EE3000091B55601960FFF73FFC0120F8BD002158
:10EE40003046FFF733FEBA68831A0F2BDEDD064C1F
:10EE50000449246843F00103001B53600860D5E7B0
:10EE60000C97FF1FA4A1FF1F189BFF1F002945D06F
:10EE70002DE9F0410D468046FFF71CFC55F8047C57
:10EE80006A4927F00103A5F10804E2188E6850686A
:10EE9000B24220F0030062D0FE0750600BD455F858
:10EEA000087CE41B01F1080EA56875453B446FD052
:10EEB000E768EF60BD6015186D68ED0742D543F057
:10EEC00001026260E350B3F5007F18D2DB085A1CE0
:10EED0004D6851F83270A76001209B1000FA03F3CF
:10EEE00001EBC2001D430838E0604D6041F832403C
:10EEF000FC604046BDE8F041FFF7DEBB70475A0AB0
:10EF0000042A53D89A0902F139077F0002F1380523
:10EF100001EB870051F827204449083890424DD032
:10EF2000516821F003018B4202D292689042F7D1DE
:10EF3000D068E060A2608460D4604046BDE8F041E3
:10EF4000FFF7BABB95683A4FBD4203443FD0D06843
:10EF5000E86043F0010285606260E350B3E7FF07B9
:10EF6000034407D455F8082CA41A1344A068E26897
:10EF7000C26090602F4A126843F0010093426060C3
:10EF80008C60B6D32C4B40461968FFF721FFB0E7E1
:10EF900011184968C90744D49168D268CA6003440B
:10EFA00043F0010091606060E350A2E7142A17D893
:10EFB00002F15C077F0002F15B05A9E7AA104B682C
:10EFC000012505FA02F213434B600246B1E743F014
:10EFD00001024C610C61E560A5606260E35088E766
:10EFE000542A06D81A0B02F16F077F0002F16E0552
:10EFF0008EE7B2F5AA7F06D8DA0B02F178077F0018
:10F0000002F1770584E740F25450824206D89A0C08
:10F0100002F17D077F0002F17C0579E7FE277E255E
:10F0200076E743F001026260E35062E70C97FF1F4E
:10F030001497FF1F149BFF1FA0A1FF1FF2FFFFFFEC
:10F04000F3FFFFFFF4FFFFFFF4FFFFFFF5FFFFFFFC
:10F05000F6FFFFFFF7FFFFFFF8FFFFFFF9FFFFFFDE
:10F06000FAFFFFFFFBFFFFFFFCFFFFFFFDFFFFFFBE
:10F07000FDFFFFFFFEFFFFFFFFFFFFFF000000009F
:10F08000000078053408540B800C3C0F5C12E0152E
:10F09000FA19141E6022AC265C2B0C30BC34023AE8
:10F0A000FF3FFFFF10F40000ECF30000C8F3000086
:10F0B000A4F300008CF10000D8F00000FCF0000088
:10F0C00020F1000044F1000090F20000B4F20000D2
:10F0D00080F000006CF2000000005802460566084F
:10F0E000540BD80E5C12E015FA19141E6022AC26DF
:10F0F0005C2B0C30BC34023AFF3FFFFF0000900154
:10F1000020031405D0075A0AAC0DCC10B4146A18A9
:10F11000E81C342180252A2B70301437FF3FFFFF75
:10F120000000C800F4018403140508072E091C0C14
:10F13000D80EF811AE159619401F1C25F22B583425
:10F14000FF3FFFFF00006400C8009001BC021A04EA
:10F15000DC059E07F609800CA00F2413A2174C1D96
:10F160005424442FFF3FFFFF40067805B004E80316
:10F1700084032003BC025802F40190012C01FA0020
:10F18000C8009600640032001900FFFF0000FF0372
:10F19000FF07FF0BFF0FFF13FF17FF1BFF1FFF23CF
:10F1A000FF27FF2BFF2FFF33FF37FF3BFF3FFFFF03
:10F1B000010201010201010102010101020101003C
:10F1C000010101020001010201010101010102002E
:10F1D000010102010102010101020100010201011C
:10F1E000020101010000000102010102010101010F
:10F1F00000000102010102010100020202010201FC
:10F2000001020100020202020102010102000102E8
:10F2100002020201020101000000020202020102D8
:10F2200001010100000202020201020100020202C9
:10F2300002020202010200020201020202020201B3
:10F2400001000202020202020202010000020200A8
:10F250000202020202000201020202020202020291
:10F260000002000202020202020202FF0000D007B6
:10F27000800CD80E0010C012EC130C17FA19141ED3
:10F280006022AC265C2B0C30BC34023AFF3FFFFFFF
:10F290000000580246056608540BD80E5C12701721
:10F2A000FC21F82A70305834DC37663A8C3C803EBA
:10F2B000FF3FFFFF0000580246056608540BA00FF1
:10F2C000D4172823F82A442F643284354038663A0C
:10F2D0008C3C803EFF3FFFFF2C011301FA00E10050
:10F2E000C800AF0096007D0064004B00320019009A
:10F2F00000000000CDCC4C3DCDCCCC3D9A99193EC0
:10F30000CDCC4C3E0000803E9A99993E3333B33EBB
:10F31000CDCCCC3E6666E63E000000000700000053
:10F320000C00000010000000130000001600000098
:10F330001800000000000000070000000C000000A2
:10F3400013000000180000001F000000240000004F
:10F35000000000000C000000180000002400000065
:10F36000300000003C0000004800000000000000E9
:10F37000FBFFFFFFF4FFFFFFEFFFFFFFE8FFFFFFD3
:10F38000E3FFFFFFDCFFFFFF00000000F4FFFFFFD3
:10F39000E8FFFFFFDCFFFFFFD0FFFFFFC4FFFFFF21
:10F3A000B8FFFFFF00007805220B0410B4143219D7
:10F3B000B01DFC214826FE29822D383126344637DF
:10F3C000663A223DFF3FFFFF0000D007100E881372
:10F3D0003219AA1E282374275C2B442F64328435EB
:10F3E0004038663A8C3C803EFF3FFFFF0000540BE4
:10F3F000EC13FA1908201C253629EC2C0C302C3380
:10F40000E8357238663AF63B863D163FFF3FFFFF10
:10F410000000CC10581BFC21AC26C62A7C2E3831AB
:10F42000F4334C36A438983A5A3C543D803E7A3FE7
:10F43000FF3FFFFFA4F40000FA9BFF1F0000FF0F37
:10F44000A09DFF1F0000FF0F613B000070F4000053
:10F450009C9DFF1F32005E010000000000000000C4
:10F46000013B000054485200534E53004D41580098
:10F47000544F5543482053454E5345004558545228
:10F480004120434F4E54524F4C4C45520000000017
:10F4900050495443482042454E4400004249544597
:10F4A0000000000042524541544800FF7CF4000037
:10F4B000F49CFF1FF401A00FEE9CFF1FF401A00FAE
:10F4C0000D3B00009CF40000B29BFF1FBC025C12CD
:10F4D000749DFF1FBC025C12453B000090F40000CD
:10F4E000469DFF1FF401A00F809BFF1FF401A00F9A
:10F4F000293B0000D4FC0000DCFC0000C8FC00003C
:10F50000CCFC0000D0FC00006CFB00008CFC000078
:10F51000A8FC0000ACFC0000B0FC0000B4FC000043
:10F52000B8FC0000BCFC0000C0FC000094FC000023
:10F53000C4FC00006CFB000068FB00009CFC0000A9
:10F54000A0FC0000A4FC00006CFB00008CFC000090
:10F5500090FC000094FC000098FC000078FC000087
:10F560007CFC000080FC000084FC000088FC0000A3
:10F5700068FC00006CFC000070FC000078010100D9
:10F5800074FC0000E4FC0000E8FC0000ECFC00005F
:10F59000F0FC0000F4FC0000F8FC0000FCFC0000A3
:10F5A00000FD000004FD000008FD00000CFD00004F
:10F5B00010FD000014FD00000100000018FD000017
:10F5C000070000000000000001000000A948000042
:10F5D00090FE00000000050108000000948DFF1F50
:10F5E000D94700000600000009000000188FFF1F27
:10F5F0000000000080FF000074FF0000589DFF1F06
:10F600000000300000000000B9550000E546000091
:10F61000000000001CFE00000000010108000000C6
:10F62000B08EFF1F7CFD0000000002010C000000F6
:10F63000608FFF1F0000000050FF00005CFF000013
:10F64000949BFF1F0000010001000000A94B000077
:10F6500019450000000000000100000098FE0000B5
:10F660000600000018FD000000000405080000006E
:10F67000AC8BFF1F0100000090FE0000090000009D
:10F6800000000000010000006D61000001000000AA
:10F69000B8FE0000030000000000000098FF00001A
:10F6A00074FF0000549DFF1F0000300000000000A8
:10F6B000B9550000E5460000000000000000000011
:10F6C000010000004D52000000000000C0FE0000DC
:10F6D000C8FE0000FC9CFF1F010010000600000097
:10F6E000A55D000039450000B14F0000000000009A
:10F6F00068FF000074FF00005A9DFF1F00003000EB
:10F7000000000000B9550000E546000000000000C0
:10F7100000000000000000000000000000000000E9
:10F7200000000000000000000000000000000000D9
:10F7300000000000000000000000000000000000C9
:10F7400000000000000000000000000000000000B9
:10F7500000000000000000000000000000000000A9
:10F760000000000000000000000000000000000099
:10F770000000000000000000000000000000000089
:10F780000000000000000000000000000000000079
:10F790000000000000000000000000000000000069
:10F7A0000000000000000000000000000000000059
:10F7B0000000000000000000000000000000000049
:10F7C0000000000000000000000000000000000039
:10F7D0000000000000000000000000000000000029
:10F7E0000000000000000000000000000000000019
:10F7F0000000000000000000000000000000000009
:10F8000000000000000000000000000000000000F8
:10F8100000000000000000000000000000000000E8
:10F8200000000000000000000000000000000000D8
:10F8300000000000007FFFFF000003F9FFFFFC0055
:10F8400000000000007FFFFF800007F9FFFFFE00BF
:10F850000000000000600001C0000E1980000700D9
:10F8600000000000006FFFFCC0001DD9BFFFF300C7
:10F8700000000000006FFFFEC0003BD9BFFFFB008F
:10F8800000000000006C0006C00077D9B0001B002B
:10F8900000000000006C0006C000EED9B0001B00A4
:10F8A00000000000006C0006C001DCD9B0001B00A5
:10F8B00000000800006C0006C003B8D9B0001B00AF
:10F8C00000001800006FFFFEC0077FD9B0001B00CA
:10F8D00000001800006FFFFCC00EFFD9B0001B0035
:10F8E00000C0180000600001C01C0019B0001B001F
:10F8F00000C03800006FFBFF803BFFD9B0001B0049
:10F9000000C03000006FFDFF0077FFD9B0001B0082
:10F9100001E03000006C0EE000EE00D9B0001B00EA
:10F9200001E03000006C077001DC00D9B0001B0062
:10F9300001B03000006C03B803B800D9B0001B0060
:10F9400001B03000006C01DC077000D9B0001B0072
:10F95000019820C0406C00EE0EE000D9B0001B0002
:10F96000030C20C0C06C00771DC000D9BFFFFB0096
:10F97000030C20C0C06C003BBB8000D9BFFFF3006C
:10F98000030620C1C06C001DF70000D980000700ED
:10F9900003032083806C000EEE0000D9FFFFFE0001
:10F9A0000303B183806C00075C0000D9FFFFFC00FB
:10F9B0000301F1878000000000000000000000004B
:10F9C0000300F18D80000000000000000000000036
:10F9D000030071B98000000000000000000000007A
:10F9E000030031F180000000000000000000000072
:10F9F000030000C1800000000000000000000000C3
:10FA000003000000000000000000000000000000F3
:10FA100003000000000000000000000000000000E3
:10FA200002000000000000000000000000000000D4
:10FA300000000000000000000000000000000000C6
:10FA400000000000000000000000000000000000B6
:10FA500000000000000000000000000000000000A6
:10FA60000000000000000000000000000000000096
:10FA70000000000000000000000000000000000086
:10FA80000000000000000000000000000000000076
:10FA90000000000000000000000000000000000066
:10FAA0000000000000000000000000000000000056
:10FAB0000000000000000000000000000000000046
:10FAC0000000000000000000000000000000000036
:10FAD0000000000000000000000000000000000026
:10FAE0000000000000000000000000000000000016
:10FAF0000000000000000000000000000000000006
:10FB000000000000000000000000000000000000F5
:10FB100040FF000000000301060000007C8DFF1F75
:10FB200000000000A4FF000074FF0000789BFF1F8E
:10FB30000000300000000000A95500002945000029
:10FB4000000000000000000074FD000040FD000007
:10FB5000689BFF1F0000090000000000CD4B000063
:10FB600059450000000000004F4E00004F4646007F
:10FB700055534200424154004C4F572000000000B2
:10FB80004D454E5520202020202020202058585818
:10FB900020592E595600000058000000524F5400C2
:10FBA0004D454C0044594E006D73000042544800CE
:10FBB000424954004C5652004E524D005245560098
:10FBC000312F0000415400004D4F4400504244008A
:10FBD00045434200454353004C564C004C565000A0
:10FBE000474C440045434800762E0000312E342E09
:10FBF0003600000053455400434C52004E755241AC
:10FC0000440000006669726D7761726520762E008F
:10FC100055534220706F776572000000416C6B6134
:10FC20006C696E6520626174746572790000000011
:10FC300030202520617420004E694D482062617497
:10FC400074657279000000004C69506F2062617425
:10FC50007465727900000000444F4E275400000084
:10FC600050414E4943000000455749004557580050
:10FC70005341580045565200484D530035544800F2
:10FC80004F43540035444E004F444E004D57000042
:10FC900046500000434600005350000053570000F8
:10FCA00053454C005345450042520000564C00005D
:10FCB000455800004D572B0042522B00564C2B004C
:10FCC00045582B00554E4F00414C4B004E4D4800BF
:10FCD0004C495000425254480000000050544348E0
:10FCE000000000002D3400002D3300002D320000F4
:10FCF0002D3100004C494E002B3100002B3200000A
:10FD00002B3300002B34000053310000533200002D
:10FD10005A3100005A3200005649425241544F00B5
:10FD2000444952454354494F4E000000434F4E54FE
:10FD3000524F4C00535155454C434820420000005F
:10FD40004C4556454C00000053454E534520425407
:10FD500045000000535155454C4348204C000000DD
:10FD600053454E5345204C565200000052455455C1
:10FD7000524E00004445505448000000534554552D
:10FD800050204354524C5300455854524120504B3C
:10FD90004559000046494E474552494E470000002C
:10FDA0004C4556454C204343000000004D4F442035
:10FDB0004B4559004445474C495443480000000016
:10FDC0004841524D2053454C0000000053455249D4
:10FDD0004553000045584354204841524D0000000F
:10FDE0004841524D2052414E47450000455843542A
:10FDF0002043432042000000455843542043432001
:10FE000041000000504954434842454E4400000020
:10FE1000504F52542F474C44000000005345545556
:10FE200050204252454154480000000056454C20A5
:10FE3000424F4F535400000056454C2044454C411E
:10FE400059000000435552564500000056454C4F9E
:10FE50004349545900000000425245415448204152
:10FE60005400000043432042205249534500000003
:10FE7000425254482043432042000000425254481A
:10FE8000204343204100000041424F5554000000F0
:10FE90004558545241530000524F5441544F520060
:10FEA00053455455502043544C000000534554557D
:10FEB000502042520000000041444A555354000073
:10FEC0004D494449204348004D4944492043484E48
:10FED0004C0000004241542054595045000000009D
:10FEE000574C204348414E00574C20504F574552E5
:10FEF000000000004641535420424F4F5400000080
:10FF0000444143204F55540053504543204B4559DD
:10FF1000000000004C454741435920425200000078
:10FF20004C45474143592050420000004F43544143
:10FF3000564500005452414E53504F534500000067
:10FF4000524F5441544F52205345545550000000D5
:10FF50005052494F52495459000000004D4F4E4FE6
:10FF6000205052494F000000524F54415445203414
:10FF70000000000053454D49544F4E4553000000CA
:10FF8000524F54415445203300000000524F544119
:10FF90005445203200000000524F54415445203156
:10FFA00000000000504152414C4C454C00FFFFFF07
:10FFB00001000000ACFE0000040000002C01000065
:10FFC000000000008CFF000074FF0000569DFF1F22
:10FFD0000000300000000000B9550000E5460000B8
:10FFE0000000000001000000A0FE0000050000006D
:10FFF0000000000044FE000044FE00006C9BFF1F58
:020000021000EC
:1000000000000C0003000000C95C0000494500002E
:10001000000000000100000088FE00000800000051
:100020000021110202000000002111020504FFFF5F
:10003000003E7FFF4E754556496330310000000099
:100040007676764E75455649636363007676764ECE
:10005000754556496330346565767676767676767C
:1000600076000000496E76616C696420636F6E668D
:10007000696720666F726D6174000000496E766179
:100080006C696420636865636B73756D00000000C4
:10009000496E76616C696420636F6E666967207370
:1000A000697A6500496E76616C696420636F6E667B
:1000B00069672076657273696F6E00004E754556EC
:1000C00049000000496E76616C6964206D65737348
:1000D0006167652E0000000065303000633030003D
:1000E00053656E64696E6720636F6E6669672E2E56
:1000F0002E000000436F6E6669672073656E742E74
:10010000000000006330330053656E64696E672041
:1001100076657273696F6E2E0000000063303200E6
:10012000526563656976696E6720636F6E6669679D
:100130002E2E2E004E657720636F6E6669672073E2
:10014000617665642E000000556E6B6E6F776E20D1
:100150006D6573736167652E0000000065303100C6
:10016000436F6E666967206D676D7400506F7765C9
:1001700072206F6666204E7545564900746F206583
:100180007869740052656164792E00FF3480044000
:10019000400000001211FFFFFF02020000001310D8
:1001A000FFFFFF020200000018000000348004403E
:1001B000800000001EFFFFFFFF02000000001DFF87
:1001C000FFFFFF0200000000190000000000000017
:1001D00000000000757D0000397D0000ED7C00000E
:1001E000357D0000F17C0000FD7C00001D7D0000DD
:1001F000000103070F1F3F7F2200FF2100FFFFFFC9
:100200000080C0E0F0F8FCFE0000000000000000EC
:10021000CD9C000029A10000ED7C0000F9860000C3
:100220009187000075950000299500005D950000FC
:100230003595000049950000459400007595000033
:100240009D9500008D890000D591000071910000FE
:100250006D96000079950000D1960000719700001E
:10026000DA02818FDA1281FF0000600000000000D6
:10027000000000000000000000E00000000000009E
:100280000000000000000001E0000000000000008D
:1002900000000000000001F000000000000000006D
:1002A000000000000003F00000000000000000005B
:1002B0000000000007F00000000000000000000047
:1002C00000000007F800000000000000000000002F
:1002D00000000FF800000003C0007E000001E000F5
:1002E0007F0FF800000003C000FE000001E000FFE7
:1002F000EFF800000003C000FE000001E000FFFF77
:10030000F800000003C000F00000000F007FFE7F37
:10031000C0000003C000F00000000F003FFE7FF8A7
:100320003FF1FBCFFCFEF3BC3DEFE01FFE7FFF7F04
:10033000FBFFDFFEFEFFBC3DEFE01FC6FFFF7FFBC4
:10034000FFDFFEFEFFBC3DEFE00FE3C7FE787BC39F
:10035000DE1EF0FFBC3DEF0007FF87FC787BC3DEAD
:100360001EF0F83C3DEF0001FFFFF0007BC3C01E14
:10037000F0F03C3DEF0001F37FE03FFBC3CFFEF028
:10038000F03C3DEF0003E33F807FFBC3DFFEF0F076
:100390003C3DEF0007E73C00787BC3DE1EF0F03CFD
:1003A0003DEF0007FFBE00787BC3DE1EF0F03C3D52
:1003B000EF0007FFFE00787BC3DE1EF0F03C3DEF50
:1003C000000FFFFE007FFBFFDFFEF0F03FFDEFE0E0
:1003D0000FFFFF007FFBFFDFFEF0F03FFDEFE00FC0
:1003E000F9FF003E79F9CF9EF0F01F3DE7E01FF1E5
:1003F000FF0000000000000000000000001F80FF60
:10040000007FFFFFFFFFFFFFFFFFFFE01C007F00FB
:100410007FFFFFFFFEB46D888D18E000001F007F96
:10042000FFFFFFFE95AD7DB577E000000F007FFF79
:10043000FFFFFEA5AD9D8D19E0000006007FFFFFC8
:10044000FFFEB5ADEDB57EE0AED580A8D300408D02
:100450002000A1C8DB40A4A62EAFFFFF00000000D3
:100460000001800000000000000000000380000088
:100470000000000000000007C000000000000000B5
:10048000000007C00000000000000000000FC000D6
:1004900000000000000000001FE00000000000005D
:1004A0000000001FE00000000000000000003FE02E
:1004B0000000000000000000003FF000000000000D
:1004C000000000007FF0000000000000001FF87F27
:1004D000F0000000000000003FFE7FF00000000080
:1004E0000000003FFF7FF0000000000000001FFF41
:1004F000FBE0000000000000000FFFF9FFC000005B
:10050000000000000FFFF9FFF800000000000007E6
:10051000FFF1FFFF00000000000003FC73FFFF80FD
:10052000000000000001FE3FFFFF8000000000000F
:1005300000FF1E0FFF000000000000007FFE1FFCF8
:10054000000000000000003FFFFFF8000000000076
:1005500000000FDFFFE0000000000000001F19FF97
:10056000C0000000000000003F3CFF000000000051
:100570000000007E7CF800000000000000007FFE0C
:100580007C0000000000000000FFFFFC00000000F5
:1005900000000000FFFFFE0000000000000000FF60
:1005A000FFFE0000000000000001FFEFFE00000061
:1005B0000000000001FFCFFE00000000000000036B
:1005C000FF07FE0000000000000003FC07FE000023
:1005D000000000000003F003FE0000000000000027
:1005E000018000FE000000000000000000007E000E
:1005F0000000000000000000003E000000000000BD
:10060000000000000C000000000000078000FC005B
:100610000003C0000000078001FC000003C00000D0
:1006200000078001FC000003C0000000078001E01B
:100630000000001E000000078001E00000001E0016
:100640007FE3F79FF9FDE7787BDFC0FFF7FFBFFD92
:10065000FDFF787BDFC0FFF7FFBFFDFDFF787BDF8D
:10066000C0F0F787BC3DE1FF787BDE00F0F787BC88
:100670003DE1F0787BDE0000F787803DE1E0787BAC
:10068000DE007FF7879FFDE1E0787BDE00FFF787E4
:10069000BFFDE1E0787BDE00F0F787BC3DE1E0786C
:1006A0007BDE00F0F787BC3DE1E0787BDE00F0F711
:1006B00087BC3DE1E0787BDE00FFF7FFBFFDE1E0B6
:1006C0007FFBDFC0FFF7FFBFFDE1E07FFBDFC07C0A
:1006D000F3F39F3DE1E03E7BCFC00000000000004F
:1006E0000000000000FFFFFFFFFFFFFFFFFFFFC054
:1006F000FFFFFFFFFD68DB111A31C0FFFFFFFFFDA9
:100700002B5AFB6AEFC0FFFFFFFFFD4B5B3B1A3329
:10071000C0FFFFFFFFFD6B5BDB6AFDC0DA0281FFFC
:100720000000000000000000CD9C000029A1000096
:10073000ED7C0000F9860000ADA800007595000072
:10074000299500005D950000359500004995000051
:1007500045940000759500009D9500009995000056
:10076000C1950000199600006D9600007995000073
:10077000D19600007197000000000000003E5B4F22
:100780005B3E3E6B4F6B3E1C3E7C3E1C183C7E3CF1
:10079000181C577D571C1C5E7F5E1C00183C1800FF
:1007A000FFE7C3E7FF0018241800FFE7DBE7FF308F
:1007B000483A060E2629792926407F050507407FFD
:1007C00005253F5A3CE73C5A7F3E1C1C08081C1C70
:1007D0003E7F14227F22145F5F005F5F06097F0166
:1007E0007F006689956A606060606094A2FFA29451
:1007F00008047E040810207E201008082A1C08081F
:100800001C2A08081E101010100C1E0C1E0C30386C
:100810003E3830060E3E0E06000000000000005F6D
:1008200000000007000700147F147F14242A7F2A89
:10083000122313086462364956205000080703004B
:10084000001C2241000041221C002A1C7F1C2A0897
:10085000083E0808008070300008080808080000FA
:1008600060600020100804023E5149453E00427F6E
:10087000400072494949462141494D331814127FBD
:100880001027454545393C4A49493141211109075D
:100890003649494936464949291E000014000000DE
:1008A00040340000000814224114141414140041B0
:1008B00022140802015909063E415D594E7C12116D
:1008C000127C7F494949363E414141227F414141A5
:1008D0003E7F494949417F090909013E4141517320
:1008E0007F0808087F00417F41002040413F017F91
:1008F000081422417F404040407F021C027F7F0459
:1009000008107F3E4141413E7F090909063E4151A1
:10091000215E7F09192946264949493203017F0191
:10092000033F4040403F1F2040201F3F4038403F92
:10093000631408146303047804036159494D4300A8
:100940007F4141410204081020004141417F0402DF
:100950000102044040404040000307080020545476
:1009600078407F2844443838444444283844442854
:100970007F385454541800087E090218A4A49C78A7
:100980007F0804047800447D40002040403D007F03
:100990001028440000417F40007C047804787C08E3
:1009A0000404783844444438FC18242418182424B7
:1009B00018FC7C08040408485454542404043F449C
:1009C000243C4040207C1C2040201C3C4030403CCB
:1009D00044281028444C9090907C4464544C44002B
:1009E000083641000000770000004136080002018F
:1009F0000204023C2623263C1EA1A161123A40407B
:100A0000207A3854545559215555794122545478F7
:100A100042215554784020545579400C1E52721290
:100A20003955555559395454545939555454580019
:100A300000457C410002457D420001457C407D121D
:100A400011127DF0282528F07C545545002054547F
:100A50007C547C0A097F4932494949323A4444442A
:100A60003A324A4848303A4141217A3A4240207865
:100A7000009DA0A07D3D4242423D3D4040403D3C66
:100A800024FF2424487E4943662B2FFC2F2BFF098B
:100A900029F620C0887E090320545479410000447F
:100AA0007D413048484A32384040227A007A0A0A6A
:100AB000727D0D19317D2629292F282629292926DD
:100AC00030484D4020380808080808080808382F22
:100AD00010C8ACBA2F102834FA00007B00000814AC
:100AE0002A142222142A14085500550055AA55AA82
:100AF00055AAFF55FF55FF000000FF00101010FF22
:100B000000141414FF001010FF00FF1010F010F07C
:100B1000141414FC001414F700FF0000FF00FF146D
:100B200014F404FC141417101F10101F101F1414B9
:100B3000141F00101010F0000000001F1010101003
:100B40001F10101010F010000000FF1010101010F7
:100B500010101010FF10000000FF140000FF00FF35
:100B600000001F10170000FC04F4141417101714D1
:100B700014F404F40000FF00F714141414141414F3
:100B8000F700F7141414171410101F101F14141466
:100B9000F4141010F010F000001F101F0000001FD0
:100BA00014000000FC140000F010F01010FF10FF03
:100BB000141414FF141010101F00000000F010FF98
:100BC000FFFFFFFFF0F0F0F0F0FFFFFF000000007C
:100BD00000FFFF0F0F0F0F0F3844443844FC4A4A00
:100BE0004A347E02020606027E027E0263554941B5
:100BF000633844443C04407E201E2006027E0202EC
:100C000099A5E7A5991C2A492A1C4C7201724C30FF
:100C10004A4D4D303048784830BC625A463D3E49D6
:100C20004949007E0101017E2A2A2A2A2A44445F7A
:100C3000444440514A444040444A51400000FF016E
:100C400003E080FF000008086B6B0836123624367C
:100C5000060F090F060000181800000010100030E1
:100C600040FF0101001F01011E00191D1712003C69
:100C70003C3C3C00000000000D0AFFFF050E080987
:100C80000D0C06070F0400130393050E08090D0C45
:100C900006070F04FFFFC585848687C4FFFF001386
:100CA00003931A9217FFFFFF6FF07F03037003781F
:100CB00013F0800FFBD070474008FE4340A0044073
:100CC0004408FE4344A004400018FE4300C0044012
:100CD0003000FE43309004403400FE433490044022
:100CE0001C18FE431CC004401018FE4310C00440F2
:100CF0000818FE4308C004400C18FE430CC0044012
:100D00000C10FE430CB004401010FE4310B0044021
:100D10001810FE4318B004401C10FE431CB00440E1
:100D20001410FE4314B004400418FE4304C00440F1
:100D30000010FE4300B004400008FE4300A0044041
:100D40000408FE4304A004400C08FE430CA0044029
:100D50000808FE4308A004401418FE4314C00440D1
:100D60001818FE4318C004400410FE4304B00440A9
:100D70000810FE4308B004401400FE4314900440E1
:100D80004C08FE434CA004400420FE4304D0044021
:100D90002410FE4324B004402010FE4320B0044041
:100DA0002810FE4328B004402C10FE432CB0044011
:100DB0000020FE4300D004404808FE4348A0044001
:100DC0001000FE4310900440090AFFFFFFFFFFFFE1
:100DD000FFFFFFFFFFFFFF0D00060807FFFF0E0FDD
:100DE000FF0CFFFFFFFFFFFF0B05FFFF1519151994
:100DF00000010000FC91FF1F120000000002000033
:100E00002892FF1F73000000002201009C92FF1F28
:100E100021000000002101008492FF1F0900000052
:100E200000030000C092FF1F00000000010309043E
:100E30001092FF1F00000000020309040C90FF1F26
:100E40000000000003030904C492FF1F000000001B
:100E50000000000000000000000000006578700045
:100E6000000000000000E03F000000000000E0BFC4
:100E7000763C7935EF39EA3D763C7935EF39EABD94
:100E80000000E0FE422EE63F0000E0FE422EE6BFFC
:100E9000E092FF1FF8B500BFF8BC08BC9E46704743
:100EA00089ED000035040000A53A000061560000FD
:040EB000697900005C
:040EB400F8B500BFCE
:100EB80038B5084B1C681C6054B1074D94FAA4F36C
:100EC800B3FA83F355F823309847631E1C40F5D1D5
:100ED80038BD00BFA0D00440EC91FF1F38B5084BC7
:100EE8001C681C6054B1074D94FAA4F3B3FA83F359
:100EF80055F823309847631E1C40F5D138BD00BF14
:100F0800A0C00440CC91FF1F38B5084B1C681C607A
:100F180054B1074D94FAA4F3B3FA83F355F8233088
:100F28009847631E1C40F5D138BD00BFA0B00440EF
:100F38009C91FF1F38B5084B1C681C6054B1074DC5
:100F480094FAA4F3B3FA83F355F823309847631E51
:100F58001C40F5D138BD00BFA0A004404C91FF1F34
:100F680038B5084B1C681C6054B1074D94FAA4F3BB
:100F7800B3FA83F355F823309847631E1C40F5D124
:100F880038BD00BFA09004401491FF1F000000006E
:100F9800002000000000F041280000000C000000C4
:100FA8005A000000F3FFFFFFDFFFFFFFA3FFFFFF73
:100FB800AEFFFFFF73000000760000000200000093
:100FC80004000000D8FFFFFFB5FFFFFFA2FFFFFFEF
:100FD80002000000FBFFFFFF00000000000000000F
:100FE80000000000000000000000000000000000F9
:100FF80000000000000000000100000000200000C8
:101008000020000000100000AB0A000000080000EB
:101018006606000055050000920400000004000068
:101028008E03000033030000E8020000AB0200005A
:101038000020000014050000000102070B01020750
:101048000B4A140002000C0024000000A8FFFFFF58
:10105800BCFFFFFFE1FFFFFF0D00000004000000E0
:101068007800000079000000BCFFFFFFABFFFFFF26
:10107800DEFFFFFF1700000057000000100000000F
:101088000A00000008000000150000001800000019
:10109800290000000200FFFFFFFF000034F40000F9
:1010A800C4F40000DCF40000ACF400004CF40000D0
:1010B8000000000088FD000088FD0000C89DFF1F9B
:1010C80000001900000000000000000000000000FF
:1010D800000000000000000020FD000020FD0000CE
:1010E800E09BFF1F0000010001000000000000005D
:1010F8000000000000000000000000002CFD0000BF
:101108002CFD0000EA9CFF1F000002000100000007
:1011180000000000000000000000000000000000C7
:1011280054FD000040FD0000D689FF1F01001E008D
:1011380000000000000000000000000000000000A7
:10114800010000000000000094FD000094FD000074
:10115800449BFF1F00000400010000000000000085
:1011680000000000000000000000000010FE000069
:1011780010FE0000FE9BFF1F00000400010000009D
:101188000000000000000000000000000000000057
:10119800C0FD0000CCFD00006C9DFF1F0000040096
:1011A8000100000000000000000000000000000036
:1011B80000000000A0FD0000A0FD0000CC9BFF1F68
:1011C80000007F0001000000000000000000000097
:1011D800000000000000000048FD000040FD000085
:1011E800248AFF1F01001100000000000000000019
:1011F80000000000000000000000000058FE000091
:1012080058FE0000F29BFF1F0000010001000000D3
:10121800000000000000000000000000888AFF1F96
:1012280044FB0000908FFF1F648AFF1FF08BFF1F95
:10123800AC8AFF1F648BFF1F8C8EFF1F000000000D
:101248007CFE00007CFE0000389DFF1F00000A00A5
:101258000100000000000000000000000000000085
:101268000000000060FD000040FD0000D489FF1F61
:1012780001000C0000000000000000000000000059
:10128800000000000000000014FF000014FF000030
:10129800EE9BFF1F0000010001000000000000009D
:1012A80000000000000000000000000038FE000000
:1012B80038FE0000EC9BFF1F00001E00010000002C
:1012C8000000000000000000000000000000000016
:1012D80064FE000064FE0000549BFF1F01000A002A
:1012E80001000000000000000000000000000000F5
:1012F80000000000F4FE0000F4FE0000429DFF1F05
:1013080000000100000000000000000000000000D4
:10131800000000000000000004FE000004FE0000C1
:101328009E9BFF1F00000C00000000000000000052
:1013380000000000000000000000000008FF00009E
:1013480008FF00004E9DFF1F000001000100000083
:101358000000000000000000000000000000000085
:10136800E0FE0000E0FE0000E48FFF1F04005000D4
:101378000000000000000000000000000000000065
:1013880000000000E8FE0000E8FE00004C9EFF1F81
:101398000000030000000000000000000000000042
:1013A800000000000000000034FF000034FF0000CF
:1013B800589BFF1F000018000000000000000000FC
:1013C8000000000000000000000000002CFE0000EB
:1013D8002CFE0000489BFF1F0000090001000000D0
:1013E80000000000000000000000000020FB0000DA
:1013F80098F60000C0FF0000F0F50000ECF60000D1
:1014080034F60000D88DFF1F148CFF1FC88CFF1FF7
:10141800E88FFF1F448EFF1F808CFF1F108DFF1F5A
:10142800EC8CFF1F00000000D4FD0000E0FD000070
:10143800A49DFF1F0000060001000000000000003E
:1014480000000000000000000000000020FF000075
:1014580020FF0000B09BFF1F0000010001000000FA
:101468000000000000000000000000000000000074
:10147800ACFD0000ACFD0000769DFF1F00001E00C3
:101488000000000000000000000000000000000054
:1014980000000000F8FD0000F8FD0000969BFF1F0B
:1014A800000004000100000000000000000000002F
:1014B8000000000000000000D4FE0000D4FE000080
:1014C800DE9CFF1F00000200010000000000000079
:1014D8000000000000000000000000002CFF0000D9
:1014E8002CFF0000509DFF1F0000060000000000B8
:1014F80000000000000000000000000000000000E4
:1015080034FD000040FD00002C89FF1F01001E0073
:1015180000000000000000000000000000000000C3
:10152800CC8BFF1FD08EFF1F5C8CFF1F888BFF1F8B
:101538003C8FFF1FF0FF0000388CFF1F588DFF1FE6
:101548000000000070FE000070FE00007A9DFF1F82
:1015580000007F0001000000000000000000000003
:101568000000000000000000B4FD0000B4FD000011
:10157800869DFF1F000046000000000000000000DC
:101588000000000000000000348DFF1F688EFF1F60
:10159800C8F600008CF60000B0FF0000E4FF000071
:1015A80058F6000074F60000140001000000000066
:1015B8004CFE00004CFE00005C9BFF1F00007F00FB
:1015C8000100000000000000000000000000000012
:1015D800F88AFF1F208EFF1FC08FFF1FB48DFF1FCB
:1015E8001C8BFF1FB8F50000F48EFF1FFC8DFF1F3A
:1015F800408BFF1F408AFF1FD48AFF1FA48CFF1F48
:10160800000000006CFD000040FD00006089FF1F25
:1016180000000400000000000000000000000000BE
:1016280000000000000000000100000000000000B1
:1016380000000000ECFD0000ECFD0000889DFF1F8D
:1016480000007F0001000000000000000000000012
:1016580000000000040000000000000000FF00007F
:1016680000FF00004C9DFF1F00000100000000006B
:1016780000000000000000000000000016034E00FB
:10168800750045005600490020004D0049004400FF
:1016980049000000D401010000000000E803000038
:1016A80000000000006006408C01010000000000FE
:1016B8000000000000000000000000000000000022
:1016C8000000000000000000000000000000000012
:1016D8000000000000000000000000000000000002
:1016E80000000000000000000000000000000000F2
:1016F80000000000000000000000000000000000E2
:10170800D401010000000000E80300000000000010
:1017180000700640AC01010000000000000000005D
:1017280000000000000000000000000000000000B1
:1017380000000000000000000000000000000000A1
:101748000000000000000000000000000000000091
:101758000000000000000000000000000000000081
:10176800000000000000000000000000FD9F0000D5
:10177800FD9F0000FD9F0000FD9F00000A0400007F
:1017880004A3FF1F39A9000039A9000039A90000E6
:1017980039A9000039A9000039A9000039A90000B9
:1017A80039A9000039A9000039A9000039A90000A9
:1017B80039A9000039A9000039A9000039A9000099
:1017C80039A9000039A9000039A9000039A9000089
:1017D80039A9000039A9000039A9000039A9000079
:1017E80039A9000039A9000039A9000039A9000069
:1017F80039A9000039A9000039A9000039A9000059
:1018080039A9000039A9000039A9000039A9000048
:1018180039A9000039A9000039A9000039A9000038
:1018280039A9000039A9000039A9000039A9000028
:1018380039A9000039A9000039A9000039A9000018
:1018480039A9000039A9000039A9000039A9000008
:1018580039A9000039A9000039A9000039A90000F8
:1018680039A9000008000000FFFFFFFF1201100166
:1018780000000040C0168504750201020301000043
:1018880018035400650065006E0073007900640059
:10189800750069006E006F0009027300020100C044
:1018A8003209040000020103000007240100012599
:1018B8000006240201010006240202020009240392
:1018C80001030102010009240302040101010009C6
:1018D80005040240000000000525010101090583F7
:1018E800024000000000052501010309040100026F
:1018F80003000000092111010001222100070581D0
:1019080003400001070502032000020006C9FF0981
:1019180004A15C7508150026FF0095400975810231
:1019280095200976910295040976B102C00000005D
:10193800040309040C03000000000000000000007C
:10194800000000000000000000000100000000008E
:1019580000000000CC95FF1F3496FF1F9C96FF1FC8
:10196800000000000000000000000000000000006F
:10197800000000000000000000000000000000005F
:10198800000000000000000000000000000000004F
:10199800000000000000000000000000000000003F
:1019A800000000000000000000000000000000002F
:1019B800000000000000000000000000000000001F
:1019C800000000000000000000000000000000000F
:1019D80000000000000000000000000000000000FF
:1019E80000000000000000000000000000000000EF
:1019F80000000000000000000100000000000000DE
:101A08000E33CDAB34126DE6ECDE05000B000000A2
:101A180000000000000000000000000000000000BE
:101A280000000000000000000000000000000000AE
:101A3800000000000000000000000000000000009E
:101A4800000000000000000000000000000000008E
:101D78000000000000000000E092FF1F00000000CB
:101D8800000000000C97FF1F0C97FF1F1497FF1F00
:101D98001497FF1F1C97FF1F1C97FF1F2497FF1FF7
:101DA8002497FF1F2C97FF1F2C97FF1F3497FF1FA7
:101DB8003497FF1F3C97FF1F3C97FF1F4497FF1F57
:101DC8004497FF1F4C97FF1F4C97FF1F5497FF1F07
:101DD8005497FF1F5C97FF1F5C97FF1F6497FF1FB7
:101DE8006497FF1F6C97FF1F6C97FF1F7497FF1F67
:101DF8007497FF1F7C97FF1F7C97FF1F8497FF1F17
:101E08008497FF1F8C97FF1F8C97FF1F9497FF1FC6
:101E18009497FF1F9C97FF1F9C97FF1FA497FF1F76
:101E2800A497FF1FAC97FF1FAC97FF1FB497FF1F26
:101E3800B497FF1FBC97FF1FBC97FF1FC497FF1FD6
:101E4800C497FF1FCC97FF1FCC97FF1FD497FF1F86
:101E5800D497FF1FDC97FF1FDC97FF1FE497FF1F36
:101E6800E497FF1FEC97FF1FEC97FF1FF497FF1FE6
:101E7800F497FF1FFC97FF1FFC97FF1F0498FF1F95
:101E88000498FF1F0C98FF1F0C98FF1F1498FF1F42
:101E98001498FF1F1C98FF1F1C98FF1F2498FF1FF2
:101EA8002498FF1F2C98FF1F2C98FF1F3498FF1FA2
:101EB8003498FF1F3C98FF1F3C98FF1F4498FF1F52
:101EC8004498FF1F4C98FF1F4C98FF1F5498FF1F02
:101ED8005498FF1F5C98FF1F5C98FF1F6498FF1FB2
:101EE8006498FF1F6C98FF1F6C98FF1F7498FF1F62
:101EF8007498FF1F7C98FF1F7C98FF1F8498FF1F12
:101F08008498FF1F8C98FF1F8C98FF1F9498FF1FC1
:101F18009498FF1F9C98FF1F9C98FF1FA498FF1F71
